 gdi+

 Timestamp is 5b32b115 (Wed Jun 27 00:33:09 2018)

 Preferred load address is 0000000180000000

 Start         Length     Name                   Class
 0001:00000000 00010210H .text$mn                CODE
 0001:00010210 00000020H .text$mn$00             CODE
 0001:00010230 00000270H .text$x                 CODE
 0002:00000000 00000310H .idata$5                DATA
 0002:00000310 00000010H .00cfg                  DATA
 0002:00000320 00000008H .CRT$XCA                DATA
 0002:00000328 00000008H .CRT$XCZ                DATA
 0002:00000330 00000008H .CRT$XIA                DATA
 0002:00000338 00000018H .CRT$XIC                DATA
 0002:00000350 00000008H .CRT$XIZ                DATA
 0002:00000358 00000008H .CRT$XPA                DATA
 0002:00000360 00000010H .CRT$XPX                DATA
 0002:00000370 00000008H .CRT$XPXA               DATA
 0002:00000378 00000008H .CRT$XPZ                DATA
 0002:00000380 00000008H .CRT$XTA                DATA
 0002:00000388 00000008H .CRT$XTZ                DATA
 0002:00000390 00000000H .gfids$x                DATA
 0002:00000390 00000000H .gfids$y                DATA
 0002:00000390 00007db0H .rdata                  DATA
 0002:00008140 00000000H .rdata$r                DATA
 0002:00008140 00000300H .rdata$zzzdbg           DATA
 0002:00008440 00000008H .rtc$IAA                DATA
 0002:00008448 00000008H .rtc$IZZ                DATA
 0002:00008450 00000008H .rtc$TAA                DATA
 0002:00008458 00000008H .rtc$TZZ                DATA
 0002:00008460 00000d30H .xdata                  DATA
 0002:00009190 00000000H .xdata$x                DATA
 0002:00009190 00000094H .edata                  DATA
 0002:00009224 00000050H .idata$2                DATA
 0002:00009274 00000014H .idata$3                DATA
 0002:00009288 00000310H .idata$4                DATA
 0002:00009598 000006b8H .idata$6                DATA
 0003:00000000 00000900H .data                   DATA
 0003:00000900 00000000H .data$r                 DATA
 0003:00000900 000099b8H .bss                    DATA
 0004:00000000 00000ffcH .pdata                  DATA
 0005:00000000 000000a0H .rsrc$01                DATA
 0005:000000a0 00000490H .rsrc$02                DATA

  Address         Publics by Value              Rva+Base               Lib:Object

 0000:00000000       __guard_iat_table          0000000000000000     <absolute>
 0000:00000000       __dynamic_value_reloc_table 0000000000000000     <absolute>
 0000:00000000       __hybrid_code_map          0000000000000000     <absolute>
 0000:00000000       __hybrid_code_map_count    0000000000000000     <absolute>
 0000:00000000       __guard_iat_count          0000000000000000     <absolute>
 0000:00000000       __hybrid_auxiliary_iat     0000000000000000     <absolute>
 0000:00000000       __guard_longjmp_table      0000000000000000     <absolute>
 0000:00000000       __guard_longjmp_count      0000000000000000     <absolute>
 0000:00000000       __guard_fids_count         0000000000000000     <absolute>
 0000:00000000       __enclave_config           0000000000000000     <absolute>
 0000:00000000       ___safe_se_handler_table   0000000000000000     <absolute>
 0000:00000000       ___safe_se_handler_count   0000000000000000     <absolute>
 0000:00000000       __guard_fids_table         0000000000000000     <absolute>
 0000:00000100       __guard_flags              0000000000000100     <absolute>
 0000:00000000       __ImageBase                0000000180000000     <linker-defined>
 0001:00000000       ?CET_Cancel@@YAXPEAX@Z     0000000180001000 f   gdip.obj
 0001:00000018       ?CET_Done@@YAXPEAUCET_Init@@@Z 0000000180001018 f   gdip.obj
 0001:00000040       ?CET_Free@@YAXPEAUCET_LoadInfo@@@Z 0000000180001040 f   gdip.obj
 0001:000000e4       ?CET_Init@@YAHPEAU0@@Z     00000001800010e4 f   gdip.obj
 0001:00000174       ?CET_Load@@YAHPEAUCET_LoadInfo@@@Z 0000000180001174 f   gdip.obj
 0001:00000430       ?CalculateShowSize@GDIPlusImage@@QEAAXAEAH0000@Z 0000000180001430 f i gdip.obj
 0001:000005b0       ?Close@GDIPlusDecoder@@QEAAXXZ 00000001800015b0 f i gdip.obj
 0001:00000680       ?Close@GDIPlusImage@@QEAAXXZ 0000000180001680 f i gdip.obj
 0001:00000700       ?DrawImageAbortCallback@GDIPlusImage@@SAHPEAUGDIPlusDecoder@@@Z 0000000180001700 f i gdip.obj
 0001:0000070c       ?FreeThreadProc@GDIPlusDecoder@@SAKPEAX@Z 000000018000170c f i gdip.obj
 0001:0000072c       ?GetExifTagValueAsInt@GDIPlusImage@@QEAA_NKAEAH@Z 000000018000172c f i gdip.obj
 0001:0000080c       ?GetPageBits@GDIPlusImage@@QEAA_NPEAUCET_LoadInfo@@@Z 000000018000180c f i gdip.obj
 0001:00000d18       ?Init@GDIPlusDecoder@@QEAA_NPEAUCET_Init@@@Z 0000000180001d18 f i gdip.obj
 0001:00001024       ?Open@GDIPlusImage@@QEAA_N_NPEB_WPEBE_JU_COORD@@@Z 0000000180002024 f i gdip.obj
 0001:000013ec       ?SelectPage@GDIPlusImage@@QEAA_NI@Z 00000001800023ec f i gdip.obj
 0001:000014b8       ??2@YAPEAX_K@Z             00000001800024b8 f   common-kernel64:Memory.obj
 0001:000014ec       ??3@YAXPEAX@Z              00000001800024ec f   common-kernel64:Memory.obj
 0001:000014ec       ??_V@YAXPEAX@Z             00000001800024ec f   common-kernel64:Memory.obj
 0001:00001514       ??_U@YAPEAX_K@Z            0000000180002514 f   common-kernel64:Memory.obj
 0001:00001528       ?HeapDeinitialize@@YAXXZ   0000000180002528 f   common-kernel64:Memory.obj
 0001:0000154c       ?HeapInitialize@@YA_NXZ    000000018000254c f   common-kernel64:Memory.obj
 0001:00001580       ??$sprintf_c@$0CI@@@YAHAEAY0CI@DPEBDZZ 0000000180002580 f i common-kernel64:WThreads.obj
 0001:000015ac       ?SetThreadName@@YAXKPEAD@Z 00000001800025ac f   common-kernel64:WThreads.obj
 0001:000015e4       ?StringCchVPrintfA@@YAJPEAD_KPEBD0@Z 00000001800025e4 f i common-kernel64:WThreads.obj
 0001:0000168c       ?apiCreateThread@@YAPEAXP6AKPEAX@Z0PEAKPEBDH@Z 000000018000268c f   common-kernel64:WThreads.obj
 0001:000017e0       ?apiTerminateThreadEx@@YAHPEAXKPEBDH@Z 00000001800027e0 f   common-kernel64:WThreads.obj
 0001:000018e8       ?apiThreadHelper@@YAKPEAX@Z 00000001800028e8 f   common-kernel64:WThreads.obj
 0001:00001af4       __local_stdio_printf_options 0000000180002af4 f i common-kernel64:WThreads.obj
 0001:00001afc       ?sprintf_c@@YAHPEAD_JPEBDZZ 0000000180002afc f   common-kernel64:MStrSafe.obj
 0001:00001b3c       __raise_securityfailure    0000000180002b3c f   LIBCMT:gs_report.obj
 0001:00001b70       __report_gsfailure         0000000180002b70 f   LIBCMT:gs_report.obj
 0001:00001c44       __report_rangecheckfailure 0000000180002c44 f   LIBCMT:gs_report.obj
 0001:00001c58       __report_securityfailure   0000000180002c58 f   LIBCMT:gs_report.obj
 0001:00001dd8       __GSHandlerCheck           0000000180002dd8 f   LIBCMT:_gshandler_.obj
 0001:00001df8       __GSHandlerCheckCommon     0000000180002df8 f   LIBCMT:_gshandler_.obj
 0001:00001e70       __security_check_cookie    0000000180002e70 f   LIBCMT:_amdsecgs_.obj
 0001:000021b4       _DllMainCRTStartup         00000001800031b4 f   LIBCMT:dll_dllmain.obj
 0001:000021f4       ??3@YAXPEAX_K@Z            00000001800031f4 f   LIBCMT:delete_scalar_size.obj
 0001:000021fc       __security_init_cookie     00000001800031fc f   LIBCMT:gs_support.obj
 0001:000022ac       DllMain                    00000001800032ac f   LIBCMT:dll_dllmain_stub.obj
 0001:000022ac       _get_startup_argv_mode     00000001800032ac f   LIBCMT:argv_mode.obj
 0001:000022b4       ?__scrt_initialize_type_info@@YAXXZ 00000001800032b4 f   LIBCMT:tncleanup.obj
 0001:000022c4       ?__scrt_uninitialize_type_info@@YAXXZ 00000001800032c4 f   LIBCMT:tncleanup.obj
 0001:000022d0       __local_stdio_scanf_options 00000001800032d0 f i LIBCMT:default_local_stdio_options.obj
 0001:000022d8       __scrt_initialize_default_local_stdio_options 00000001800032d8 f   LIBCMT:default_local_stdio_options.obj
 0001:000022f4       __scrt_acquire_startup_lock 00000001800032f4 f   LIBCMT:utility.obj
 0001:00002330       __scrt_dllmain_after_initialize_c 0000000180003330 f   LIBCMT:utility.obj
 0001:00002364       __scrt_dllmain_before_initialize_c 0000000180003364 f   LIBCMT:utility.obj
 0001:0000237c       __scrt_dllmain_crt_thread_attach 000000018000337c f   LIBCMT:utility.obj
 0001:000023a4       __scrt_dllmain_crt_thread_detach 00000001800033a4 f   LIBCMT:utility.obj
 0001:000023bc       __scrt_dllmain_exception_filter 00000001800033bc f   LIBCMT:utility.obj
 0001:0000241c       __scrt_dllmain_uninitialize_c 000000018000341c f   LIBCMT:utility.obj
 0001:0000244c       __scrt_dllmain_uninitialize_critical 000000018000344c f   LIBCMT:utility.obj
 0001:00002460       __scrt_initialize_crt      0000000180003460 f   LIBCMT:utility.obj
 0001:000024ac       __scrt_initialize_onexit_tables 00000001800034ac f   LIBCMT:utility.obj
 0001:00002588       __scrt_is_nonwritable_in_current_image 0000000180003588 f   LIBCMT:utility.obj
 0001:00002624       __scrt_release_startup_lock 0000000180003624 f   LIBCMT:utility.obj
 0001:00002648       __scrt_uninitialize_crt    0000000180003648 f   LIBCMT:utility.obj
 0001:00002674       __scrt_get_dyn_tls_init_callback 0000000180003674 f   LIBCMT:dyn_tls_init.obj
 0001:0000267c       __crt_debugger_hook        000000018000367c f   LIBCMT:utility_desktop.obj
 0001:00002684       __scrt_fastfail            0000000180003684 f   LIBCMT:utility_desktop.obj
 0001:000027d0       _RTC_Initialize            00000001800037d0 f   LIBCMT:_initsect_.obj
 0001:0000280c       _RTC_Terminate             000000018000380c f   LIBCMT:_initsect_.obj
 0001:00002848       _guard_check_icall_nop     0000000180003848 f i LIBCMT:guard_support.obj
 0001:0000284c       __isa_available_init       000000018000384c f   LIBCMT:_cpu_disp_.obj
 0001:00002a08       __scrt_is_ucrt_dll_in_use  0000000180003a08 f   LIBCMT:ucrt_detection.obj
 0001:00002a20       wcsrchr                    0000000180003a20 f   libvcruntime:wcsrchr.obj
 0001:00002af0       memset                     0000000180003af0 f   libvcruntime:memset.obj
 0001:00002ca0       strchr                     0000000180003ca0 f   libvcruntime:strchr.obj
 0001:00002d2c       strrchr                    0000000180003d2c f   libvcruntime:strrchr.obj
 0001:00002e78       __C_specific_handler       0000000180003e78 f   libvcruntime:_riscchandler_.obj
 0001:00003084       __std_type_info_destroy_list 0000000180004084 f   libvcruntime:std_type_info.obj
 0001:000030b0       __vcrt_initialize          00000001800040b0 f   libvcruntime:initialization.obj
 0001:000030e4       __vcrt_thread_attach       00000001800040e4 f   libvcruntime:initialization.obj
 0001:000030f8       __vcrt_thread_detach       00000001800040f8 f   libvcruntime:initialization.obj
 0001:0000310c       __vcrt_uninitialize        000000018000410c f   libvcruntime:initialization.obj
 0001:0000312c       __vcrt_uninitialize_critical 000000018000412c f   libvcruntime:initialization.obj
 0001:00003150       _local_unwind              0000000180004150 f   libvcruntime:_jmpuwind_.obj
 0001:00003180       _NLG_Notify                0000000180004180 f   libvcruntime:_jmpuwind_.obj
 0001:000031a0       __NLG_Dispatch2            00000001800041a0 f   libvcruntime:_jmpuwind_.obj
 0001:000031b0       __NLG_Return2              00000001800041b0 f   libvcruntime:_jmpuwind_.obj
 0001:000031b4       __except_validate_context_record 00000001800041b4 f   libvcruntime:jbcxrval.obj
 0001:000031ec       __vcrt_freefls             00000001800041ec f   libvcruntime:per_thread_data.obj
 0001:0000320c       __vcrt_freeptd             000000018000420c f   libvcruntime:per_thread_data.obj
 0001:0000325c       __vcrt_getptd_noexit       000000018000425c f   libvcruntime:per_thread_data.obj
 0001:00003314       __vcrt_initialize_ptd      0000000180004314 f   libvcruntime:per_thread_data.obj
 0001:00003364       __vcrt_uninitialize_ptd    0000000180004364 f   libvcruntime:per_thread_data.obj
 0001:00003388       __vcrt_initialize_locks    0000000180004388 f   libvcruntime:locks.obj
 0001:000033d0       __vcrt_uninitialize_locks  00000001800043d0 f   libvcruntime:locks.obj
 0001:000035e0       __vcrt_FlsAlloc            00000001800045e0 f   libvcruntime:winapi_downlevel.obj
 0001:00003628       __vcrt_FlsFree             0000000180004628 f   libvcruntime:winapi_downlevel.obj
 0001:00003670       __vcrt_FlsGetValue         0000000180004670 f   libvcruntime:winapi_downlevel.obj
 0001:000036b8       __vcrt_FlsSetValue         00000001800046b8 f   libvcruntime:winapi_downlevel.obj
 0001:0000370c       __vcrt_InitializeCriticalSectionEx 000000018000470c f   libvcruntime:winapi_downlevel.obj
 0001:00003770       __vcrt_initialize_winapi_thunks 0000000180004770 f   libvcruntime:winapi_downlevel.obj
 0001:000037a0       __vcrt_uninitialize_winapi_thunks 00000001800047a0 f   libvcruntime:winapi_downlevel.obj
 0001:000037e0       __vcrt_initialize_pure_virtual_call_handler 00000001800047e0 f   libvcruntime:purevirt_data.obj
 0001:00003800       memmove                    0000000180004800 f   libvcruntime:memcpy.obj
 0001:00003800       memcpy                     0000000180004800 f   libvcruntime:memcpy.obj
 0001:00003c60       _CallSettingFrame          0000000180004c60 f   libvcruntime:handlers.obj
 0001:00003ca0       __DestructExceptionObject  0000000180004ca0 f   libvcruntime:ehhelpers.obj
 0001:00003d14       ?_CallMemberFunction0@@YAXQEAX0@Z 0000000180004d14 f i libvcruntime:ehhelpers.obj
 0001:00003d18       ??$ensure_buffer_is_big_enough@D@formatting_buffer@__crt_stdio_output@@QEAA_N_K@Z 0000000180004d18 f i libucrt:output.obj
 0001:00003dc4       ??$is_wide_character_specifier@D@__crt_stdio_output@@YA_N_KDW4length_modifier@0@@Z 0000000180004dc4 f i libucrt:output.obj
 0001:00003df4       ??$type_case_integer_parse_into_buffer@I@?$output_processor@DV?$string_output_adapter@D@__crt_stdio_output@@V?$standard_base@DV?$string_output_adapter@D@__crt_stdio_output@@@2@@__crt_stdio_output@@AEAAXII_N@Z 0000000180004df4 f i libucrt:output.obj
 0001:00003e90       ??$type_case_integer_parse_into_buffer@_K@?$output_processor@DV?$string_output_adapter@D@__crt_stdio_output@@V?$standard_base@DV?$string_output_adapter@D@__crt_stdio_output@@@2@@__crt_stdio_output@@AEAAX_KI_N@Z 0000000180004e90 f i libucrt:output.obj
 0001:00003f2c       ??$write_multiple_characters@V?$string_output_adapter@D@__crt_stdio_output@@D@__crt_stdio_output@@YAXAEBV?$string_output_adapter@D@0@DHQEAH@Z 0000000180004f2c f i libucrt:output.obj
 0001:00003f88       ??0?$output_processor@DV?$string_output_adapter@D@__crt_stdio_output@@V?$standard_base@DV?$string_output_adapter@D@__crt_stdio_output@@@2@@__crt_stdio_output@@QEAA@AEBV?$string_output_adapter@D@1@_KQEBDQEAU__crt_locale_pointers@@QEAD@Z 0000000180004f88 f i libucrt:output.obj
 0001:00004004       ??0_LocaleUpdate@@QEAA@QEAU__crt_locale_pointers@@@Z 0000000180005004 f i libucrt:output.obj
 0001:00004094       ?force_decimal_point@__crt_stdio_output@@YAXPEADQEAU__crt_locale_pointers@@@Z 0000000180005094 f i libucrt:output.obj
 0001:00004104       ?parse_int_from_format_string@?$output_processor@DV?$string_output_adapter@D@__crt_stdio_output@@V?$standard_base@DV?$string_output_adapter@D@__crt_stdio_output@@@2@@__crt_stdio_output@@AEAA_NQEAH@Z 0000000180005104 f i libucrt:output.obj
 0001:00004188       ?process@?$output_processor@DV?$string_output_adapter@D@__crt_stdio_output@@V?$standard_base@DV?$string_output_adapter@D@__crt_stdio_output@@@2@@__crt_stdio_output@@QEAAHXZ 0000000180005188 f i libucrt:output.obj
 0001:0000438c       ?state_case_normal@?$output_processor@DV?$string_output_adapter@D@__crt_stdio_output@@V?$standard_base@DV?$string_output_adapter@D@__crt_stdio_output@@@2@@__crt_stdio_output@@AEAA_NXZ 000000018000538c f i libucrt:output.obj
 0001:00004400       ?state_case_normal_tchar@?$output_processor@DV?$string_output_adapter@D@__crt_stdio_output@@V?$standard_base@DV?$string_output_adapter@D@__crt_stdio_output@@@2@@__crt_stdio_output@@AEAA_ND@Z 0000000180005400 f i libucrt:output.obj
 0001:00004498       ?state_case_size@?$output_processor@DV?$string_output_adapter@D@__crt_stdio_output@@V?$standard_base@DV?$string_output_adapter@D@__crt_stdio_output@@@2@@__crt_stdio_output@@AEAA_NXZ 0000000180005498 f i libucrt:output.obj
 0001:00004614       ?state_case_type@?$output_processor@DV?$string_output_adapter@D@__crt_stdio_output@@V?$standard_base@DV?$string_output_adapter@D@__crt_stdio_output@@@2@@__crt_stdio_output@@AEAA_NXZ 0000000180005614 f i libucrt:output.obj
 0001:00004890       ?type_case_Z@?$output_processor@DV?$string_output_adapter@D@__crt_stdio_output@@V?$standard_base@DV?$string_output_adapter@D@__crt_stdio_output@@@2@@__crt_stdio_output@@AEAA_NXZ 0000000180005890 f i libucrt:output.obj
 0001:00004910       ?type_case_a@?$output_processor@DV?$string_output_adapter@D@__crt_stdio_output@@V?$standard_base@DV?$string_output_adapter@D@__crt_stdio_output@@@2@@__crt_stdio_output@@AEAA_NXZ 0000000180005910 f i libucrt:output.obj
 0001:00004b2c       ?type_case_c_tchar@?$output_processor@DV?$string_output_adapter@D@__crt_stdio_output@@V?$standard_base@DV?$string_output_adapter@D@__crt_stdio_output@@@2@@__crt_stdio_output@@AEAA_ND@Z 0000000180005b2c f i libucrt:output.obj
 0001:00004be0       ?type_case_integer@?$output_processor@DV?$string_output_adapter@D@__crt_stdio_output@@V?$standard_base@DV?$string_output_adapter@D@__crt_stdio_output@@@2@@__crt_stdio_output@@AEAA_NI_N@Z 0000000180005be0 f i libucrt:output.obj
 0001:00004d80       ?type_case_n@?$output_processor@DV?$string_output_adapter@D@__crt_stdio_output@@V?$standard_base@DV?$string_output_adapter@D@__crt_stdio_output@@@2@@__crt_stdio_output@@AEAA_NXZ 0000000180005d80 f i libucrt:output.obj
 0001:00004e5c       ?type_case_s@?$output_processor@DV?$string_output_adapter@D@__crt_stdio_output@@V?$standard_base@DV?$string_output_adapter@D@__crt_stdio_output@@@2@@__crt_stdio_output@@AEAA_NXZ 0000000180005e5c f i libucrt:output.obj
 0001:00004eec       ?write_stored_string_tchar@?$output_processor@DV?$string_output_adapter@D@__crt_stdio_output@@V?$standard_base@DV?$string_output_adapter@D@__crt_stdio_output@@@2@@__crt_stdio_output@@AEAA_ND@Z 0000000180005eec f i libucrt:output.obj
 0001:00004fc4       ?write_string@?$string_output_adapter@D@__crt_stdio_output@@QEBAXQEBDHQEAH1@Z 0000000180005fc4 f i libucrt:output.obj
 0001:00005080       __stdio_common_vsprintf    0000000180006080 f   libucrt:output.obj
 0001:000052b4       wcsncmp                    00000001800062b4 f   libucrt:wcsncmp.obj
 0001:000052e0       _initterm                  00000001800062e0 f   libucrt:initterm.obj
 0001:00005358       _initterm_e                0000000180006358 f   libucrt:initterm.obj
 0001:000053a4       _seh_filter_dll            00000001800063a4 f   libucrt:exception_filter.obj
 0001:000053b8       _seh_filter_exe            00000001800063b8 f   libucrt:exception_filter.obj
 0001:00005778       __acrt_initialize_thread_local_exit_callback 0000000180006778 f   libucrt:exit.obj
 0001:00005780       _cexit                     0000000180006780 f   libucrt:exit.obj
 0001:00005790       _exit                      0000000180006790 f   libucrt:exit.obj
 0001:0000579c       _is_c_termination_complete 000000018000679c f   libucrt:exit.obj
 0001:00005960       __acrt_allocate_buffer_for_argv 0000000180006960 f   libucrt:argv_parsing.obj
 0001:000059c4       _configure_narrow_argv     00000001800069c4 f   libucrt:argv_parsing.obj
 0001:00005d20       __dcrt_uninitialize_environments_nolock 0000000180006d20 f   libucrt:environment_initialization.obj
 0001:00005d58       _initialize_narrow_environment 0000000180006d58 f   libucrt:environment_initialization.obj
 0001:00005d60       ??$?RV<lambda_e24bbb7b643b32fcea6fa61b31d4c984>@@AEAV<lambda_275893d493268fdec8709772e3fcec0e>@@V<lambda_9d71df4d7cf3f480f8d633942495c3b0>@@@?$__crt_seh_guarded_call@H@@QEAAH$$QEAV<lambda_e24bbb7b643b32fcea6fa61b31d4c984>@@AEAV<lambda_275893d493268fdec8709772e3fcec0e>@@$$QEAV<lambda_9d71df4d7cf3f480f8d633942495c3b0>@@@Z 0000000180006d60 f i libucrt:onexit.obj
 0001:00005f00       _execute_onexit_table      0000000180006f00 f   libucrt:onexit.obj
 0001:00005f3c       _initialize_onexit_table   0000000180006f3c f   libucrt:onexit.obj
 0001:00005fb4       __acrt_uninitialize_command_line 0000000180006fb4 f   libucrt:argv_data.obj
 0001:000060b4       __acrt_initialize          00000001800070b4 f   libucrt:initialization.obj
 0001:000060c8       __acrt_thread_attach       00000001800070c8 f   libucrt:initialization.obj
 0001:000060dc       __acrt_thread_detach       00000001800070dc f   libucrt:initialization.obj
 0001:000060ec       __acrt_uninitialize        00000001800070ec f   libucrt:initialization.obj
 0001:00006100       __acrt_uninitialize_critical 0000000180007100 f   libucrt:initialization.obj
 0001:00006110       terminate                  0000000180007110 f   libucrt:terminate.obj
 0001:00006138       free                       0000000180007138 f   libucrt:free.obj
 0001:00006140       strcpy_s                   0000000180007140 f   libucrt:strcpy_s.obj
 0001:000061a0       ??$is_overflow_condition@K@__crt_strtox@@YA_NIK@Z 00000001800071a0 f i libucrt:atox.obj
 0001:000061cc       ??$parse_integer@KV?$c_string_character_source@D@__crt_strtox@@@__crt_strtox@@YAKQEAU__crt_locale_pointers@@V?$c_string_character_source@D@0@H_N@Z 00000001800071cc f i libucrt:atox.obj
 0001:000064f0       strncmp                    00000001800074f0 f   libucrt:strncmp.obj
 0001:00006570       abort                      0000000180007570 f   libucrt:abort.obj
 0001:000065c8       calloc                     00000001800075c8 f   libucrt:calloc.obj
 0001:000065d0       __acrt_call_reportfault    00000001800075d0 f   libucrt:invalid_parameter.obj
 0001:0000672c       __acrt_initialize_invalid_parameter_handler 000000018000772c f   libucrt:invalid_parameter.obj
 0001:00006734       _invalid_parameter         0000000180007734 f   libucrt:invalid_parameter.obj
 0001:000067dc       _invalid_parameter_noinfo  00000001800077dc f   libucrt:invalid_parameter.obj
 0001:000067fc       _invoke_watson             00000001800077fc f   libucrt:invalid_parameter.obj
 0001:00006844       isdigit                    0000000180007844 f i libucrt:_ctype.obj
 0001:00006908       _tolower_l                 0000000180007908 f   libucrt:tolower_toupper.obj
 0001:00006a48       tolower                    0000000180007a48 f   libucrt:tolower_toupper.obj
 0001:00006a74       __acrt_errno_from_os_error 0000000180007a74 f   libucrt:errno.obj
 0001:00006abc       __acrt_errno_map_os_error  0000000180007abc f   libucrt:errno.obj
 0001:00006b0c       __doserrno                 0000000180007b0c f   libucrt:errno.obj
 0001:00006b2c       _errno                     0000000180007b2c f   libucrt:errno.obj
 0001:00006b4c       _free_base                 0000000180007b4c f   libucrt:free_base.obj
 0001:00006b8c       _malloc_base               0000000180007b8c f   libucrt:malloc_base.obj
 0001:00006bec       ??$make_c_string_character_source@DPEAPEAD@__crt_strtox@@YA?AV?$c_string_character_source@D@0@QEBDQEAPEAD@Z 0000000180007bec f i libucrt:strtox.obj
 0001:00006c00       strtol                     0000000180007c00 f   libucrt:strtox.obj
 0001:00006c30       _mbtowc_l                  0000000180007c30 f   libucrt:mbtowc.obj
 0001:00006d78       mbtowc                     0000000180007d78 f   libucrt:mbtowc.obj
 0001:00006d80       _wctomb_s_l                0000000180007d80 f   libucrt:wctomb.obj
 0001:00006f04       wctomb_s                   0000000180007f04 f   libucrt:wctomb.obj
 0001:00006f18       strnlen                    0000000180007f18 f   libucrt:strnlen.obj
 0001:00007074       wcsnlen                    0000000180008074 f   libucrt:strnlen.obj
 0001:00007264       ??$?RV<lambda_46352004c1216016012b18bd6f87e700>@@AEAV<lambda_3bd07e1a1191394380780325891bf33f>@@V<lambda_334532d3f185bcaa59b5be82d7d22bff>@@@?$__crt_seh_guarded_call@X@@QEAAX$$QEAV<lambda_46352004c1216016012b18bd6f87e700>@@AEAV<lambda_3bd07e1a1191394380780325891bf33f>@@$$QEAV<lambda_334532d3f185bcaa59b5be82d7d22bff>@@@Z 0000000180008264 f i libucrt:per_thread_data.obj
 0001:000072c4       ??$?RV<lambda_5e887d1dcbef67a5eb4283622ba103bf>@@AEAV<lambda_4466841279450cc726390878d4a41900>@@V<lambda_341c25c0346d94847f1f3c463c57e077>@@@?$__crt_seh_guarded_call@X@@QEAAX$$QEAV<lambda_5e887d1dcbef67a5eb4283622ba103bf>@@AEAV<lambda_4466841279450cc726390878d4a41900>@@$$QEAV<lambda_341c25c0346d94847f1f3c463c57e077>@@@Z 00000001800082c4 f i libucrt:per_thread_data.obj
 0001:0000730c       ??$?RV<lambda_72d1df2b273a38828b1ce30cbf4cdab5>@@AEAV<lambda_876a65b173b8412d3a47c70a915b0cf4>@@V<lambda_41932305e351933ebe8f8be3ed8bb5dc>@@@?$__crt_seh_guarded_call@X@@QEAAX$$QEAV<lambda_72d1df2b273a38828b1ce30cbf4cdab5>@@AEAV<lambda_876a65b173b8412d3a47c70a915b0cf4>@@$$QEAV<lambda_41932305e351933ebe8f8be3ed8bb5dc>@@@Z 000000018000830c f i libucrt:per_thread_data.obj
 0001:0000734c       ??$?RV<lambda_fb3a7dec4e47f37f22dae91bb15c9095>@@AEAV<lambda_698284760c8add0bfb0756c19673e34b>@@V<lambda_dfb8eca1e75fef3034a8fb18dd509707>@@@?$__crt_seh_guarded_call@X@@QEAAX$$QEAV<lambda_fb3a7dec4e47f37f22dae91bb15c9095>@@AEAV<lambda_698284760c8add0bfb0756c19673e34b>@@$$QEAV<lambda_dfb8eca1e75fef3034a8fb18dd509707>@@@Z 000000018000834c f i libucrt:per_thread_data.obj
 0001:000075dc       __acrt_freeptd             00000001800085dc f   libucrt:per_thread_data.obj
 0001:00007620       __acrt_getptd              0000000180008620 f   libucrt:per_thread_data.obj
 0001:000076b4       __acrt_getptd_noexit       00000001800086b4 f   libucrt:per_thread_data.obj
 0001:00007754       __acrt_initialize_ptd      0000000180008754 f   libucrt:per_thread_data.obj
 0001:00007790       __acrt_uninitialize_ptd    0000000180008790 f   libucrt:per_thread_data.obj
 0001:000077b4       __acrt_update_locale_info  00000001800087b4 f   libucrt:locale_update.obj
 0001:000077e8       __acrt_update_multibyte_info 00000001800087e8 f   libucrt:locale_update.obj
 0001:0000781c       ?__acrt_fp_classify@@YA?AW4__acrt_fp_class@@AEBN@Z 000000018000881c f i libucrt:cvt.obj
 0001:00008254       __acrt_fp_format           0000000180009254 f   libucrt:cvt.obj
 0001:00008498       _fileno                    0000000180009498 f   libucrt:fileno.obj
 0001:000084c0       __acrt_initialize_stdio    00000001800094c0 f   libucrt:_file.obj
 0001:000085e0       __acrt_uninitialize_stdio  00000001800095e0 f   libucrt:_file.obj
 0001:0000863c       _lock_file                 000000018000963c f   libucrt:_file.obj
 0001:00008648       _unlock_file               0000000180009648 f   libucrt:_file.obj
 0001:00008654       _get_printf_count_output   0000000180009654 f   libucrt:printf_count_output.obj
 0001:0000866c       __acrt_set_locale_changed  000000018000966c f   libucrt:wsetlocale.obj
 0001:00008678       __acrt_uninitialize_locale 0000000180009678 f   libucrt:wsetlocale.obj
 0001:000088a8       __acrt_initialize_lowio    00000001800098a8 f   libucrt:ioinit.obj
 0001:000088e4       __acrt_uninitialize_lowio  00000001800098e4 f   libucrt:ioinit.obj
 0001:00008924       __acrt_initialize_locks    0000000180009924 f   libucrt:locks.obj
 0001:0000896c       __acrt_lock                000000018000996c f   libucrt:locks.obj
 0001:00008988       __acrt_uninitialize_locks  0000000180009988 f   libucrt:locks.obj
 0001:000089c0       __acrt_unlock              00000001800099c0 f   libucrt:locks.obj
 0001:00008b7c       __acrt_FlsAlloc            0000000180009b7c f   libucrt:winapi_thunks.obj
 0001:00008bd4       __acrt_FlsFree             0000000180009bd4 f   libucrt:winapi_thunks.obj
 0001:00008c2c       __acrt_FlsGetValue         0000000180009c2c f   libucrt:winapi_thunks.obj
 0001:00008c84       __acrt_FlsSetValue         0000000180009c84 f   libucrt:winapi_thunks.obj
 0001:00008cec       __acrt_InitializeCriticalSectionEx 0000000180009cec f   libucrt:winapi_thunks.obj
 0001:00008d64       __acrt_LCMapStringEx       0000000180009d64 f   libucrt:winapi_thunks.obj
 0001:00008e54       __acrt_LocaleNameToLCID    0000000180009e54 f   libucrt:winapi_thunks.obj
 0001:00008ebc       __acrt_initialize_winapi_thunks 0000000180009ebc f   libucrt:winapi_thunks.obj
 0001:00008ef4       __acrt_is_packaged_app     0000000180009ef4 f   libucrt:winapi_thunks.obj
 0001:00008f7c       __acrt_uninitialize_winapi_thunks 0000000180009f7c f   libucrt:winapi_thunks.obj
 0001:00008fc0       _calloc_base               0000000180009fc0 f   libucrt:calloc_base.obj
 0001:00009514       ?expand_if_necessary@?$argument_list@D@?A0xca0879c4@@AEAAHXZ 000000018000a514 f i libucrt:argv_wildcards.obj
 0001:000095dc       __acrt_expand_narrow_argv_wildcards 000000018000a5dc f   libucrt:argv_wildcards.obj
 0001:000095e4       ??$?RV<lambda_99476a1ad63dd22509b5d3e65b0ffc95>@@AEAV<lambda_ad1ced32f4ac17aa236e5ef05d6b3b7c>@@V<lambda_f7424dd8d45958661754dc4f2697e9c3>@@@?$__crt_seh_guarded_call@X@@QEAAX$$QEAV<lambda_99476a1ad63dd22509b5d3e65b0ffc95>@@AEAV<lambda_ad1ced32f4ac17aa236e5ef05d6b3b7c>@@$$QEAV<lambda_f7424dd8d45958661754dc4f2697e9c3>@@@Z 000000018000a5e4 f i libucrt:mbctype.obj
 0001:00009ce0       __acrt_initialize_multibyte 000000018000ace0 f   libucrt:mbctype.obj
 0001:00009d08       __acrt_update_thread_multibyte_data 000000018000ad08 f   libucrt:mbctype.obj
 0001:00009dc8       _setmbcp_nolock            000000018000adc8 f   libucrt:mbctype.obj
 0001:0000a0e8       _ismbblead                 000000018000b0e8 f   libucrt:ismbbyte.obj
 0001:0000a0fc       __acrt_initialize_command_line 000000018000b0fc f   libucrt:argv_data.obj
 0001:0000a124       __dcrt_get_narrow_environment_from_os 000000018000b124 f   libucrt:get_environment_from_os.obj
 0001:0000a228       _recalloc                  000000018000b228 f   libucrt:recalloc.obj
 0001:0000a230       _recalloc_base             000000018000b230 f   libucrt:recalloc.obj
 0001:0000a2c8       __acrt_initialize_heap     000000018000b2c8 f   libucrt:heap_handle.obj
 0001:0000a2e4       __acrt_uninitialize_heap   000000018000b2e4 f   libucrt:heap_handle.obj
 0001:0000a2f0       __acrt_execute_initializers 000000018000b2f0 f   libucrt:shared_initialization.obj
 0001:0000a384       __acrt_execute_uninitializers 000000018000b384 f   libucrt:shared_initialization.obj
 0001:0000a3d4       __acrt_initialize_new_handler 000000018000b3d4 f   libucrt:new_handler.obj
 0001:0000a3dc       _callnewh                  000000018000b3dc f   libucrt:new_handler.obj
 0001:0000a41c       _query_new_handler         000000018000b41c f   libucrt:new_handler.obj
 0001:0000a450       ??$?RV<lambda_c36588078e9f5dfd39652860aa6b3aaf>@@AEAV<lambda_ec61778202f4f5fc7e7711acc23c3bca>@@V<lambda_dc9d2797ccde5d239b4a0efae8ebd7db>@@@?$__crt_seh_guarded_call@P6AXH@Z@@QEAAP6AXH@Z$$QEAV<lambda_c36588078e9f5dfd39652860aa6b3aaf>@@AEAV<lambda_ec61778202f4f5fc7e7711acc23c3bca>@@$$QEAV<lambda_dc9d2797ccde5d239b4a0efae8ebd7db>@@@Z 000000018000b450 f i libucrt:signal.obj
 0001:0000a498       __acrt_get_sigabrt_handler 000000018000b498 f   libucrt:signal.obj
 0001:0000a4c8       __acrt_initialize_signal_handlers 000000018000b4c8 f   libucrt:signal.obj
 0001:0000a4e8       raise                      000000018000b4e8 f   libucrt:signal.obj
 0001:0000a784       __acrt_has_user_matherr    000000018000b784 f   libucrt:matherr.obj
 0001:0000a7a4       __acrt_initialize_user_matherr 000000018000b7a4 f   libucrt:matherr.obj
 0001:0000a7ac       __acrt_invoke_user_matherr 000000018000b7ac f   libucrt:matherr.obj
 0001:0000a7f4       __pctype_func              000000018000b7f4 f   libucrt:ctype.obj
 0001:0000a824       _isctype_l                 000000018000b824 f   libucrt:isctype.obj
 0001:0000a934       _isleadbyte_l              000000018000b934 f i libucrt:_wctype.obj
 0001:0000acd0       __acrt_LCMapStringA        000000018000bcd0 f   libucrt:lcmapstringa.obj
 0001:0000ad68       _query_new_mode            000000018000bd68 f   libucrt:new_mode.obj
 0001:0000ad70       __acrt_add_locale_ref      000000018000bd70 f   libucrt:locale_refcounting.obj
 0001:0000adfc       __acrt_free_locale         000000018000bdfc f   libucrt:locale_refcounting.obj
 0001:0000af74       __acrt_locale_add_lc_time_reference 000000018000bf74 f   libucrt:locale_refcounting.obj
 0001:0000af9c       __acrt_locale_free_lc_time_if_unreferenced 000000018000bf9c f   libucrt:locale_refcounting.obj
 0001:0000afd4       __acrt_locale_release_lc_time_reference 000000018000bfd4 f   libucrt:locale_refcounting.obj
 0001:0000affc       __acrt_release_locale_ref  000000018000bffc f   libucrt:locale_refcounting.obj
 0001:0000b0a4       __acrt_update_thread_locale_data 000000018000c0a4 f   libucrt:locale_refcounting.obj
 0001:0000b114       _updatetlocinfoEx_nolock   000000018000c114 f   libucrt:locale_refcounting.obj
 0001:0000b17c       __acrt_fp_strflt_to_string 000000018000c17c f   libucrt:_fptostr.obj
 0001:0000b240       ?divide@__crt_strtox@@YA_KAEAUbig_integer@1@AEBU21@@Z 000000018000c240 f i libucrt:cfout.obj
 0001:0000b710       __acrt_fltout              000000018000c710 f   libucrt:cfout.obj
 0001:0000cb04       _fcloseall                 000000018000db04 f   libucrt:closeall.obj
 0001:0000cbb8       __acrt_stdio_flush_nolock  000000018000dbb8 f   libucrt:fflush.obj
 0001:0000cc30       _fflush_nolock             000000018000dc30 f   libucrt:fflush.obj
 0001:0000cc7c       _flushall                  000000018000dc7c f   libucrt:fflush.obj
 0001:0000cd6c       __acrt_stdio_free_buffer_nolock 000000018000dd6c f   libucrt:_freebuf.obj
 0001:0000cdac       _isatty                    000000018000ddac f   libucrt:isatty.obj
 0001:0000ce0c       __acrt_locale_free_monetary 000000018000de0c f   libucrt:initmon.obj
 0001:0000cf18       __acrt_locale_free_numeric 000000018000df18 f   libucrt:initnum.obj
 0001:0000cfdc       __acrt_locale_free_time    000000018000dfdc f   libucrt:inittime.obj
 0001:0000d0e4       __acrt_GetStringTypeA      000000018000e0e4 f   libucrt:getstringtypea.obj
 0001:0000d298       __acrt_lowio_create_handle_array 000000018000e298 f   libucrt:osfinfo.obj
 0001:0000d330       __acrt_lowio_destroy_handle_array 000000018000e330 f   libucrt:osfinfo.obj
 0001:0000d380       __acrt_lowio_ensure_fh_exists 000000018000e380 f   libucrt:osfinfo.obj
 0001:0000d438       __acrt_lowio_lock_fh       000000018000e438 f   libucrt:osfinfo.obj
 0001:0000d45c       __acrt_lowio_unlock_fh     000000018000e45c f   libucrt:osfinfo.obj
 0001:0000d480       _free_osfhnd               000000018000e480 f   libucrt:osfinfo.obj
 0001:0000d53c       _get_osfhandle             000000018000e53c f   libucrt:osfinfo.obj
 0001:0000d67c       __acrt_DownlevelLocaleNameToLCID 000000018000e67c f   libucrt:lcidtoname_downlevel.obj
 0001:0000d780       qsort                      000000018000e780 f   libucrt:qsort.obj
 0001:0000dab4       strncpy_s                  000000018000eab4 f   libucrt:strncpy_s.obj
 0001:0000db88       strpbrk                    000000018000eb88 f   libucrt:strpbrk.obj
 0001:0000dc28       _mbsdec                    000000018000ec28 f   libucrt:mbsdec.obj
 0001:0000dc30       _mbsdec_l                  000000018000ec30 f   libucrt:mbsdec.obj
 0001:0000dce0       _msize                     000000018000ece0 f   libucrt:msize.obj
 0001:0000dd1c       _realloc_base              000000018000ed1c f   libucrt:realloc_base.obj
 0001:0000dda0       __strncnt                  000000018000eda0 f   libucrt:strncnt.obj
 0001:0000ddb8       fegetenv                   000000018000edb8 f   libucrt:fegetenv.obj
 0001:0000ddd8       fesetenv                   000000018000edd8 f   libucrt:fesetenv.obj
 0001:0000de24       feholdexcept               000000018000ee24 f   libucrt:feholdexcept.obj
 0001:0000de74       ceil                       000000018000ee74 f   libucrt:ceil.obj
 0001:0000df40       log10                      000000018000ef40 f   libucrt:log10.obj
 0001:0000ea8c       _write                     000000018000fa8c f   libucrt:write.obj
 0001:0000eb78       _write_nolock              000000018000fb78 f   libucrt:write.obj
 0001:0000eef8       _lseeki64_nolock           000000018000fef8 f   libucrt:lseek.obj
 0001:0000ef00       _fclose_nolock             000000018000ff00 f   libucrt:fclose.obj
 0001:0000ef84       fclose                     000000018000ff84 f   libucrt:fclose.obj
 0001:0000eff0       ??$?RV<lambda_b521505b218e5242e90febf6bfebc422>@@AEAV<lambda_6978c1fb23f02e42e1d9e99668cc68aa>@@V<lambda_314360699dd331753a4119843814e9a7>@@@?$__crt_seh_guarded_call@H@@QEAAH$$QEAV<lambda_b521505b218e5242e90febf6bfebc422>@@AEAV<lambda_6978c1fb23f02e42e1d9e99668cc68aa>@@$$QEAV<lambda_314360699dd331753a4119843814e9a7>@@@Z 000000018000fff0 f i libucrt:commit.obj
 0001:0000f07c       _commit                    000000018001007c f   libucrt:commit.obj
 0001:0000f110       _query_app_type            0000000180010110 f   libucrt:report_runtime_error.obj
 0001:0000f118       _getfpcontrolword          0000000180010118 f   libucrt:_fenvutils.obj
 0001:0000f130       _getfpstatusword           0000000180010130 f   libucrt:_fenvutils.obj
 0001:0000f144       _setfpcontrolword          0000000180010144 f   libucrt:_fenvutils.obj
 0001:0000f150       _setfpstatusword           0000000180010150 f   libucrt:_fenvutils.obj
 0001:0000f1a0       _clearfp                   00000001800101a0 f   libucrt:ieee.obj
 0001:0000f1f4       _controlfp                 00000001800101f4 f   libucrt:ieee.obj
 0001:0000f200       _statusfp                  0000000180010200 f   libucrt:ieee.obj
 0001:0000f604       _handle_error              0000000180010604 f   libucrt:libm_error.obj
 0001:0000f72c       _handle_nan                000000018001072c f   libucrt:libm_error.obj
 0001:0000f750       __acrt_initialize_fma3     0000000180010750 f   libucrt:fma3_available.obj
 0001:0000f7c0       _log10_special             00000001800107c0 f   libucrt:log_special.obj
 0001:0000f878       _putwch_nolock             0000000180010878 f   libucrt:putwch.obj
 0001:0000f8d4       ??$?RV<lambda_bfedae4ebbf01fab1bb6dcc6a9e276e0>@@AEAV<lambda_2fe9b910cf3cbf4a0ab98a02ba45b3ec>@@V<lambda_237c231691f317818eb88cc1d5d642d6>@@@?$__crt_seh_guarded_call@H@@QEAAH$$QEAV<lambda_bfedae4ebbf01fab1bb6dcc6a9e276e0>@@AEAV<lambda_2fe9b910cf3cbf4a0ab98a02ba45b3ec>@@$$QEAV<lambda_237c231691f317818eb88cc1d5d642d6>@@@Z 00000001800108d4 f i libucrt:close.obj
 0001:0000f948       _close                     0000000180010948 f   libucrt:close.obj
 0001:0000f9ec       _close_nolock              00000001800109ec f   libucrt:close.obj
 0001:0000faa8       ?__acrt_stdio_free_stream@@YAXV__crt_stdio_stream@@@Z 0000000180010aa8 f   libucrt:stream.obj
 0001:0000fb00       _get_fpsr                  0000000180010b00 f   libucrt:fpsr.obj
 0001:0000fb10       _set_fpsr                  0000000180010b10 f   libucrt:fpsr.obj
 0001:0000fb1a       _fclrf                     0000000180010b1a f   libucrt:fpsr.obj
 0001:0000fb2e       _frnd                      0000000180010b2e f   libucrt:fpsr.obj
 0001:0000fb50       _raise_exc                 0000000180010b50 f   libucrt:fpexcept.obj
 0001:0000fb78       _raise_exc_ex              0000000180010b78 f   libucrt:fpexcept.obj
 0001:0000fe80       _set_errno_from_matherr    0000000180010e80 f   libucrt:fpexcept.obj
 0001:0000feb0       _clrfp                     0000000180010eb0 f   libucrt:fpctrl.obj
 0001:0000fed0       _ctrlfp                    0000000180010ed0 f   libucrt:fpctrl.obj
 0001:0000ff4c       _set_statfp                0000000180010f4c f   libucrt:fpctrl.obj
 0001:0000ff6c       _statfp                    0000000180010f6c f   libucrt:fpctrl.obj
 0001:0000ff80       __dcrt_lowio_initialize_console_output 0000000180010f80 f   libucrt:initcon.obj
 0001:0000ffbc       __dcrt_terminate_console_output 0000000180010fbc f   libucrt:initcon.obj
 0001:0000ffdc       IsProcessorFeaturePresent  0000000180010fdc f   kernel32:KERNEL32.dll
 0001:0000ffe2       RtlUnwindEx                0000000180010fe2 f   kernel32:KERNEL32.dll
 0001:0000fff0       _FindPESection             0000000180010ff0 f   LIBCMT:pesect.obj
 0001:00010040       _IsNonwritableInCurrentImage 0000000180011040 f   LIBCMT:pesect.obj
 0001:00010090       _ValidateImageBase         0000000180011090 f   LIBCMT:pesect.obj
 0001:000100d0       _alloca_probe              00000001800110d0 f   LIBCMT:_chkstk_.obj
 0001:000100d0       __chkstk                   00000001800110d0 f   LIBCMT:_chkstk_.obj
 0001:00010140       memcmp                     0000000180011140 f   libvcruntime:memcmp.obj
 0001:00010220       _guard_dispatch_icall_nop  0000000180011220 f   LIBCMT:_guard_dispatch_.obj
 0002:00000000       __imp_SelectObject         0000000180012000     gdi32:GDI32.dll
 0002:00000008       __imp_DeleteObject         0000000180012008     gdi32:GDI32.dll
 0002:00000010       __imp_DeleteDC             0000000180012010     gdi32:GDI32.dll
 0002:00000018       __imp_CreateSolidBrush     0000000180012018     gdi32:GDI32.dll
 0002:00000020       __imp_CreateCompatibleDC   0000000180012020     gdi32:GDI32.dll
 0002:00000028       __imp_CreateDIBSection     0000000180012028     gdi32:GDI32.dll
 0002:00000030       \177GDI32_NULL_THUNK_DATA  0000000180012030     gdi32:GDI32.dll
 0002:00000038       __imp_WriteFile            0000000180012038     kernel32:KERNEL32.dll
 0002:00000040       __imp_CloseHandle          0000000180012040     kernel32:KERNEL32.dll
 0002:00000048       __imp_lstrcpynW            0000000180012048     kernel32:KERNEL32.dll
 0002:00000050       __imp_lstrcpyW             0000000180012050     kernel32:KERNEL32.dll
 0002:00000058       __imp_lstrcatW             0000000180012058     kernel32:KERNEL32.dll
 0002:00000060       __imp_lstrlenW             0000000180012060     kernel32:KERNEL32.dll
 0002:00000068       __imp_LoadLibraryW         0000000180012068     kernel32:KERNEL32.dll
 0002:00000070       __imp_WaitForSingleObject  0000000180012070     kernel32:KERNEL32.dll
 0002:00000078       __imp_GetTempFileNameW     0000000180012078     kernel32:KERNEL32.dll
 0002:00000080       __imp_CreateFileW          0000000180012080     kernel32:KERNEL32.dll
 0002:00000088       __imp_DeleteFileW          0000000180012088     kernel32:KERNEL32.dll
 0002:00000090       __imp_WriteConsoleW        0000000180012090     kernel32:KERNEL32.dll
 0002:00000098       __imp_FlushFileBuffers     0000000180012098     kernel32:KERNEL32.dll
 0002:000000a0       __imp_SetFilePointerEx     00000001800120a0     kernel32:KERNEL32.dll
 0002:000000a8       __imp_GetLastError         00000001800120a8     kernel32:KERNEL32.dll
 0002:000000b0       __imp_GetProcessHeap       00000001800120b0     kernel32:KERNEL32.dll
 0002:000000b8       __imp_HeapFree             00000001800120b8     kernel32:KERNEL32.dll
 0002:000000c0       __imp_HeapAlloc            00000001800120c0     kernel32:KERNEL32.dll
 0002:000000c8       __imp_GetProcAddress       00000001800120c8     kernel32:KERNEL32.dll
 0002:000000d0       __imp_GetTempPathW         00000001800120d0     kernel32:KERNEL32.dll
 0002:000000d8       __imp_FreeLibrary          00000001800120d8     kernel32:KERNEL32.dll
 0002:000000e0       __imp_GetConsoleMode       00000001800120e0     kernel32:KERNEL32.dll
 0002:000000e8       __imp_GetConsoleCP         00000001800120e8     kernel32:KERNEL32.dll
 0002:000000f0       __imp_HeapSize             00000001800120f0     kernel32:KERNEL32.dll
 0002:000000f8       __imp_HeapCreate           00000001800120f8     kernel32:KERNEL32.dll
 0002:00000100       __imp_HeapDestroy          0000000180012100     kernel32:KERNEL32.dll
 0002:00000108       __imp_HeapReAlloc          0000000180012108     kernel32:KERNEL32.dll
 0002:00000110       __imp_RaiseException       0000000180012110     kernel32:KERNEL32.dll
 0002:00000118       __imp_CreateThread         0000000180012118     kernel32:KERNEL32.dll
 0002:00000120       __imp_GetCurrentThreadId   0000000180012120     kernel32:KERNEL32.dll
 0002:00000128       __imp_TerminateThread      0000000180012128     kernel32:KERNEL32.dll
 0002:00000130       __imp_SetLastError         0000000180012130     kernel32:KERNEL32.dll
 0002:00000138       __imp_ResumeThread         0000000180012138     kernel32:KERNEL32.dll
 0002:00000140       __imp_IsDebuggerPresent    0000000180012140     kernel32:KERNEL32.dll
 0002:00000148       __imp_GetTickCount         0000000180012148     kernel32:KERNEL32.dll
 0002:00000150       __imp_lstrcpynA            0000000180012150     kernel32:KERNEL32.dll
 0002:00000158       __imp_DebugBreak           0000000180012158     kernel32:KERNEL32.dll
 0002:00000160       __imp_RtlCaptureContext    0000000180012160     kernel32:KERNEL32.dll
 0002:00000168       __imp_RtlLookupFunctionEntry 0000000180012168     kernel32:KERNEL32.dll
 0002:00000170       __imp_RtlVirtualUnwind     0000000180012170     kernel32:KERNEL32.dll
 0002:00000178       __imp_UnhandledExceptionFilter 0000000180012178     kernel32:KERNEL32.dll
 0002:00000180       __imp_SetUnhandledExceptionFilter 0000000180012180     kernel32:KERNEL32.dll
 0002:00000188       __imp_GetCurrentProcess    0000000180012188     kernel32:KERNEL32.dll
 0002:00000190       __imp_TerminateProcess     0000000180012190     kernel32:KERNEL32.dll
 0002:00000198       __imp_IsProcessorFeaturePresent 0000000180012198     kernel32:KERNEL32.dll
 0002:000001a0       __imp_QueryPerformanceCounter 00000001800121a0     kernel32:KERNEL32.dll
 0002:000001a8       __imp_GetCurrentProcessId  00000001800121a8     kernel32:KERNEL32.dll
 0002:000001b0       __imp_GetSystemTimeAsFileTime 00000001800121b0     kernel32:KERNEL32.dll
 0002:000001b8       __imp_InitializeSListHead  00000001800121b8     kernel32:KERNEL32.dll
 0002:000001c0       __imp_GetStartupInfoW      00000001800121c0     kernel32:KERNEL32.dll
 0002:000001c8       __imp_GetModuleHandleW     00000001800121c8     kernel32:KERNEL32.dll
 0002:000001d0       __imp_RtlUnwindEx          00000001800121d0     kernel32:KERNEL32.dll
 0002:000001d8       __imp_InterlockedFlushSList 00000001800121d8     kernel32:KERNEL32.dll
 0002:000001e0       __imp_EnterCriticalSection 00000001800121e0     kernel32:KERNEL32.dll
 0002:000001e8       __imp_LeaveCriticalSection 00000001800121e8     kernel32:KERNEL32.dll
 0002:000001f0       __imp_DeleteCriticalSection 00000001800121f0     kernel32:KERNEL32.dll
 0002:000001f8       __imp_InitializeCriticalSectionAndSpinCount 00000001800121f8     kernel32:KERNEL32.dll
 0002:00000200       __imp_TlsAlloc             0000000180012200     kernel32:KERNEL32.dll
 0002:00000208       __imp_TlsGetValue          0000000180012208     kernel32:KERNEL32.dll
 0002:00000210       __imp_TlsSetValue          0000000180012210     kernel32:KERNEL32.dll
 0002:00000218       __imp_TlsFree              0000000180012218     kernel32:KERNEL32.dll
 0002:00000220       __imp_LoadLibraryExW       0000000180012220     kernel32:KERNEL32.dll
 0002:00000228       __imp_ExitProcess          0000000180012228     kernel32:KERNEL32.dll
 0002:00000230       __imp_GetModuleHandleExW   0000000180012230     kernel32:KERNEL32.dll
 0002:00000238       __imp_GetModuleFileNameA   0000000180012238     kernel32:KERNEL32.dll
 0002:00000240       __imp_MultiByteToWideChar  0000000180012240     kernel32:KERNEL32.dll
 0002:00000248       __imp_WideCharToMultiByte  0000000180012248     kernel32:KERNEL32.dll
 0002:00000250       __imp_GetACP               0000000180012250     kernel32:KERNEL32.dll
 0002:00000258       __imp_GetStdHandle         0000000180012258     kernel32:KERNEL32.dll
 0002:00000260       __imp_GetFileType          0000000180012260     kernel32:KERNEL32.dll
 0002:00000268       __imp_LCMapStringW         0000000180012268     kernel32:KERNEL32.dll
 0002:00000270       __imp_FindClose            0000000180012270     kernel32:KERNEL32.dll
 0002:00000278       __imp_FindFirstFileExA     0000000180012278     kernel32:KERNEL32.dll
 0002:00000280       __imp_FindNextFileA        0000000180012280     kernel32:KERNEL32.dll
 0002:00000288       __imp_IsValidCodePage      0000000180012288     kernel32:KERNEL32.dll
 0002:00000290       __imp_GetOEMCP             0000000180012290     kernel32:KERNEL32.dll
 0002:00000298       __imp_GetCPInfo            0000000180012298     kernel32:KERNEL32.dll
 0002:000002a0       __imp_GetCommandLineA      00000001800122a0     kernel32:KERNEL32.dll
 0002:000002a8       __imp_GetCommandLineW      00000001800122a8     kernel32:KERNEL32.dll
 0002:000002b0       __imp_GetEnvironmentStringsW 00000001800122b0     kernel32:KERNEL32.dll
 0002:000002b8       __imp_FreeEnvironmentStringsW 00000001800122b8     kernel32:KERNEL32.dll
 0002:000002c0       __imp_GetStringTypeW       00000001800122c0     kernel32:KERNEL32.dll
 0002:000002c8       __imp_SetStdHandle         00000001800122c8     kernel32:KERNEL32.dll
 0002:000002d0       \177KERNEL32_NULL_THUNK_DATA 00000001800122d0     kernel32:KERNEL32.dll
 0002:000002d8       __imp_wsprintfW            00000001800122d8     user32:USER32.dll
 0002:000002e0       __imp_CharLowerBuffW       00000001800122e0     user32:USER32.dll
 0002:000002e8       __imp_FillRect             00000001800122e8     user32:USER32.dll
 0002:000002f0       \177USER32_NULL_THUNK_DATA 00000001800122f0     user32:USER32.dll
 0002:000002f8       __imp_CoUninitialize       00000001800122f8     ole32:ole32.dll
 0002:00000300       __imp_CoInitialize         0000000180012300     ole32:ole32.dll
 0002:00000308       \177ole32_NULL_THUNK_DATA  0000000180012308     ole32:ole32.dll
 0002:00000310       __guard_check_icall_fptr   0000000180012310     LIBCMT:guard_support.obj
 0002:00000318       __guard_dispatch_icall_fptr 0000000180012318     LIBCMT:guard_support.obj
 0002:00000320       __xc_a                     0000000180012320     LIBCMT:initializers.obj
 0002:00000328       __xc_z                     0000000180012328     LIBCMT:initializers.obj
 0002:00000330       __xi_a                     0000000180012330     LIBCMT:initializers.obj
 0002:00000338       __acrt_stdio_initializer   0000000180012338     libucrt:stdio_initializer.obj
 0002:00000340       __acrt_multibyte_initializer 0000000180012340     libucrt:multibyte_initializer.obj
 0002:00000348       __acrt_tran_fma3_initializer 0000000180012348     libucrt:fma3_initializer.obj
 0002:00000350       __xi_z                     0000000180012350     LIBCMT:initializers.obj
 0002:00000358       __xp_a                     0000000180012358     LIBCMT:initializers.obj
 0002:00000360       __acrt_locale_terminator   0000000180012360     libucrt:locale_initializer.obj
 0002:00000368       __dcrt_console_output_terminator 0000000180012368     libucrt:console_output_initializer.obj
 0002:00000370       __acrt_stdio_terminator    0000000180012370     libucrt:stdio_initializer.obj
 0002:00000378       __xp_z                     0000000180012378     LIBCMT:initializers.obj
 0002:00000380       __xt_a                     0000000180012380     LIBCMT:initializers.obj
 0002:00000388       __xt_z                     0000000180012388     LIBCMT:initializers.obj
 0002:00000390       FrameDimensionTime         0000000180012390     gdip.obj
 0002:000003a0       FrameDimensionPage         00000001800123a0     gdip.obj
 0002:000003b0       ??_C@_1BI@LOJECBFD@?$AAG?$AAd?$AAi?$AAP?$AAl?$AAu?$AAs?$AA?4?$AAd?$AAl?$AAl?$AA?$AA@ 00000001800123b0     gdip.obj
 0002:000003c8       ??_C@_0P@NIGHOHPH@GdiplusStartup?$AA@ 00000001800123c8     gdip.obj
 0002:000003d8       ??_C@_0BA@OMKIAPCJ@GdiplusShutdown?$AA@ 00000001800123d8     gdip.obj
 0002:000003e8       ??_C@_0BJ@IPKMAACN@GdipCreateBitmapFromFile?$AA@ 00000001800123e8     gdip.obj
 0002:00000408       ??_C@_0BG@OPKFAGML@GdipGetImageThumbnail?$AA@ 0000000180012408     gdip.obj
 0002:00000420       ??_C@_0BC@DPLNHGNM@GdipGetImageWidth?$AA@ 0000000180012420     gdip.obj
 0002:00000438       ??_C@_0BD@JIGBIPOH@GdipGetImageHeight?$AA@ 0000000180012438     gdip.obj
 0002:00000450       ??_C@_0BI@DDNLFBKI@GdipGetImagePixelFormat?$AA@ 0000000180012450     gdip.obj
 0002:00000468       ??_C@_0BB@MGCHKKMH@GdipDisposeImage?$AA@ 0000000180012468     gdip.obj
 0002:00000480       ??_C@_0BH@PCHOHMFI@GdipImageGetFrameCount?$AA@ 0000000180012480     gdip.obj
 0002:00000498       ??_C@_0BL@FLMDGKNM@GdipImageSelectActiveFrame?$AA@ 0000000180012498     gdip.obj
 0002:000004b8       ??_C@_0BI@PFDIBLKB@GdipGetPropertyItemSize?$AA@ 00000001800124b8     gdip.obj
 0002:000004d0       ??_C@_0BE@JLBHAGMH@GdipGetPropertyItem?$AA@ 00000001800124d0     gdip.obj
 0002:000004e8       ??_C@_0BE@HNMMICFD@GdipImageRotateFlip?$AA@ 00000001800124e8     gdip.obj
 0002:00000500       ??_C@_0BG@BONHLFMI@GdipGetImageRawFormat?$AA@ 0000000180012500     gdip.obj
 0002:00000518       ??_C@_0BC@PACDIGJN@GdipCreateFromHDC?$AA@ 0000000180012518     gdip.obj
 0002:00000530       ??_C@_0BD@MFGJCODH@GdipDeleteGraphics?$AA@ 0000000180012530     gdip.obj
 0002:00000548       ??_C@_0BH@MHAPNLKM@GdipDrawImageRectRectI?$AA@ 0000000180012548     gdip.obj
 0002:00000560       ??_C@_0BF@OBPAMLNN@gdip?3?3FreeThreadProc?$AA@ 0000000180012560     gdip.obj
 0002:00000580       ??_C@_0EA@GIECIGNA@t?3?2vcproject?2maximus5?2conemu?2src@ 0000000180012580     gdip.obj
 0002:000005c0       ??_C@_17CGDFOGLC@?$AAC?$AAE?$AAT?$AA?$AA@ 00000001800125c0     gdip.obj
 0002:000005c8       ??_C@_19JJJNAIHN@?$AAJ?$AAP?$AAE?$AAG?$AA?$AA@ 00000001800125c8     gdip.obj
 0002:000005d8       ??_C@_19PNCGIGON@?$AAT?$AAI?$AAF?$AAF?$AA?$AA@ 00000001800125d8     gdip.obj
 0002:000005e8       ??_C@_19HEANOPFL@?$AAE?$AAX?$AAI?$AAF?$AA?$AA@ 00000001800125e8     gdip.obj
 0002:000005f8       ??_C@_1CA@KKEPPKFF@?$AA?$CF?$AAi?$AA?5?$AAx?$AA?5?$AA?$CF?$AAi?$AA?5?$AAx?$AA?5?$AA?$CF?$AAi?$AAb?$AAp?$AAp?$AA?$AA@ 00000001800125f8     gdip.obj
 0002:00000618       ??_C@_1M@HKOFHKAI@?$AA?5?$AA?$FL?$AA?$CF?$AAi?$AA?$FN?$AA?$AA@ 0000000180012618     gdip.obj
 0002:00000624       ??_C@_13HOIJIPNN@?$AA?5?$AA?$AA@ 0000000180012624     gdip.obj
 0002:00000628       ??_C@_05LCABBMOG@?$CFs?3?$CFi?$AA@ 0000000180012628     common-kernel64:WThreads.obj
 0002:00000640       _pRawDllMain               0000000180012640     LIBCMT:dll_dllmain.obj
 0002:00000640       _pDefaultRawDllMain        0000000180012640     LIBCMT:dll_dllmain.obj
 0002:00000980       ??_C@_08EHJDFFNH@__based?$CI?$AA@ 0000000180012980     libvcruntime:undname.obj
 0002:00000990       ??_C@_07KOLFKCDI@__cdecl?$AA@ 0000000180012990     libvcruntime:undname.obj
 0002:00000998       ??_C@_08GHMPAG@__pascal?$AA@ 0000000180012998     libvcruntime:undname.obj
 0002:000009a8       ??_C@_09IFJBGAPI@__stdcall?$AA@ 00000001800129a8     libvcruntime:undname.obj
 0002:000009b8       ??_C@_0L@NPHFGOKO@__thiscall?$AA@ 00000001800129b8     libvcruntime:undname.obj
 0002:000009c8       ??_C@_0L@JMKHOMEK@__fastcall?$AA@ 00000001800129c8     libvcruntime:undname.obj
 0002:000009d8       ??_C@_0N@BCKKPABJ@__vectorcall?$AA@ 00000001800129d8     libvcruntime:undname.obj
 0002:000009e8       ??_C@_09HIJEGCPM@__clrcall?$AA@ 00000001800129e8     libvcruntime:undname.obj
 0002:000009f4       ??_C@_06GHPCKEAG@__eabi?$AA@ 00000001800129f4     libvcruntime:undname.obj
 0002:00000a00       ??_C@_07EECFKIPL@__swift?$AA@ 0000000180012a00     libvcruntime:undname.obj
 0002:00000a08       ??_C@_07JOMMBBKO@__ptr64?$AA@ 0000000180012a08     libvcruntime:undname.obj
 0002:00000a10       ??_C@_0L@PILCLIHE@__restrict?$AA@ 0000000180012a10     libvcruntime:undname.obj
 0002:00000a20       ??_C@_0M@GFIIJFMG@__unaligned?$AA@ 0000000180012a20     libvcruntime:undname.obj
 0002:00000a30       ??_C@_09DHDLOLLB@restrict?$CI?$AA@ 0000000180012a30     libvcruntime:undname.obj
 0002:00000a3a       ??_C@_00CNPNBAHC@?$AA@     0000000180012a3a     libvcruntime:undname.obj
 0002:00000a3c       ??_C@_04NIHEBCM@?5new?$AA@ 0000000180012a3c     libvcruntime:undname.obj
 0002:00000a48       ??_C@_07FPCDHGMM@?5delete?$AA@ 0000000180012a48     libvcruntime:undname.obj
 0002:00000a50       ??_C@_01NEMOKFLO@?$DN?$AA@ 0000000180012a50     libvcruntime:undname.obj
 0002:00000a54       ??_C@_02GPIOPFAK@?$DO?$DO?$AA@ 0000000180012a54     libvcruntime:undname.obj
 0002:00000a58       ??_C@_02FODMEDOG@?$DM?$DM?$AA@ 0000000180012a58     libvcruntime:undname.obj
 0002:00000a5c       ??_C@_01DCLJPIOD@?$CB?$AA@ 0000000180012a5c     libvcruntime:undname.obj
 0002:00000a60       ??_C@_02EGOFBIJA@?$DN?$DN?$AA@ 0000000180012a60     libvcruntime:undname.obj
 0002:00000a64       ??_C@_02FDNJECIE@?$CB?$DN?$AA@ 0000000180012a64     libvcruntime:undname.obj
 0002:00000a68       ??_C@_02GPECMEKF@?$FL?$FN?$AA@ 0000000180012a68     libvcruntime:undname.obj
 0002:00000a70       ??_C@_08LHJFAFGD@operator?$AA@ 0000000180012a70     libvcruntime:undname.obj
 0002:00000a7c       ??_C@_02HBOOOICD@?9?$DO?$AA@ 0000000180012a7c     libvcruntime:undname.obj
 0002:00000a80       ??_C@_01NBENCBCI@?$CK?$AA@ 0000000180012a80     libvcruntime:undname.obj
 0002:00000a84       ??_C@_02ECNGHCIF@?$CL?$CL?$AA@ 0000000180012a84     libvcruntime:undname.obj
 0002:00000a88       ??_C@_02BAABKJLB@?9?9?$AA@ 0000000180012a88     libvcruntime:undname.obj
 0002:00000a8c       ??_C@_01JOAMLHOP@?9?$AA@   0000000180012a8c     libvcruntime:undname.obj
 0002:00000a90       ??_C@_01MIFGBAGJ@?$CL?$AA@ 0000000180012a90     libvcruntime:undname.obj
 0002:00000a94       ??_C@_01HNPIGOCE@?$CG?$AA@ 0000000180012a94     libvcruntime:undname.obj
 0002:00000a98       ??_C@_03MNHNFDLC@?9?$DO?$CK?$AA@ 0000000180012a98     libvcruntime:undname.obj
 0002:00000a9c       ??_C@_01KMDKNFGN@?1?$AA@   0000000180012a9c     libvcruntime:undname.obj
 0002:00000aa0       ??_C@_01FGNFDNOH@?$CF?$AA@ 0000000180012aa0     libvcruntime:undname.obj
 0002:00000aa4       ??_C@_01MNNFJEPP@?$DM?$AA@ 0000000180012aa4     libvcruntime:undname.obj
 0002:00000aa8       ??_C@_02EHCHHCKH@?$DM?$DN?$AA@ 0000000180012aa8     libvcruntime:undname.obj
 0002:00000aac       ??_C@_01PPODPGHN@?$DO?$AA@ 0000000180012aac     libvcruntime:undname.obj
 0002:00000ab0       ??_C@_02EEKDKGMJ@?$DO?$DN?$AA@ 0000000180012ab0     libvcruntime:undname.obj
 0002:00000ab4       ??_C@_01IHBHIGKO@?0?$AA@   0000000180012ab4     libvcruntime:undname.obj
 0002:00000ab8       ??_C@_02HCKGKOFO@?$CI?$CJ?$AA@ 0000000180012ab8     libvcruntime:undname.obj
 0002:00000abc       ??_C@_01PJKLJHI@?$HO?$AA@  0000000180012abc     libvcruntime:undname.obj
 0002:00000ac0       ??_C@_01JKBOJNNK@?$FO?$AA@ 0000000180012ac0     libvcruntime:undname.obj
 0002:00000ac4       ??_C@_01DNKMNLPK@?$HM?$AA@ 0000000180012ac4     libvcruntime:undname.obj
 0002:00000ac8       ??_C@_02PPKAJPJL@?$CG?$CG?$AA@ 0000000180012ac8     libvcruntime:undname.obj
 0002:00000acc       ??_C@_02NONPIBCD@?$HM?$HM?$AA@ 0000000180012acc     libvcruntime:undname.obj
 0002:00000ad0       ??_C@_02FPIMKNGF@?$CK?$DN?$AA@ 0000000180012ad0     libvcruntime:undname.obj
 0002:00000ad4       ??_C@_02FOEOMHFC@?$CL?$DN?$AA@ 0000000180012ad4     libvcruntime:undname.obj
 0002:00000ad8       ??_C@_02FKMDLLOA@?9?$DN?$AA@ 0000000180012ad8     libvcruntime:undname.obj
 0002:00000adc       ??_C@_02FJEHGPIO@?1?$DN?$AA@ 0000000180012adc     libvcruntime:undname.obj
 0002:00000ae0       ??_C@_02FENAOKFI@?$CF?$DN?$AA@ 0000000180012ae0     libvcruntime:undname.obj
 0002:00000ae4       ??_C@_03IKFCCPFF@?$DO?$DO?$DN?$AA@ 0000000180012ae4     libvcruntime:undname.obj
 0002:00000ae8       ??_C@_03CDNPDDLA@?$DM?$DM?$DN?$AA@ 0000000180012ae8     libvcruntime:undname.obj
 0002:00000aec       ??_C@_02FGJGFEAB@?$CG?$DN?$AA@ 0000000180012aec     libvcruntime:undname.obj
 0002:00000af0       ??_C@_02DHLNPPGH@?$HM?$DN?$AA@ 0000000180012af0     libvcruntime:undname.obj
 0002:00000af4       ??_C@_02MHEGNOJ@?$FO?$DN?$AA@ 0000000180012af4     libvcruntime:undname.obj
 0002:00000af8       ??_C@_09IFPLHPGF@?$GAvftable?8?$AA@ 0000000180012af8     libvcruntime:undname.obj
 0002:00000b08       ??_C@_09BLBHBJP@?$GAvbtable?8?$AA@ 0000000180012b08     libvcruntime:undname.obj
 0002:00000b18       ??_C@_07FEEIOKP@?$GAvcall?8?$AA@ 0000000180012b18     libvcruntime:undname.obj
 0002:00000b20       ??_C@_08LLFFHHDJ@?$GAtypeof?8?$AA@ 0000000180012b20     libvcruntime:undname.obj
 0002:00000b30       ??_C@_0BF@KDPPACIK@?$GAlocal?5static?5guard?8?$AA@ 0000000180012b30     libvcruntime:undname.obj
 0002:00000b48       ??_C@_08OBABFOLI@?$GAstring?8?$AA@ 0000000180012b48     libvcruntime:undname.obj
 0002:00000b58       ??_C@_0BD@JDLKDPAB@?$GAvbase?5destructor?8?$AA@ 0000000180012b58     libvcruntime:undname.obj
 0002:00000b70       ??_C@_0BN@DEGPLNFK@?$GAvector?5deleting?5destructor?8?$AA@ 0000000180012b70     libvcruntime:undname.obj
 0002:00000b90       ??_C@_0BO@OBMKPJIG@?$GAdefault?5constructor?5closure?8?$AA@ 0000000180012b90     libvcruntime:undname.obj
 0002:00000bb0       ??_C@_0BN@IMDCHIKM@?$GAscalar?5deleting?5destructor?8?$AA@ 0000000180012bb0     libvcruntime:undname.obj
 0002:00000bd0       ??_C@_0BO@PFGOCPJJ@?$GAvector?5constructor?5iterator?8?$AA@ 0000000180012bd0     libvcruntime:undname.obj
 0002:00000bf0       ??_C@_0BN@LFPFMEDL@?$GAvector?5destructor?5iterator?8?$AA@ 0000000180012bf0     libvcruntime:undname.obj
 0002:00000c10       ??_C@_0CE@IKBNEHA@?$GAvector?5vbase?5constructor?5iterat@ 0000000180012c10     libvcruntime:undname.obj
 0002:00000c38       ??_C@_0BL@NILFHHPC@?$GAvirtual?5displacement?5map?8?$AA@ 0000000180012c38     libvcruntime:undname.obj
 0002:00000c58       ??_C@_0CB@JONCMFFK@?$GAeh?5vector?5constructor?5iterator?8@ 0000000180012c58     libvcruntime:undname.obj
 0002:00000c80       ??_C@_0CA@GCEOPDGL@?$GAeh?5vector?5destructor?5iterator?8?$AA@ 0000000180012c80     libvcruntime:undname.obj
 0002:00000ca0       ??_C@_0CH@OOJPLCPH@?$GAeh?5vector?5vbase?5constructor?5ite@ 0000000180012ca0     libvcruntime:undname.obj
 0002:00000cc8       ??_C@_0BL@LLKPOHJI@?$GAcopy?5constructor?5closure?8?$AA@ 0000000180012cc8     libvcruntime:undname.obj
 0002:00000ce8       ??_C@_0BA@KBCDOMBN@?$GAudt?5returning?8?$AA@ 0000000180012ce8     libvcruntime:undname.obj
 0002:00000cf8       ??_C@_03KLGMFNMG@?$GAEH?$AA@ 0000000180012cf8     libvcruntime:undname.obj
 0002:00000cfc       ??_C@_05KHLCHHI@?$GARTTI?$AA@ 0000000180012cfc     libvcruntime:undname.obj
 0002:00000d08       ??_C@_0BA@KKLDJDLB@?$GAlocal?5vftable?8?$AA@ 0000000180012d08     libvcruntime:undname.obj
 0002:00000d18       ??_C@_0CE@IIHCMGGL@?$GAlocal?5vftable?5constructor?5closu@ 0000000180012d18     libvcruntime:undname.obj
 0002:00000d3c       ??_C@_06FHBGPFGH@?5new?$FL?$FN?$AA@ 0000000180012d3c     libvcruntime:undname.obj
 0002:00000d48       ??_C@_09LBNFPBCA@?5delete?$FL?$FN?$AA@ 0000000180012d48     libvcruntime:undname.obj
 0002:00000d58       ??_C@_0P@HJKNJFNN@?$GAomni?5callsig?8?$AA@ 0000000180012d58     libvcruntime:undname.obj
 0002:00000d68       ??_C@_0BL@CNOONJFP@?$GAplacement?5delete?5closure?8?$AA@ 0000000180012d68     libvcruntime:undname.obj
 0002:00000d88       ??_C@_0BN@CKNJLHMB@?$GAplacement?5delete?$FL?$FN?5closure?8?$AA@ 0000000180012d88     libvcruntime:undname.obj
 0002:00000da8       ??_C@_0CG@CFDHKGGD@?$GAmanaged?5vector?5constructor?5iter@ 0000000180012da8     libvcruntime:undname.obj
 0002:00000dd0       ??_C@_0CF@IMGKMJNO@?$GAmanaged?5vector?5destructor?5itera@ 0000000180012dd0     libvcruntime:undname.obj
 0002:00000df8       ??_C@_0CG@HLDDJMAG@?$GAeh?5vector?5copy?5constructor?5iter@ 0000000180012df8     libvcruntime:undname.obj
 0002:00000e20       ??_C@_0CM@FCBBDIGB@?$GAeh?5vector?5vbase?5copy?5constructo@ 0000000180012e20     libvcruntime:undname.obj
 0002:00000e50       ??_C@_0BL@CLIPGLGB@?$GAdynamic?5initializer?5for?5?8?$AA@ 0000000180012e50     libvcruntime:undname.obj
 0002:00000e70       ??_C@_0CB@PDBIFEP@?$GAdynamic?5atexit?5destructor?5for?5?8@ 0000000180012e70     libvcruntime:undname.obj
 0002:00000e98       ??_C@_0CD@CGAJBKEJ@?$GAvector?5copy?5constructor?5iterato@ 0000000180012e98     libvcruntime:undname.obj
 0002:00000ec0       ??_C@_0CJ@GJELGAMM@?$GAvector?5vbase?5copy?5constructor?5i@ 0000000180012ec0     libvcruntime:undname.obj
 0002:00000ef0       ??_C@_0CL@FGIJHLCE@?$GAmanaged?5vector?5copy?5constructor@ 0000000180012ef0     libvcruntime:undname.obj
 0002:00000f20       ??_C@_0BM@PMGGMLDN@?$GAlocal?5static?5thread?5guard?8?$AA@ 0000000180012f20     libvcruntime:undname.obj
 0002:00000f40       ??_C@_0N@BDNMDMOL@operator?5?$CC?$CC?5?$AA@ 0000000180012f40     libvcruntime:undname.obj
 0002:00000f50       ??_C@_0BC@GGEBGALA@operator?5co_await?$AA@ 0000000180012f50     libvcruntime:undname.obj
 0002:00000f68       ??_C@_0BC@DAFEJGAK@?5Type?5Descriptor?8?$AA@ 0000000180012f68     libvcruntime:undname.obj
 0002:00000f80       ??_C@_0BM@LDKODKLH@?5Base?5Class?5Descriptor?5at?5?$CI?$AA@ 0000000180012f80     libvcruntime:undname.obj
 0002:00000fa0       ??_C@_0BD@LGICGFMM@?5Base?5Class?5Array?8?$AA@ 0000000180012fa0     libvcruntime:undname.obj
 0002:00000fb8       ??_C@_0BN@MECKDCOJ@?5Class?5Hierarchy?5Descriptor?8?$AA@ 0000000180012fb8     libvcruntime:undname.obj
 0002:00000fd8       ??_C@_0BK@CFCOFLF@?5Complete?5Object?5Locator?8?$AA@ 0000000180012fd8     libvcruntime:undname.obj
 0002:00001010       ??_C@_1DM@KHCHBNEB@?$AAa?$AAp?$AAi?$AA?9?$AAm?$AAs?$AA?9?$AAw?$AAi?$AAn?$AA?9?$AAc?$AAo?$AAr?$AAe?$AA?9?$AAf?$AAi?$AAb?$AAe?$AAr?$AAs?$AA?9?$AAl?$AA1?$AA?9?$AA1?$AA?9?$AA1?$AA?$AA@ 0000000180013010     libvcruntime:winapi_downlevel.obj
 0002:00001050       ??_C@_1DK@LPPGFMPP@?$AAa?$AAp?$AAi?$AA?9?$AAm?$AAs?$AA?9?$AAw?$AAi?$AAn?$AA?9?$AAc?$AAo?$AAr?$AAe?$AA?9?$AAs?$AAy?$AAn?$AAc?$AAh?$AA?9?$AAl?$AA1?$AA?9?$AA2?$AA?9?$AA0?$AA?$AA@ 0000000180013050     libvcruntime:winapi_downlevel.obj
 0002:00001090       ??_C@_1BC@GDMECMAK@?$AAk?$AAe?$AAr?$AAn?$AAe?$AAl?$AA3?$AA2?$AA?$AA@ 0000000180013090     libvcruntime:winapi_downlevel.obj
 0002:000010a8       ??_C@_1BA@PFFKHIOG@?$AAa?$AAp?$AAi?$AA?9?$AAm?$AAs?$AA?9?$AA?$AA@ 00000001800130a8     libvcruntime:winapi_downlevel.obj
 0002:000010b8       ??_C@_1BA@IAIFMGEF@?$AAe?$AAx?$AAt?$AA?9?$AAm?$AAs?$AA?9?$AA?$AA@ 00000001800130b8     libvcruntime:winapi_downlevel.obj
 0002:000010d0       ??_C@_08KNHFBNJ@FlsAlloc?$AA@ 00000001800130d0     libvcruntime:winapi_downlevel.obj
 0002:000010e8       ??_C@_07PEJMOBNF@FlsFree?$AA@ 00000001800130e8     libvcruntime:winapi_downlevel.obj
 0002:000010f8       ??_C@_0M@GDNOONDI@FlsGetValue?$AA@ 00000001800130f8     libvcruntime:winapi_downlevel.obj
 0002:00001110       ??_C@_0M@JCPCPOEF@FlsSetValue?$AA@ 0000000180013110     libvcruntime:winapi_downlevel.obj
 0002:00001128       ??_C@_0BM@HCFOFFN@InitializeCriticalSectionEx?$AA@ 0000000180013128     libvcruntime:winapi_downlevel.obj
 0002:00001148       _pDestructExceptionObject  0000000180013148     libvcruntime:ehhelpers.obj
 0002:00001150       standard_lookup_table      0000000180013150     libucrt:output.obj
 0002:000011ac       ??_C@_06OJHGLDPL@?$CInull?$CJ?$AA@ 00000001800131ac     libucrt:output.obj
 0002:000011b8       ??_C@_1O@CEDCILHN@?$AA?$CI?$AAn?$AAu?$AAl?$AAl?$AA?$CJ?$AA?$AA@ 00000001800131b8     libucrt:output.obj
 0002:000011d0       __acrt_exception_action_table 00000001800131d0     libucrt:exception_filter.obj
 0002:00001290       __acrt_signal_action_table_count 0000000180013290     libucrt:exception_filter.obj
 0002:00001298       __acrt_signal_action_first_fpe_index 0000000180013298     libucrt:exception_filter.obj
 0002:000012a0       __acrt_signal_action_fpe_count 00000001800132a0     libucrt:exception_filter.obj
 0002:000012a8       ??_C@_1BI@BGOHAHKC@?$AAm?$AAs?$AAc?$AAo?$AAr?$AAe?$AAe?$AA?4?$AAd?$AAl?$AAl?$AA?$AA@ 00000001800132a8     libucrt:exit.obj
 0002:000012c0       ??_C@_0P@MIGLKIOC@CorExitProcess?$AA@ 00000001800132c0     libucrt:exit.obj
 0002:00001528       ??_C@_03OEIAHPBN@INF?$AA@  0000000180013528     libucrt:cvt.obj
 0002:0000152c       ??_C@_03OJHLLCGB@inf?$AA@  000000018001352c     libucrt:cvt.obj
 0002:00001530       ??_C@_03LKNCIKJB@NAN?$AA@  0000000180013530     libucrt:cvt.obj
 0002:00001534       ??_C@_03LHCJEHON@nan?$AA@  0000000180013534     libucrt:cvt.obj
 0002:00001538       ??_C@_09OFJJIMPC@NAN?$CISNAN?$CJ?$AA@ 0000000180013538     libucrt:cvt.obj
 0002:00001548       ??_C@_09IPFBKMDL@nan?$CIsnan?$CJ?$AA@ 0000000180013548     libucrt:cvt.obj
 0002:00001558       ??_C@_08IKHNHAJ@NAN?$CIIND?$CJ?$AA@ 0000000180013558     libucrt:cvt.obj
 0002:00001568       ??_C@_08OFCDMILK@nan?$CIind?$CJ?$AA@ 0000000180013568     libucrt:cvt.obj
 0002:00001574       ??_C@_05KLBDPFGC@e?$CL000?$AA@ 0000000180013574     libucrt:cvt.obj
 0002:00001580       __lc_time_c                0000000180013580     libucrt:nlsdata.obj
 0002:00001840       ??_C@_03KOEHGMDN@Sun?$AA@  0000000180013840     libucrt:nlsdata.obj
 0002:00001844       ??_C@_03PDAGKDH@Mon?$AA@   0000000180013844     libucrt:nlsdata.obj
 0002:00001848       ??_C@_03NAGEINEP@Tue?$AA@  0000000180013848     libucrt:nlsdata.obj
 0002:0000184c       ??_C@_03MHOMLAJA@Wed?$AA@  000000018001384c     libucrt:nlsdata.obj
 0002:00001850       ??_C@_03IOFIKPDN@Thu?$AA@  0000000180013850     libucrt:nlsdata.obj
 0002:00001854       ??_C@_03IDIOELNC@Fri?$AA@  0000000180013854     libucrt:nlsdata.obj
 0002:00001858       ??_C@_03FEFJNEK@Sat?$AA@   0000000180013858     libucrt:nlsdata.obj
 0002:0000185c       ??_C@_06OOPIFAJ@Sunday?$AA@ 000000018001385c     libucrt:nlsdata.obj
 0002:00001864       ??_C@_06JLEDEDGH@Monday?$AA@ 0000000180013864     libucrt:nlsdata.obj
 0002:00001870       ??_C@_07BAAGCFCM@Tuesday?$AA@ 0000000180013870     libucrt:nlsdata.obj
 0002:00001878       ??_C@_09DLIGFAKA@Wednesday?$AA@ 0000000180013878     libucrt:nlsdata.obj
 0002:00001888       ??_C@_08HACCIKIA@Thursday?$AA@ 0000000180013888     libucrt:nlsdata.obj
 0002:00001894       ??_C@_06JECMNKMI@Friday?$AA@ 0000000180013894     libucrt:nlsdata.obj
 0002:000018a0       ??_C@_08INBOOONO@Saturday?$AA@ 00000001800138a0     libucrt:nlsdata.obj
 0002:000018ac       ??_C@_03JIHJHPIE@Jan?$AA@  00000001800138ac     libucrt:nlsdata.obj
 0002:000018b0       ??_C@_03HJBDCHOM@Feb?$AA@  00000001800138b0     libucrt:nlsdata.obj
 0002:000018b4       ??_C@_03ODNJBKGA@Mar?$AA@  00000001800138b4     libucrt:nlsdata.obj
 0002:000018b8       ??_C@_03LEOLGMJP@Apr?$AA@  00000001800138b8     libucrt:nlsdata.obj
 0002:000018bc       ??_C@_03CNMDKL@May?$AA@    00000001800138bc     libucrt:nlsdata.obj
 0002:000018c0       ??_C@_03IDFGHECI@Jun?$AA@  00000001800138c0     libucrt:nlsdata.obj
 0002:000018c4       ??_C@_03LBGABGKK@Jul?$AA@  00000001800138c4     libucrt:nlsdata.obj
 0002:000018c8       ??_C@_03IFJFEIGA@Aug?$AA@  00000001800138c8     libucrt:nlsdata.obj
 0002:000018cc       ??_C@_03GGCAPAJC@Sep?$AA@  00000001800138cc     libucrt:nlsdata.obj
 0002:000018d0       ??_C@_03BMAOKBAD@Oct?$AA@  00000001800138d0     libucrt:nlsdata.obj
 0002:000018d4       ??_C@_03JPJOFNIA@Nov?$AA@  00000001800138d4     libucrt:nlsdata.obj
 0002:000018d8       ??_C@_03MKABNOCG@Dec?$AA@  00000001800138d8     libucrt:nlsdata.obj
 0002:000018e0       ??_C@_07CGJPFGJA@January?$AA@ 00000001800138e0     libucrt:nlsdata.obj
 0002:000018e8       ??_C@_08GNJGEPFN@February?$AA@ 00000001800138e8     libucrt:nlsdata.obj
 0002:000018f4       ??_C@_05HPCKOFNC@March?$AA@ 00000001800138f4     libucrt:nlsdata.obj
 0002:000018fc       ??_C@_05DMJDNLEJ@April?$AA@ 00000001800138fc     libucrt:nlsdata.obj
 0002:00001904       ??_C@_04CNLMGBGM@June?$AA@ 0000000180013904     libucrt:nlsdata.obj
 0002:0000190c       ??_C@_04MIEPOIFP@July?$AA@ 000000018001390c     libucrt:nlsdata.obj
 0002:00001914       ??_C@_06LBBHFDDG@August?$AA@ 0000000180013914     libucrt:nlsdata.obj
 0002:00001920       ??_C@_09BHHEALKD@September?$AA@ 0000000180013920     libucrt:nlsdata.obj
 0002:00001930       ??_C@_07JJNFCEND@October?$AA@ 0000000180013930     libucrt:nlsdata.obj
 0002:00001938       ??_C@_08HCHEGEOA@November?$AA@ 0000000180013938     libucrt:nlsdata.obj
 0002:00001948       ??_C@_08EDHMEBNP@December?$AA@ 0000000180013948     libucrt:nlsdata.obj
 0002:00001954       ??_C@_02DEDBPAFC@AM?$AA@   0000000180013954     libucrt:nlsdata.obj
 0002:00001958       ??_C@_02CJNFDJBF@PM?$AA@   0000000180013958     libucrt:nlsdata.obj
 0002:00001960       ??_C@_08BPBNCDIB@MM?1dd?1yy?$AA@ 0000000180013960     libucrt:nlsdata.obj
 0002:00001970       ??_C@_0BE@CKGJFCPC@dddd?0?5MMMM?5dd?0?5yyyy?$AA@ 0000000180013970     libucrt:nlsdata.obj
 0002:00001988       ??_C@_08JCCMCCIL@HH?3mm?3ss?$AA@ 0000000180013988     libucrt:nlsdata.obj
 0002:00001998       ??_C@_17MBGCMIPB@?$AAS?$AAu?$AAn?$AA?$AA@ 0000000180013998     libucrt:nlsdata.obj
 0002:000019a0       ??_C@_17KBOMKBF@?$AAM?$AAo?$AAn?$AA?$AA@ 00000001800139a0     libucrt:nlsdata.obj
 0002:000019a8       ??_C@_17BMKGEGOJ@?$AAT?$AAu?$AAe?$AA?$AA@ 00000001800139a8     libucrt:nlsdata.obj
 0002:000019b0       ??_C@_17CJEDCEPE@?$AAW?$AAe?$AAd?$AA?$AA@ 00000001800139b0     libucrt:nlsdata.obj
 0002:000019b8       ??_C@_17PDPHAADD@?$AAT?$AAh?$AAu?$AA?$AA@ 00000001800139b8     libucrt:nlsdata.obj
 0002:000019c0       ??_C@_17HFOLPPLP@?$AAF?$AAr?$AAi?$AA?$AA@ 00000001800139c0     libucrt:nlsdata.obj
 0002:000019c8       ??_C@_17GGIBDPIH@?$AAS?$AAa?$AAt?$AA?$AA@ 00000001800139c8     libucrt:nlsdata.obj
 0002:000019d0       ??_C@_1O@IHNHDHPB@?$AAS?$AAu?$AAn?$AAd?$AAa?$AAy?$AA?$AA@ 00000001800139d0     libucrt:nlsdata.obj
 0002:000019e0       ??_C@_1O@MMNBFLIA@?$AAM?$AAo?$AAn?$AAd?$AAa?$AAy?$AA?$AA@ 00000001800139e0     libucrt:nlsdata.obj
 0002:000019f0       ??_C@_1BA@ENFBFFEK@?$AAT?$AAu?$AAe?$AAs?$AAd?$AAa?$AAy?$AA?$AA@ 00000001800139f0     libucrt:nlsdata.obj
 0002:00001a00       ??_C@_1BE@EBOGMDOH@?$AAW?$AAe?$AAd?$AAn?$AAe?$AAs?$AAd?$AAa?$AAy?$AA?$AA@ 0000000180013a00     libucrt:nlsdata.obj
 0002:00001a18       ??_C@_1BC@HHMNLIHE@?$AAT?$AAh?$AAu?$AAr?$AAs?$AAd?$AAa?$AAy?$AA?$AA@ 0000000180013a18     libucrt:nlsdata.obj
 0002:00001a30       ??_C@_1O@PDICJHAG@?$AAF?$AAr?$AAi?$AAd?$AAa?$AAy?$AA?$AA@ 0000000180013a30     libucrt:nlsdata.obj
 0002:00001a40       ??_C@_1BC@ENMNNPAJ@?$AAS?$AAa?$AAt?$AAu?$AAr?$AAd?$AAa?$AAy?$AA?$AA@ 0000000180013a40     libucrt:nlsdata.obj
 0002:00001a58       ??_C@_17DKNBKCHM@?$AAJ?$AAa?$AAn?$AA?$AA@ 0000000180013a58     libucrt:nlsdata.obj
 0002:00001a60       ??_C@_17LMDJEKJN@?$AAF?$AAe?$AAb?$AA?$AA@ 0000000180013a60     libucrt:nlsdata.obj
 0002:00001a68       ??_C@_17CKNLEDEC@?$AAM?$AAa?$AAr?$AA?$AA@ 0000000180013a68     libucrt:nlsdata.obj
 0002:00001a70       ??_C@_17LFPOIHDD@?$AAA?$AAp?$AAr?$AA?$AA@ 0000000180013a70     libucrt:nlsdata.obj
 0002:00001a78       ??_C@_17PNNKMEED@?$AAM?$AAa?$AAy?$AA?$AA@ 0000000180013a78     libucrt:nlsdata.obj
 0002:00001a80       ??_C@_17KCJGOCPB@?$AAJ?$AAu?$AAn?$AA?$AA@ 0000000180013a80     libucrt:nlsdata.obj
 0002:00001a88       ??_C@_17IJPCKHK@?$AAJ?$AAu?$AAl?$AA?$AA@ 0000000180013a88     libucrt:nlsdata.obj
 0002:00001a90       ??_C@_17ICPELBCN@?$AAA?$AAu?$AAg?$AA?$AA@ 0000000180013a90     libucrt:nlsdata.obj
 0002:00001a98       ??_C@_17HCHCOKMG@?$AAS?$AAe?$AAp?$AA?$AA@ 0000000180013a98     libucrt:nlsdata.obj
 0002:00001aa0       ??_C@_17FNLKOI@?$AAO?$AAc?$AAt?$AA?$AA@ 0000000180013aa0     libucrt:nlsdata.obj
 0002:00001aa8       ??_C@_17BBDMLCIG@?$AAN?$AAo?$AAv?$AA?$AA@ 0000000180013aa8     libucrt:nlsdata.obj
 0002:00001ab0       ??_C@_17EGKACKIF@?$AAD?$AAe?$AAc?$AA?$AA@ 0000000180013ab0     libucrt:nlsdata.obj
 0002:00001ab8       ??_C@_1BA@EFMEIEBA@?$AAJ?$AAa?$AAn?$AAu?$AAa?$AAr?$AAy?$AA?$AA@ 0000000180013ab8     libucrt:nlsdata.obj
 0002:00001ac8       ??_C@_1BC@JGDDFFAM@?$AAF?$AAe?$AAb?$AAr?$AAu?$AAa?$AAr?$AAy?$AA?$AA@ 0000000180013ac8     libucrt:nlsdata.obj
 0002:00001ae0       ??_C@_1M@IKEENEDF@?$AAM?$AAa?$AAr?$AAc?$AAh?$AA?$AA@ 0000000180013ae0     libucrt:nlsdata.obj
 0002:00001af0       ??_C@_1M@GJNLMHFD@?$AAA?$AAp?$AAr?$AAi?$AAl?$AA?$AA@ 0000000180013af0     libucrt:nlsdata.obj
 0002:00001b00       ??_C@_19EPFLPGAP@?$AAJ?$AAu?$AAn?$AAe?$AA?$AA@ 0000000180013b00     libucrt:nlsdata.obj
 0002:00001b10       ??_C@_19BIFMLPCD@?$AAJ?$AAu?$AAl?$AAy?$AA?$AA@ 0000000180013b10     libucrt:nlsdata.obj
 0002:00001b20       ??_C@_1O@PAHLKOAC@?$AAA?$AAu?$AAg?$AAu?$AAs?$AAt?$AA?$AA@ 0000000180013b20     libucrt:nlsdata.obj
 0002:00001b30       ??_C@_1BE@DKAAMBJL@?$AAS?$AAe?$AAp?$AAt?$AAe?$AAm?$AAb?$AAe?$AAr?$AA?$AA@ 0000000180013b30     libucrt:nlsdata.obj
 0002:00001b48       ??_C@_1BA@EPANDLNG@?$AAO?$AAc?$AAt?$AAo?$AAb?$AAe?$AAr?$AA?$AA@ 0000000180013b48     libucrt:nlsdata.obj
 0002:00001b58       ??_C@_1BC@BGLIFPF@?$AAN?$AAo?$AAv?$AAe?$AAm?$AAb?$AAe?$AAr?$AA?$AA@ 0000000180013b58     libucrt:nlsdata.obj
 0002:00001b70       ??_C@_1BC@FEMKIFH@?$AAD?$AAe?$AAc?$AAe?$AAm?$AAb?$AAe?$AAr?$AA?$AA@ 0000000180013b70     libucrt:nlsdata.obj
 0002:00001b84       ??_C@_15ODEHAHHF@?$AAA?$AAM?$AA?$AA@ 0000000180013b84     libucrt:nlsdata.obj
 0002:00001b8c       ??_C@_15CLMNNGEL@?$AAP?$AAM?$AA?$AA@ 0000000180013b8c     libucrt:nlsdata.obj
 0002:00001b98       ??_C@_1BC@IEBCMHCM@?$AAM?$AAM?$AA?1?$AAd?$AAd?$AA?1?$AAy?$AAy?$AA?$AA@ 0000000180013b98     libucrt:nlsdata.obj
 0002:00001bb0       ??_C@_1CI@KNAKOEBC@?$AAd?$AAd?$AAd?$AAd?$AA?0?$AA?5?$AAM?$AAM?$AAM?$AAM?$AA?5?$AAd?$AAd?$AA?0?$AA?5?$AAy?$AAy?$AAy?$AAy?$AA?$AA@ 0000000180013bb0     libucrt:nlsdata.obj
 0002:00001bd8       ??_C@_1BC@GDGBMEMK@?$AAH?$AAH?$AA?3?$AAm?$AAm?$AA?3?$AAs?$AAs?$AA?$AA@ 0000000180013bd8     libucrt:nlsdata.obj
 0002:00001bf0       ??_C@_1M@BMHNFIME@?$AAe?$AAn?$AA?9?$AAU?$AAS?$AA?$AA@ 0000000180013bf0     libucrt:nlsdata.obj
 0002:00001ca0       ??_C@_1EG@CNNIPFIM@?$AAa?$AAp?$AAi?$AA?9?$AAm?$AAs?$AA?9?$AAw?$AAi?$AAn?$AA?9?$AAa?$AAp?$AAp?$AAm?$AAo?$AAd?$AAe?$AAl?$AA?9?$AAr?$AAu?$AAn?$AAt?$AAi?$AAm?$AAe?$AA?9?$AAl?$AA1?$AA?9?$AA1@ 0000000180013ca0     libucrt:winapi_thunks.obj
 0002:00001cf0       ??_C@_1EA@JGEFHKEI@?$AAa?$AAp?$AAi?$AA?9?$AAm?$AAs?$AA?9?$AAw?$AAi?$AAn?$AA?9?$AAc?$AAo?$AAr?$AAe?$AA?9?$AAd?$AAa?$AAt?$AAe?$AAt?$AAi?$AAm?$AAe?$AA?9?$AAl?$AA1?$AA?9?$AA1?$AA?9?$AA1?$AA?$AA@ 0000000180013cf0     libucrt:winapi_thunks.obj
 0002:00001d30       ??_C@_1DI@GCIAAENM@?$AAa?$AAp?$AAi?$AA?9?$AAm?$AAs?$AA?9?$AAw?$AAi?$AAn?$AA?9?$AAc?$AAo?$AAr?$AAe?$AA?9?$AAf?$AAi?$AAl?$AAe?$AA?9?$AAl?$AA2?$AA?9?$AA1?$AA?9?$AA1?$AA?$AA@ 0000000180013d30     libucrt:winapi_thunks.obj
 0002:00001d70       ??_C@_1EI@MPIAOHOC@?$AAa?$AAp?$AAi?$AA?9?$AAm?$AAs?$AA?9?$AAw?$AAi?$AAn?$AA?9?$AAc?$AAo?$AAr?$AAe?$AA?9?$AAl?$AAo?$AAc?$AAa?$AAl?$AAi?$AAz?$AAa?$AAt?$AAi?$AAo?$AAn?$AA?9?$AAl?$AA1?$AA?9@ 0000000180013d70     libucrt:winapi_thunks.obj
 0002:00001dc0       ??_C@_1FK@FPHCKFIE@?$AAa?$AAp?$AAi?$AA?9?$AAm?$AAs?$AA?9?$AAw?$AAi?$AAn?$AA?9?$AAc?$AAo?$AAr?$AAe?$AA?9?$AAl?$AAo?$AAc?$AAa?$AAl?$AAi?$AAz?$AAa?$AAt?$AAi?$AAo?$AAn?$AA?9?$AAo?$AAb?$AAs@ 0000000180013dc0     libucrt:winapi_thunks.obj
 0002:00001e20       ??_C@_1EM@DILCGIIO@?$AAa?$AAp?$AAi?$AA?9?$AAm?$AAs?$AA?9?$AAw?$AAi?$AAn?$AA?9?$AAc?$AAo?$AAr?$AAe?$AA?9?$AAp?$AAr?$AAo?$AAc?$AAe?$AAs?$AAs?$AAt?$AAh?$AAr?$AAe?$AAa?$AAd?$AAs?$AA?9?$AAl@ 0000000180013e20     libucrt:winapi_thunks.obj
 0002:00001e70       ??_C@_1DM@LNCGDDPN@?$AAa?$AAp?$AAi?$AA?9?$AAm?$AAs?$AA?9?$AAw?$AAi?$AAn?$AA?9?$AAc?$AAo?$AAr?$AAe?$AA?9?$AAs?$AAt?$AAr?$AAi?$AAn?$AAg?$AA?9?$AAl?$AA1?$AA?9?$AA1?$AA?9?$AA0?$AA?$AA@ 0000000180013e70     libucrt:winapi_thunks.obj
 0002:00001eb0       ??_C@_1DO@FPAPJEMD@?$AAa?$AAp?$AAi?$AA?9?$AAm?$AAs?$AA?9?$AAw?$AAi?$AAn?$AA?9?$AAc?$AAo?$AAr?$AAe?$AA?9?$AAs?$AAy?$AAs?$AAi?$AAn?$AAf?$AAo?$AA?9?$AAl?$AA1?$AA?9?$AA2?$AA?9?$AA1?$AA?$AA@ 0000000180013eb0     libucrt:winapi_thunks.obj
 0002:00001ef0       ??_C@_1DK@NDHNAHIO@?$AAa?$AAp?$AAi?$AA?9?$AAm?$AAs?$AA?9?$AAw?$AAi?$AAn?$AA?9?$AAc?$AAo?$AAr?$AAe?$AA?9?$AAw?$AAi?$AAn?$AAr?$AAt?$AA?9?$AAl?$AA1?$AA?9?$AA1?$AA?9?$AA0?$AA?$AA@ 0000000180013ef0     libucrt:winapi_thunks.obj
 0002:00001f30       ??_C@_1DM@KGHDGBCM@?$AAa?$AAp?$AAi?$AA?9?$AAm?$AAs?$AA?9?$AAw?$AAi?$AAn?$AA?9?$AAc?$AAo?$AAr?$AAe?$AA?9?$AAx?$AAs?$AAt?$AAa?$AAt?$AAe?$AA?9?$AAl?$AA2?$AA?9?$AA1?$AA?9?$AA0?$AA?$AA@ 0000000180013f30     libucrt:winapi_thunks.obj
 0002:00001f70       ??_C@_1EO@IJIOEFOH@?$AAa?$AAp?$AAi?$AA?9?$AAm?$AAs?$AA?9?$AAw?$AAi?$AAn?$AA?9?$AAr?$AAt?$AAc?$AAo?$AAr?$AAe?$AA?9?$AAn?$AAt?$AAu?$AAs?$AAe?$AAr?$AA?9?$AAw?$AAi?$AAn?$AAd?$AAo?$AAw?$AA?9@ 0000000180013f70     libucrt:winapi_thunks.obj
 0002:00001fc0       ??_C@_1FG@HHGEKANL@?$AAa?$AAp?$AAi?$AA?9?$AAm?$AAs?$AA?9?$AAw?$AAi?$AAn?$AA?9?$AAs?$AAe?$AAc?$AAu?$AAr?$AAi?$AAt?$AAy?$AA?9?$AAs?$AAy?$AAs?$AAt?$AAe?$AAm?$AAf?$AAu?$AAn?$AAc?$AAt?$AAi@ 0000000180013fc0     libucrt:winapi_thunks.obj
 0002:00002020       ??_C@_1FG@NCKKOLKO@?$AAe?$AAx?$AAt?$AA?9?$AAm?$AAs?$AA?9?$AAw?$AAi?$AAn?$AA?9?$AAk?$AAe?$AAr?$AAn?$AAe?$AAl?$AA3?$AA2?$AA?9?$AAp?$AAa?$AAc?$AAk?$AAa?$AAg?$AAe?$AA?9?$AAc?$AAu?$AAr?$AAr@ 0000000180014020     libucrt:winapi_thunks.obj
 0002:00002080       ??_C@_1EG@DBIOJECG@?$AAe?$AAx?$AAt?$AA?9?$AAm?$AAs?$AA?9?$AAw?$AAi?$AAn?$AA?9?$AAn?$AAt?$AAu?$AAs?$AAe?$AAr?$AA?9?$AAd?$AAi?$AAa?$AAl?$AAo?$AAg?$AAb?$AAo?$AAx?$AA?9?$AAl?$AA1?$AA?9?$AA1@ 0000000180014080     libucrt:winapi_thunks.obj
 0002:000020d0       ??_C@_1EO@FIHMJCLF@?$AAe?$AAx?$AAt?$AA?9?$AAm?$AAs?$AA?9?$AAw?$AAi?$AAn?$AA?9?$AAn?$AAt?$AAu?$AAs?$AAe?$AAr?$AA?9?$AAw?$AAi?$AAn?$AAd?$AAo?$AAw?$AAs?$AAt?$AAa?$AAt?$AAi?$AAo?$AAn?$AA?9@ 00000001800140d0     libucrt:winapi_thunks.obj
 0002:00002120       ??_C@_1BC@DNHGCMLG@?$AAa?$AAd?$AAv?$AAa?$AAp?$AAi?$AA3?$AA2?$AA?$AA@ 0000000180014120     libucrt:winapi_thunks.obj
 0002:00002138       ??_C@_1O@BCCLBEOE@?$AAu?$AAs?$AAe?$AAr?$AA3?$AA2?$AA?$AA@ 0000000180014138     libucrt:winapi_thunks.obj
 0002:00002170       ??_C@_0BE@JOGNEJCI@GetCurrentPackageId?$AA@ 0000000180014170     libucrt:winapi_thunks.obj
 0002:00002198       ??_C@_0O@KKBNKAPF@LCMapStringEx?$AA@ 0000000180014198     libucrt:winapi_thunks.obj
 0002:000021b0       ??_C@_0BB@HBDEELFH@LocaleNameToLCID?$AA@ 00000001800141b0     libucrt:winapi_thunks.obj
 0002:000021e8       ??_C@_1M@HPNHIDJI@?$AAj?$AAa?$AA?9?$AAJ?$AAP?$AA?$AA@ 00000001800141e8     libucrt:mbctype.obj
 0002:000021f8       ??_C@_1M@BIBDDEMK@?$AAz?$AAh?$AA?9?$AAC?$AAN?$AA?$AA@ 00000001800141f8     libucrt:mbctype.obj
 0002:00002208       ??_C@_1M@JLOOOEGK@?$AAk?$AAo?$AA?9?$AAK?$AAR?$AA?$AA@ 0000000180014208     libucrt:mbctype.obj
 0002:00002218       ??_C@_1M@CLNBBOPM@?$AAz?$AAh?$AA?9?$AAT?$AAW?$AA?$AA@ 0000000180014218     libucrt:mbctype.obj
 0002:00002230       __newctype                 0000000180014230     libucrt:ctype.obj
 0002:00002530       __newclmap                 0000000180014530     libucrt:ctype.obj
 0002:000026b0       __newcumap                 00000001800146b0     libucrt:ctype.obj
 0002:00002830       ?large_power_data@?1??multiply_by_power_of_ten@__crt_strtox@@YA_NAEAUbig_integer@2@I@Z@4QBIB 0000000180014830     libucrt:cfout.obj
 0002:00003140       ?large_power_indices@?1??multiply_by_power_of_ten@__crt_strtox@@YA_NAEAUbig_integer@2@I@Z@4QBUunpack_index@?1??12@YA_N0I@Z@B 0000000180015140     libucrt:cfout.obj
 0002:000031d8       ?small_powers_of_ten@?6??multiply_by_power_of_ten@__crt_strtox@@YA_NAEAUbig_integer@2@I@Z@4QBIB 00000001800151d8     libucrt:cfout.obj
 0002:000031fc       ??_C@_01GBGANLPD@0?$AA@    00000001800151fc     libucrt:cfout.obj
 0002:00003200       ??_C@_05DNEBIAHO@1?$CDINF?$AA@ 0000000180015200     libucrt:cfout.obj
 0002:00003208       ??_C@_06IMKFLFPG@1?$CDQNAN?$AA@ 0000000180015208     libucrt:cfout.obj
 0002:00003210       ??_C@_06PGGFOGJG@1?$CDSNAN?$AA@ 0000000180015210     libucrt:cfout.obj
 0002:00003218       ??_C@_05PHHOCPM@1?$CDIND?$AA@ 0000000180015218     libucrt:cfout.obj
 0002:00003220       ??_C@_15PJPFLCCM@?$AAu?$AAk?$AA?$AA@ 0000000180015220     libucrt:get_qualified_locale.obj
 0002:00004070       ??_C@_15EMKDOKLE@?$AAa?$AAr?$AA?$AA@ 0000000180016070     libucrt:lcidtoname_downlevel.obj
 0002:00004078       ??_C@_15KNPADPLH@?$AAb?$AAg?$AA?$AA@ 0000000180016078     libucrt:lcidtoname_downlevel.obj
 0002:00004080       ??_C@_15EDMHLDMO@?$AAc?$AAa?$AA?$AA@ 0000000180016080     libucrt:lcidtoname_downlevel.obj
 0002:00004088       ??_C@_1O@BPEAJADD@?$AAz?$AAh?$AA?9?$AAC?$AAH?$AAS?$AA?$AA@ 0000000180016088     libucrt:lcidtoname_downlevel.obj
 0002:00004098       ??_C@_15LJNHCMNK@?$AAc?$AAs?$AA?$AA@ 0000000180016098     libucrt:lcidtoname_downlevel.obj
 0002:000040a0       ??_C@_15FOMCIDHG@?$AAd?$AAa?$AA?$AA@ 00000001800160a0     libucrt:lcidtoname_downlevel.obj
 0002:000040a8       ??_C@_15NBKABECB@?$AAd?$AAe?$AA?$AA@ 00000001800160a8     libucrt:lcidtoname_downlevel.obj
 0002:000040b0       ??_C@_15GHPEIIAO@?$AAe?$AAl?$AA?$AA@ 00000001800160b0     libucrt:lcidtoname_downlevel.obj
 0002:000040b8       ??_C@_15MNPNEAIF@?$AAe?$AAn?$AA?$AA@ 00000001800160b8     libucrt:lcidtoname_downlevel.obj
 0002:000040c0       ??_C@_15GPIOMPMH@?$AAe?$AAs?$AA?$AA@ 00000001800160c0     libucrt:lcidtoname_downlevel.obj
 0002:000040c8       ??_C@_15NGLOAKJC@?$AAf?$AAi?$AA?$AA@ 00000001800160c8     libucrt:lcidtoname_downlevel.obj
 0002:000040d0       ??_C@_15FBKGNKAM@?$AAf?$AAr?$AA?$AA@ 00000001800160d0     libucrt:lcidtoname_downlevel.obj
 0002:000040d8       ??_C@_15KGGCNEFK@?$AAh?$AAe?$AA?$AA@ 00000001800160d8     libucrt:lcidtoname_downlevel.obj
 0002:000040e0       ??_C@_15PGHLIDMF@?$AAh?$AAu?$AA?$AA@ 00000001800160e0     libucrt:lcidtoname_downlevel.obj
 0002:000040e8       ??_C@_15BIEMAPLM@?$AAi?$AAs?$AA?$AA@ 00000001800160e8     libucrt:lcidtoname_downlevel.obj
 0002:000040f0       ??_C@_15IFJLDHAF@?$AAi?$AAt?$AA?$AA@ 00000001800160f0     libucrt:lcidtoname_downlevel.obj
 0002:000040f8       ??_C@_15GEMIOCAG@?$AAj?$AAa?$AA?$AA@ 00000001800160f8     libucrt:lcidtoname_downlevel.obj
 0002:00004100       ??_C@_15EPELEGJA@?$AAk?$AAo?$AA?$AA@ 0000000180016100     libucrt:lcidtoname_downlevel.obj
 0002:00004108       ??_C@_15NDDHIMN@?$AAn?$AAl?$AA?$AA@ 0000000180016108     libucrt:lcidtoname_downlevel.obj
 0002:00004110       ??_C@_15BPIGNHCD@?$AAn?$AAo?$AA?$AA@ 0000000180016110     libucrt:lcidtoname_downlevel.obj
 0002:00004118       ??_C@_15DEOPBLCG@?$AAp?$AAl?$AA?$AA@ 0000000180016118     libucrt:lcidtoname_downlevel.obj
 0002:00004120       ??_C@_15KBECGEFG@?$AAp?$AAt?$AA?$AA@ 0000000180016120     libucrt:lcidtoname_downlevel.obj
 0002:00004128       ??_C@_15GLJCBFMD@?$AAr?$AAo?$AA?$AA@ 0000000180016128     libucrt:lcidtoname_downlevel.obj
 0002:00004130       ??_C@_15FEDGKCDI@?$AAr?$AAu?$AA?$AA@ 0000000180016130     libucrt:lcidtoname_downlevel.obj
 0002:00004138       ??_C@_15GLKMLLHM@?$AAh?$AAr?$AA?$AA@ 0000000180016138     libucrt:lcidtoname_downlevel.obj
 0002:00004140       ??_C@_15CPKMFBDB@?$AAs?$AAk?$AA?$AA@ 0000000180016140     libucrt:lcidtoname_downlevel.obj
 0002:00004148       ??_C@_15BAAIOGMK@?$AAs?$AAq?$AA?$AA@ 0000000180016148     libucrt:lcidtoname_downlevel.obj
 0002:00004150       ??_C@_15INNPNOHD@?$AAs?$AAv?$AA?$AA@ 0000000180016150     libucrt:lcidtoname_downlevel.obj
 0002:00004158       ??_C@_15CABMMOGH@?$AAt?$AAh?$AA?$AA@ 0000000180016158     libucrt:lcidtoname_downlevel.obj
 0002:00004160       ??_C@_15BPLIHJJM@?$AAt?$AAr?$AA?$AA@ 0000000180016160     libucrt:lcidtoname_downlevel.obj
 0002:00004168       ??_C@_15NEOEKKDJ@?$AAu?$AAr?$AA?$AA@ 0000000180016168     libucrt:lcidtoname_downlevel.obj
 0002:00004170       ??_C@_15NFICGAJK@?$AAi?$AAd?$AA?$AA@ 0000000180016170     libucrt:lcidtoname_downlevel.obj
 0002:00004178       ??_C@_15HPJPHDM@?$AAb?$AAe?$AA?$AA@ 0000000180016178     libucrt:lcidtoname_downlevel.obj
 0002:00004180       ??_C@_15LCHLGJII@?$AAs?$AAl?$AA?$AA@ 0000000180016180     libucrt:lcidtoname_downlevel.obj
 0002:00004188       ??_C@_15PCFJPHHO@?$AAe?$AAt?$AA?$AA@ 0000000180016188     libucrt:lcidtoname_downlevel.obj
 0002:00004190       ??_C@_15HPFPGODN@?$AAl?$AAv?$AA?$AA@ 0000000180016190     libucrt:lcidtoname_downlevel.obj
 0002:00004198       ??_C@_15NFFGKGLG@?$AAl?$AAt?$AA?$AA@ 0000000180016198     libucrt:lcidtoname_downlevel.obj
 0002:000041a0       ??_C@_15BDAKCCHN@?$AAf?$AAa?$AA?$AA@ 00000001800161a0     libucrt:lcidtoname_downlevel.obj
 0002:000041a8       ??_C@_15NFGIAIAJ@?$AAv?$AAi?$AA?$AA@ 00000001800161a8     libucrt:lcidtoname_downlevel.obj
 0002:000041b0       ??_C@_15LMKNDMHN@?$AAh?$AAy?$AA?$AA@ 00000001800161b0     libucrt:lcidtoname_downlevel.obj
 0002:000041b8       ??_C@_15IJBHMCFL@?$AAa?$AAz?$AA?$AA@ 00000001800161b8     libucrt:lcidtoname_downlevel.obj
 0002:000041c0       ??_C@_15EKOFJABL@?$AAe?$AAu?$AA?$AA@ 00000001800161c0     libucrt:lcidtoname_downlevel.obj
 0002:000041c8       ??_C@_15BGHADCNK@?$AAm?$AAk?$AA?$AA@ 00000001800161c8     libucrt:lcidtoname_downlevel.obj
 0002:000041d0       ??_C@_15JDNICKHM@?$AAa?$AAf?$AA?$AA@ 00000001800161d0     libucrt:lcidtoname_downlevel.obj
 0002:000041d8       ??_C@_15KPJEDBKD@?$AAk?$AAa?$AA?$AA@ 00000001800161d8     libucrt:lcidtoname_downlevel.obj
 0002:000041e0       ??_C@_15PDNFFFEO@?$AAf?$AAo?$AA?$AA@ 00000001800161e0     libucrt:lcidtoname_downlevel.obj
 0002:000041e8       ??_C@_15OMLEGLOC@?$AAh?$AAi?$AA?$AA@ 00000001800161e8     libucrt:lcidtoname_downlevel.obj
 0002:000041f0       ??_C@_15IDNNENKK@?$AAm?$AAs?$AA?$AA@ 00000001800161f0     libucrt:lcidtoname_downlevel.obj
 0002:000041f8       ??_C@_15MACJNBMH@?$AAk?$AAk?$AA?$AA@ 00000001800161f8     libucrt:lcidtoname_downlevel.obj
 0002:00004200       ??_C@_15DKDJEOND@?$AAk?$AAy?$AA?$AA@ 0000000180016200     libucrt:lcidtoname_downlevel.obj
 0002:00004208       ??_C@_15DFGDLJBG@?$AAs?$AAw?$AA?$AA@ 0000000180016208     libucrt:lcidtoname_downlevel.obj
 0002:00004210       ??_C@_15BBFAICNG@?$AAu?$AAz?$AA?$AA@ 0000000180016210     libucrt:lcidtoname_downlevel.obj
 0002:00004218       ??_C@_15DKNDCGEA@?$AAt?$AAt?$AA?$AA@ 0000000180016218     libucrt:lcidtoname_downlevel.obj
 0002:00004220       ??_C@_15MGIFMDPL@?$AAp?$AAa?$AA?$AA@ 0000000180016220     libucrt:lcidtoname_downlevel.obj
 0002:00004228       ??_C@_15HCNDBBA@?$AAg?$AAu?$AA?$AA@ 0000000180016228     libucrt:lcidtoname_downlevel.obj
 0002:00004230       ??_C@_15FNBEIBON@?$AAt?$AAa?$AA?$AA@ 0000000180016230     libucrt:lcidtoname_downlevel.obj
 0002:00004238       ??_C@_15NCHGBGLK@?$AAt?$AAe?$AA?$AA@ 0000000180016238     libucrt:lcidtoname_downlevel.obj
 0002:00004240       ??_C@_15PHPHCBPF@?$AAk?$AAn?$AA?$AA@ 0000000180016240     libucrt:lcidtoname_downlevel.obj
 0002:00004248       ??_C@_15DLGBCKMP@?$AAm?$AAr?$AA?$AA@ 0000000180016248     libucrt:lcidtoname_downlevel.obj
 0002:00004250       ??_C@_15EABBLBFF@?$AAs?$AAa?$AA?$AA@ 0000000180016250     libucrt:lcidtoname_downlevel.obj
 0002:00004258       ??_C@_15CBKOMCOI@?$AAm?$AAn?$AA?$AA@ 0000000180016258     libucrt:lcidtoname_downlevel.obj
 0002:00004260       ??_C@_15CKDMCJAF@?$AAg?$AAl?$AA?$AA@ 0000000180016260     libucrt:lcidtoname_downlevel.obj
 0002:00004268       ??_C@_17CNJFBPG@?$AAk?$AAo?$AAk?$AA?$AA@ 0000000180016268     libucrt:lcidtoname_downlevel.obj
 0002:00004270       ??_C@_17FFBJICPL@?$AAs?$AAy?$AAr?$AA?$AA@ 0000000180016270     libucrt:lcidtoname_downlevel.obj
 0002:00004278       ??_C@_17KPNDCPAF@?$AAd?$AAi?$AAv?$AA?$AA@ 0000000180016278     libucrt:lcidtoname_downlevel.obj
 0002:00004280       ??_C@_11LOCGONAA@?$AA?$AA@ 0000000180016280     libucrt:lcidtoname_downlevel.obj
 0002:00004288       ??_C@_1M@OKAHONE@?$AAa?$AAr?$AA?9?$AAS?$AAA?$AA?$AA@ 0000000180016288     libucrt:lcidtoname_downlevel.obj
 0002:00004298       ??_C@_1M@FFFIGIGK@?$AAb?$AAg?$AA?9?$AAB?$AAG?$AA?$AA@ 0000000180016298     libucrt:lcidtoname_downlevel.obj
 0002:000042a8       ??_C@_1M@BJNKEDC@?$AAc?$AAa?$AA?9?$AAE?$AAS?$AA?$AA@ 00000001800162a8     libucrt:lcidtoname_downlevel.obj
 0002:000042b8       ??_C@_1M@IJJHFJHA@?$AAc?$AAs?$AA?9?$AAC?$AAZ?$AA?$AA@ 00000001800162b8     libucrt:lcidtoname_downlevel.obj
 0002:000042c8       ??_C@_1M@CLPEOBGI@?$AAd?$AAa?$AA?9?$AAD?$AAK?$AA?$AA@ 00000001800162c8     libucrt:lcidtoname_downlevel.obj
 0002:000042d8       ??_C@_1M@MCMADGCB@?$AAd?$AAe?$AA?9?$AAD?$AAE?$AA?$AA@ 00000001800162d8     libucrt:lcidtoname_downlevel.obj
 0002:000042e8       ??_C@_1M@OOCKEMAM@?$AAe?$AAl?$AA?9?$AAG?$AAR?$AA?$AA@ 00000001800162e8     libucrt:lcidtoname_downlevel.obj
 0002:000042f8       ??_C@_1M@DDNJFGID@?$AAf?$AAi?$AA?9?$AAF?$AAI?$AA?$AA@ 00000001800162f8     libucrt:lcidtoname_downlevel.obj
 0002:00004308       ??_C@_1M@GLIPPMAC@?$AAf?$AAr?$AA?9?$AAF?$AAR?$AA?$AA@ 0000000180016308     libucrt:lcidtoname_downlevel.obj
 0002:00004318       ??_C@_1M@GFMCHPE@?$AAh?$AAe?$AA?9?$AAI?$AAL?$AA?$AA@ 0000000180016318     libucrt:lcidtoname_downlevel.obj
 0002:00004328       ??_C@_1M@MHLPGNKM@?$AAh?$AAu?$AA?9?$AAH?$AAU?$AA?$AA@ 0000000180016328     libucrt:lcidtoname_downlevel.obj
 0002:00004338       ??_C@_1M@LPDDNNPN@?$AAi?$AAs?$AA?9?$AAI?$AAS?$AA?$AA@ 0000000180016338     libucrt:lcidtoname_downlevel.obj
 0002:00004348       ??_C@_1M@MADIPODN@?$AAi?$AAt?$AA?9?$AAI?$AAT?$AA?$AA@ 0000000180016348     libucrt:lcidtoname_downlevel.obj
 0002:00004358       ??_C@_1M@IHBJJGG@?$AAn?$AAl?$AA?9?$AAN?$AAL?$AA?$AA@ 0000000180016358     libucrt:lcidtoname_downlevel.obj
 0002:00004368       ??_C@_1M@EANAGDL@?$AAn?$AAb?$AA?9?$AAN?$AAO?$AA?$AA@ 0000000180016368     libucrt:lcidtoname_downlevel.obj
 0002:00004378       ??_C@_1M@NEIEMEGP@?$AAp?$AAl?$AA?9?$AAP?$AAL?$AA?$AA@ 0000000180016378     libucrt:lcidtoname_downlevel.obj
 0002:00004388       ??_C@_1M@BOCFIGEP@?$AAp?$AAt?$AA?9?$AAB?$AAR?$AA?$AA@ 0000000180016388     libucrt:lcidtoname_downlevel.obj
 0002:00004398       ??_C@_1M@IMPFOPBG@?$AAr?$AAo?$AA?9?$AAR?$AAO?$AA?$AA@ 0000000180016398     libucrt:lcidtoname_downlevel.obj
 0002:000043a8       ??_C@_1M@IDNNEJMM@?$AAr?$AAu?$AA?9?$AAR?$AAU?$AA?$AA@ 00000001800163a8     libucrt:lcidtoname_downlevel.obj
 0002:000043b8       ??_C@_1M@LILEEOGM@?$AAh?$AAr?$AA?9?$AAH?$AAR?$AA?$AA@ 00000001800163b8     libucrt:lcidtoname_downlevel.obj
 0002:000043c8       ??_C@_1M@FKIFEHPB@?$AAs?$AAk?$AA?9?$AAS?$AAK?$AA?$AA@ 00000001800163c8     libucrt:lcidtoname_downlevel.obj
 0002:000043d8       ??_C@_1M@LJMAMNPJ@?$AAs?$AAq?$AA?9?$AAA?$AAL?$AA?$AA@ 00000001800163d8     libucrt:lcidtoname_downlevel.obj
 0002:000043e8       ??_C@_1M@GIAKDKJK@?$AAs?$AAv?$AA?9?$AAS?$AAE?$AA?$AA@ 00000001800163e8     libucrt:lcidtoname_downlevel.obj
 0002:000043f8       ??_C@_1M@MKJKIKCL@?$AAt?$AAh?$AA?9?$AAT?$AAH?$AA?$AA@ 00000001800163f8     libucrt:lcidtoname_downlevel.obj
 0002:00004408       ??_C@_1M@MFLCCMPB@?$AAt?$AAr?$AA?9?$AAT?$AAR?$AA?$AA@ 0000000180016408     libucrt:lcidtoname_downlevel.obj
 0002:00004418       ??_C@_1M@OIJHDKJN@?$AAu?$AAr?$AA?9?$AAP?$AAK?$AA?$AA@ 0000000180016418     libucrt:lcidtoname_downlevel.obj
 0002:00004428       ??_C@_1M@LHIPCIEK@?$AAi?$AAd?$AA?9?$AAI?$AAD?$AA?$AA@ 0000000180016428     libucrt:lcidtoname_downlevel.obj
 0002:00004438       ??_C@_1M@MFMOBGI@?$AAu?$AAk?$AA?9?$AAU?$AAA?$AA?$AA@ 0000000180016438     libucrt:lcidtoname_downlevel.obj
 0002:00004448       ??_C@_1M@OBGLJIPL@?$AAb?$AAe?$AA?9?$AAB?$AAY?$AA?$AA@ 0000000180016448     libucrt:lcidtoname_downlevel.obj
 0002:00004458       ??_C@_1M@BCFAJEAD@?$AAs?$AAl?$AA?9?$AAS?$AAI?$AA?$AA@ 0000000180016458     libucrt:lcidtoname_downlevel.obj
 0002:00004468       ??_C@_1M@FKFFEDDN@?$AAe?$AAt?$AA?9?$AAE?$AAE?$AA?$AA@ 0000000180016468     libucrt:lcidtoname_downlevel.obj
 0002:00004478       ??_C@_1M@KGKKAACI@?$AAl?$AAv?$AA?9?$AAL?$AAV?$AA?$AA@ 0000000180016478     libucrt:lcidtoname_downlevel.obj
 0002:00004488       ??_C@_1M@IFGBIJO@?$AAl?$AAt?$AA?9?$AAL?$AAT?$AA?$AA@ 0000000180016488     libucrt:lcidtoname_downlevel.obj
 0002:00004498       ??_C@_1M@FGEAHEDM@?$AAf?$AAa?$AA?9?$AAI?$AAR?$AA?$AA@ 0000000180016498     libucrt:lcidtoname_downlevel.obj
 0002:000044a8       ??_C@_1M@KBMAIBFN@?$AAv?$AAi?$AA?9?$AAV?$AAN?$AA?$AA@ 00000001800164a8     libucrt:lcidtoname_downlevel.obj
 0002:000044b8       ??_C@_1M@GPCBKDJK@?$AAh?$AAy?$AA?9?$AAA?$AAM?$AA?$AA@ 00000001800164b8     libucrt:lcidtoname_downlevel.obj
 0002:000044c8       ??_C@_1BG@BECMDDJB@?$AAa?$AAz?$AA?9?$AAA?$AAZ?$AA?9?$AAL?$AAa?$AAt?$AAn?$AA?$AA@ 00000001800164c8     libucrt:lcidtoname_downlevel.obj
 0002:000044e0       ??_C@_1M@MAOFCAEA@?$AAe?$AAu?$AA?9?$AAE?$AAS?$AA?$AA@ 00000001800164e0     libucrt:lcidtoname_downlevel.obj
 0002:000044f0       ??_C@_1M@IGHABKPI@?$AAm?$AAk?$AA?9?$AAM?$AAK?$AA?$AA@ 00000001800164f0     libucrt:lcidtoname_downlevel.obj
 0002:00004500       ??_C@_1M@IAIGNEJG@?$AAt?$AAn?$AA?9?$AAZ?$AAA?$AA?$AA@ 0000000180016500     libucrt:lcidtoname_downlevel.obj
 0002:00004510       ??_C@_1M@IIJCOJFA@?$AAx?$AAh?$AA?9?$AAZ?$AAA?$AA?$AA@ 0000000180016510     libucrt:lcidtoname_downlevel.obj
 0002:00004520       ??_C@_1M@LGPJHNJH@?$AAz?$AAu?$AA?9?$AAZ?$AAA?$AA?$AA@ 0000000180016520     libucrt:lcidtoname_downlevel.obj
 0002:00004530       ??_C@_1M@HOKAOIO@?$AAa?$AAf?$AA?9?$AAZ?$AAA?$AA?$AA@ 0000000180016530     libucrt:lcidtoname_downlevel.obj
 0002:00004540       ??_C@_1M@DPCLHLIE@?$AAk?$AAa?$AA?9?$AAG?$AAE?$AA?$AA@ 0000000180016540     libucrt:lcidtoname_downlevel.obj
 0002:00004550       ??_C@_1M@BLKMHJBI@?$AAf?$AAo?$AA?9?$AAF?$AAO?$AA?$AA@ 0000000180016550     libucrt:lcidtoname_downlevel.obj
 0002:00004560       ??_C@_1M@LGGJAPPB@?$AAh?$AAi?$AA?9?$AAI?$AAN?$AA?$AA@ 0000000180016560     libucrt:lcidtoname_downlevel.obj
 0002:00004570       ??_C@_1M@FIKPIHFE@?$AAm?$AAt?$AA?9?$AAM?$AAT?$AA?$AA@ 0000000180016570     libucrt:lcidtoname_downlevel.obj
 0002:00004580       ??_C@_1M@HEGGPBFA@?$AAs?$AAe?$AA?9?$AAN?$AAO?$AA?$AA@ 0000000180016580     libucrt:lcidtoname_downlevel.obj
 0002:00004590       ??_C@_1M@EIBJEEPA@?$AAm?$AAs?$AA?9?$AAM?$AAY?$AA?$AA@ 0000000180016590     libucrt:lcidtoname_downlevel.obj
 0002:000045a0       ??_C@_1M@FHLBGMPP@?$AAk?$AAk?$AA?9?$AAK?$AAZ?$AA?$AA@ 00000001800165a0     libucrt:lcidtoname_downlevel.obj
 0002:000045b0       ??_C@_1M@NGJJLCGI@?$AAk?$AAy?$AA?9?$AAK?$AAG?$AA?$AA@ 00000001800165b0     libucrt:lcidtoname_downlevel.obj
 0002:000045c0       ??_C@_1M@GIENNBFC@?$AAs?$AAw?$AA?9?$AAK?$AAE?$AA?$AA@ 00000001800165c0     libucrt:lcidtoname_downlevel.obj
 0002:000045d0       ??_C@_1BG@NDGMJIMJ@?$AAu?$AAz?$AA?9?$AAU?$AAZ?$AA?9?$AAL?$AAa?$AAt?$AAn?$AA?$AA@ 00000001800165d0     libucrt:lcidtoname_downlevel.obj
 0002:000045e8       ??_C@_1M@IDCCIHBC@?$AAt?$AAt?$AA?9?$AAR?$AAU?$AA?$AA@ 00000001800165e8     libucrt:lcidtoname_downlevel.obj
 0002:000045f8       ??_C@_1M@LOICPMOJ@?$AAb?$AAn?$AA?9?$AAI?$AAN?$AA?$AA@ 00000001800165f8     libucrt:lcidtoname_downlevel.obj
 0002:00004608       ??_C@_1M@KPKKNEAH@?$AAp?$AAa?$AA?9?$AAI?$AAN?$AA?$AA@ 0000000180016608     libucrt:lcidtoname_downlevel.obj
 0002:00004618       ??_C@_1M@PJGPPBOG@?$AAg?$AAu?$AA?9?$AAI?$AAN?$AA?$AA@ 0000000180016618     libucrt:lcidtoname_downlevel.obj
 0002:00004628       ??_C@_1M@KMKMOPHI@?$AAt?$AAa?$AA?9?$AAI?$AAN?$AA?$AA@ 0000000180016628     libucrt:lcidtoname_downlevel.obj
 0002:00004638       ??_C@_1M@KFEHEPAC@?$AAt?$AAe?$AA?9?$AAI?$AAN?$AA?$AA@ 0000000180016638     libucrt:lcidtoname_downlevel.obj
 0002:00004648       ??_C@_1M@CDCLMGHI@?$AAk?$AAn?$AA?9?$AAI?$AAN?$AA?$AA@ 0000000180016648     libucrt:lcidtoname_downlevel.obj
 0002:00004658       ??_C@_1M@MIODLDKF@?$AAm?$AAl?$AA?9?$AAI?$AAN?$AA?$AA@ 0000000180016658     libucrt:lcidtoname_downlevel.obj
 0002:00004668       ??_C@_1M@PBIEACPO@?$AAm?$AAr?$AA?9?$AAI?$AAN?$AA?$AA@ 0000000180016668     libucrt:lcidtoname_downlevel.obj
 0002:00004678       ??_C@_1M@NIDEAGPH@?$AAs?$AAa?$AA?9?$AAI?$AAN?$AA?$AA@ 0000000180016678     libucrt:lcidtoname_downlevel.obj
 0002:00004688       ??_C@_1M@FHIHCBIO@?$AAm?$AAn?$AA?9?$AAM?$AAN?$AA?$AA@ 0000000180016688     libucrt:lcidtoname_downlevel.obj
 0002:00004698       ??_C@_1M@JAIJPENP@?$AAc?$AAy?$AA?9?$AAG?$AAB?$AA?$AA@ 0000000180016698     libucrt:lcidtoname_downlevel.obj
 0002:000046a8       ??_C@_1M@PHGFBEPN@?$AAg?$AAl?$AA?9?$AAE?$AAS?$AA?$AA@ 00000001800166a8     libucrt:lcidtoname_downlevel.obj
 0002:000046b8       ??_C@_1O@KPIPDNCP@?$AAk?$AAo?$AAk?$AA?9?$AAI?$AAN?$AA?$AA@ 00000001800166b8     libucrt:lcidtoname_downlevel.obj
 0002:000046c8       ??_C@_1O@KNHJLDJA@?$AAs?$AAy?$AAr?$AA?9?$AAS?$AAY?$AA?$AA@ 00000001800166c8     libucrt:lcidtoname_downlevel.obj
 0002:000046d8       ??_C@_1O@MKEKBLAH@?$AAd?$AAi?$AAv?$AA?9?$AAM?$AAV?$AA?$AA@ 00000001800166d8     libucrt:lcidtoname_downlevel.obj
 0002:000046e8       ??_C@_1O@OHDCKDDF@?$AAq?$AAu?$AAz?$AA?9?$AAB?$AAO?$AA?$AA@ 00000001800166e8     libucrt:lcidtoname_downlevel.obj
 0002:000046f8       ??_C@_1M@LEPJNLFD@?$AAn?$AAs?$AA?9?$AAZ?$AAA?$AA?$AA@ 00000001800166f8     libucrt:lcidtoname_downlevel.obj
 0002:00004708       ??_C@_1M@OMLEIIJB@?$AAm?$AAi?$AA?9?$AAN?$AAZ?$AA?$AA@ 0000000180016708     libucrt:lcidtoname_downlevel.obj
 0002:00004718       ??_C@_1M@PMPEAILG@?$AAa?$AAr?$AA?9?$AAI?$AAQ?$AA?$AA@ 0000000180016718     libucrt:lcidtoname_downlevel.obj
 0002:00004728       ??_C@_1M@CNKPNOEE@?$AAd?$AAe?$AA?9?$AAC?$AAH?$AA?$AA@ 0000000180016728     libucrt:lcidtoname_downlevel.obj
 0002:00004738       ??_C@_1M@LKMGMLKO@?$AAe?$AAn?$AA?9?$AAG?$AAB?$AA?$AA@ 0000000180016738     libucrt:lcidtoname_downlevel.obj
 0002:00004748       ??_C@_1M@PGKJFFGL@?$AAe?$AAs?$AA?9?$AAM?$AAX?$AA?$AA@ 0000000180016748     libucrt:lcidtoname_downlevel.obj
 0002:00004758       ??_C@_1M@DNNANBDC@?$AAf?$AAr?$AA?9?$AAB?$AAE?$AA?$AA@ 0000000180016758     libucrt:lcidtoname_downlevel.obj
 0002:00004768       ??_C@_1M@HLGMDFHM@?$AAi?$AAt?$AA?9?$AAC?$AAH?$AA?$AA@ 0000000180016768     libucrt:lcidtoname_downlevel.obj
 0002:00004778       ??_C@_1M@CLLBGJH@?$AAn?$AAl?$AA?9?$AAB?$AAE?$AA?$AA@ 0000000180016778     libucrt:lcidtoname_downlevel.obj
 0002:00004788       ??_C@_1M@BODBOGLF@?$AAn?$AAn?$AA?9?$AAN?$AAO?$AA?$AA@ 0000000180016788     libucrt:lcidtoname_downlevel.obj
 0002:00004798       ??_C@_1M@HFFAHKAD@?$AAp?$AAt?$AA?9?$AAP?$AAT?$AA?$AA@ 0000000180016798     libucrt:lcidtoname_downlevel.obj
 0002:000047a8       ??_C@_1BG@LNOAKHIE@?$AAs?$AAr?$AA?9?$AAS?$AAP?$AA?9?$AAL?$AAa?$AAt?$AAn?$AA?$AA@ 00000001800167a8     libucrt:lcidtoname_downlevel.obj
 0002:000047c0       ??_C@_1M@HBMHBGAK@?$AAs?$AAv?$AA?9?$AAF?$AAI?$AA?$AA@ 00000001800167c0     libucrt:lcidtoname_downlevel.obj
 0002:000047d0       ??_C@_1BG@DGCJGJBE@?$AAa?$AAz?$AA?9?$AAA?$AAZ?$AA?9?$AAC?$AAy?$AAr?$AAl?$AA?$AA@ 00000001800167d0     libucrt:lcidtoname_downlevel.obj
 0002:000047e8       ??_C@_1M@KEJDAAHB@?$AAs?$AAe?$AA?9?$AAS?$AAE?$AA?$AA@ 00000001800167e8     libucrt:lcidtoname_downlevel.obj
 0002:000047f8       ??_C@_1M@HEIBJJAD@?$AAm?$AAs?$AA?9?$AAB?$AAN?$AA?$AA@ 00000001800167f8     libucrt:lcidtoname_downlevel.obj
 0002:00004808       ??_C@_1BG@PBGJMCEM@?$AAu?$AAz?$AA?9?$AAU?$AAZ?$AA?9?$AAC?$AAy?$AAr?$AAl?$AA?$AA@ 0000000180016808     libucrt:lcidtoname_downlevel.obj
 0002:00004820       ??_C@_1O@LAOBCMDF@?$AAq?$AAu?$AAz?$AA?9?$AAE?$AAC?$AA?$AA@ 0000000180016820     libucrt:lcidtoname_downlevel.obj
 0002:00004830       ??_C@_1M@POEEMAIO@?$AAa?$AAr?$AA?9?$AAE?$AAG?$AA?$AA@ 0000000180016830     libucrt:lcidtoname_downlevel.obj
 0002:00004840       ??_C@_1M@EFAKDEDL@?$AAz?$AAh?$AA?9?$AAH?$AAK?$AA?$AA@ 0000000180016840     libucrt:lcidtoname_downlevel.obj
 0002:00004850       ??_C@_1M@HKKIJHGI@?$AAd?$AAe?$AA?9?$AAA?$AAT?$AA?$AA@ 0000000180016850     libucrt:lcidtoname_downlevel.obj
 0002:00004860       ??_C@_1M@KBFBEHJF@?$AAe?$AAn?$AA?9?$AAA?$AAU?$AA?$AA@ 0000000180016860     libucrt:lcidtoname_downlevel.obj
 0002:00004870       ??_C@_1M@MNPLFAAH@?$AAe?$AAs?$AA?9?$AAE?$AAS?$AA?$AA@ 0000000180016870     libucrt:lcidtoname_downlevel.obj
 0002:00004880       ??_C@_1M@HJOOJFMA@?$AAf?$AAr?$AA?9?$AAC?$AAA?$AA?$AA@ 0000000180016880     libucrt:lcidtoname_downlevel.obj
 0002:00004890       ??_C@_1BG@JPOFPNAB@?$AAs?$AAr?$AA?9?$AAS?$AAP?$AA?9?$AAC?$AAy?$AAr?$AAl?$AA?$AA@ 0000000180016890     libucrt:lcidtoname_downlevel.obj
 0002:000048a8       ??_C@_1M@LNFOCMOB@?$AAs?$AAe?$AA?9?$AAF?$AAI?$AA?$AA@ 00000001800168a8     libucrt:lcidtoname_downlevel.obj
 0002:000048b8       ??_C@_1O@MGJBOAMB@?$AAq?$AAu?$AAz?$AA?9?$AAP?$AAE?$AA?$AA@ 00000001800168b8     libucrt:lcidtoname_downlevel.obj
 0002:000048c8       ??_C@_1M@GJINLBOK@?$AAa?$AAr?$AA?9?$AAL?$AAY?$AA?$AA@ 00000001800168c8     libucrt:lcidtoname_downlevel.obj
 0002:000048d8       ??_C@_1M@GGMNHJNL@?$AAz?$AAh?$AA?9?$AAS?$AAG?$AA?$AA@ 00000001800168d8     libucrt:lcidtoname_downlevel.obj
 0002:000048e8       ??_C@_1M@HOIKODND@?$AAd?$AAe?$AA?9?$AAL?$AAU?$AA?$AA@ 00000001800168e8     libucrt:lcidtoname_downlevel.obj
 0002:000048f8       ??_C@_1M@DDOCCGFG@?$AAe?$AAn?$AA?9?$AAC?$AAA?$AA?$AA@ 00000001800168f8     libucrt:lcidtoname_downlevel.obj
 0002:00004908       ??_C@_1M@BNOEMJLF@?$AAe?$AAs?$AA?9?$AAG?$AAT?$AA?$AA@ 0000000180016908     libucrt:lcidtoname_downlevel.obj
 0002:00004918       ??_C@_1M@EOGNKEK@?$AAf?$AAr?$AA?9?$AAC?$AAH?$AA?$AA@ 0000000180016918     libucrt:lcidtoname_downlevel.obj
 0002:00004928       ??_C@_1M@FLIDJFHL@?$AAh?$AAr?$AA?9?$AAB?$AAA?$AA?$AA@ 0000000180016928     libucrt:lcidtoname_downlevel.obj
 0002:00004938       ??_C@_1O@FMCELNAJ@?$AAs?$AAm?$AAj?$AA?9?$AAN?$AAO?$AA?$AA@ 0000000180016938     libucrt:lcidtoname_downlevel.obj
 0002:00004948       ??_C@_1M@JHGLJMGJ@?$AAa?$AAr?$AA?9?$AAD?$AAZ?$AA?$AA@ 0000000180016948     libucrt:lcidtoname_downlevel.obj
 0002:00004958       ??_C@_1M@JKKFDCNP@?$AAz?$AAh?$AA?9?$AAM?$AAO?$AA?$AA@ 0000000180016958     libucrt:lcidtoname_downlevel.obj
 0002:00004968       ??_C@_1M@GEEFALPE@?$AAd?$AAe?$AA?9?$AAL?$AAI?$AA?$AA@ 0000000180016968     libucrt:lcidtoname_downlevel.obj
 0002:00004978       ??_C@_1M@IGEOFBG@?$AAe?$AAn?$AA?9?$AAN?$AAZ?$AA?$AA@ 0000000180016978     libucrt:lcidtoname_downlevel.obj
 0002:00004988       ??_C@_1M@KDBONEHP@?$AAe?$AAs?$AA?9?$AAC?$AAR?$AA?$AA@ 0000000180016988     libucrt:lcidtoname_downlevel.obj
 0002:00004998       ??_C@_1M@FHMDOHNN@?$AAf?$AAr?$AA?9?$AAL?$AAU?$AA?$AA@ 0000000180016998     libucrt:lcidtoname_downlevel.obj
 0002:000049a8       ??_C@_1BG@NFKKMAFG@?$AAb?$AAs?$AA?9?$AAB?$AAA?$AA?9?$AAL?$AAa?$AAt?$AAn?$AA?$AA@ 00000001800169a8     libucrt:lcidtoname_downlevel.obj
 0002:000049c0       ??_C@_1O@IMNBEMCI@?$AAs?$AAm?$AAj?$AA?9?$AAS?$AAE?$AA?$AA@ 00000001800169c0     libucrt:lcidtoname_downlevel.obj
 0002:000049d0       ??_C@_1M@DHHMBNDP@?$AAa?$AAr?$AA?9?$AAM?$AAA?$AA?$AA@ 00000001800169d0     libucrt:lcidtoname_downlevel.obj
 0002:000049e0       ??_C@_1M@BNBLJCGH@?$AAe?$AAn?$AA?9?$AAI?$AAE?$AA?$AA@ 00000001800169e0     libucrt:lcidtoname_downlevel.obj
 0002:000049f0       ??_C@_1M@GEPAFMDL@?$AAe?$AAs?$AA?9?$AAP?$AAA?$AA?$AA@ 00000001800169f0     libucrt:lcidtoname_downlevel.obj
 0002:00004a00       ??_C@_1M@OJONDMDL@?$AAf?$AAr?$AA?9?$AAM?$AAC?$AA?$AA@ 0000000180016a00     libucrt:lcidtoname_downlevel.obj
 0002:00004a10       ??_C@_1BG@OBCNFJB@?$AAs?$AAr?$AA?9?$AAB?$AAA?$AA?9?$AAL?$AAa?$AAt?$AAn?$AA?$AA@ 0000000180016a10     libucrt:lcidtoname_downlevel.obj
 0002:00004a28       ??_C@_1O@KEMEEGPO@?$AAs?$AAm?$AAa?$AA?9?$AAN?$AAO?$AA?$AA@ 0000000180016a28     libucrt:lcidtoname_downlevel.obj
 0002:00004a38       ??_C@_1M@ELMGFODK@?$AAa?$AAr?$AA?9?$AAT?$AAN?$AA?$AA@ 0000000180016a38     libucrt:lcidtoname_downlevel.obj
 0002:00004a48       ??_C@_1M@BHDLHFAF@?$AAe?$AAn?$AA?9?$AAZ?$AAA?$AA?$AA@ 0000000180016a48     libucrt:lcidtoname_downlevel.obj
 0002:00004a58       ??_C@_1M@BMGIGLIF@?$AAe?$AAs?$AA?9?$AAD?$AAO?$AA?$AA@ 0000000180016a58     libucrt:lcidtoname_downlevel.obj
 0002:00004a68       ??_C@_1BG@CMBHIPBE@?$AAs?$AAr?$AA?9?$AAB?$AAA?$AA?9?$AAC?$AAy?$AAr?$AAl?$AA?$AA@ 0000000180016a68     libucrt:lcidtoname_downlevel.obj
 0002:00004a80       ??_C@_1O@HEDBLHNP@?$AAs?$AAm?$AAa?$AA?9?$AAS?$AAE?$AA?$AA@ 0000000180016a80     libucrt:lcidtoname_downlevel.obj
 0002:00004a90       ??_C@_1M@DAGCADIM@?$AAa?$AAr?$AA?9?$AAO?$AAM?$AA?$AA@ 0000000180016a90     libucrt:lcidtoname_downlevel.obj
 0002:00004aa0       ??_C@_1M@FODLMICG@?$AAe?$AAn?$AA?9?$AAJ?$AAM?$AA?$AA@ 0000000180016aa0     libucrt:lcidtoname_downlevel.obj
 0002:00004ab0       ??_C@_1M@DNMLCIHB@?$AAe?$AAs?$AA?9?$AAV?$AAE?$AA?$AA@ 0000000180016ab0     libucrt:lcidtoname_downlevel.obj
 0002:00004ac0       ??_C@_1O@EOKHMKJK@?$AAs?$AAm?$AAs?$AA?9?$AAF?$AAI?$AA?$AA@ 0000000180016ac0     libucrt:lcidtoname_downlevel.obj
 0002:00004ad0       ??_C@_1M@CAFJMKOF@?$AAa?$AAr?$AA?9?$AAY?$AAE?$AA?$AA@ 0000000180016ad0     libucrt:lcidtoname_downlevel.obj
 0002:00004ae0       ??_C@_1M@CBFHIJLI@?$AAe?$AAn?$AA?9?$AAC?$AAB?$AA?$AA@ 0000000180016ae0     libucrt:lcidtoname_downlevel.obj
 0002:00004af0       ??_C@_1M@BGNFLDN@?$AAe?$AAs?$AA?9?$AAC?$AAO?$AA?$AA@ 0000000180016af0     libucrt:lcidtoname_downlevel.obj
 0002:00004b00       ??_C@_1O@JMPHMAMC@?$AAs?$AAm?$AAn?$AA?9?$AAF?$AAI?$AA?$AA@ 0000000180016b00     libucrt:lcidtoname_downlevel.obj
 0002:00004b10       ??_C@_1M@JLANABKE@?$AAa?$AAr?$AA?9?$AAS?$AAY?$AA?$AA@ 0000000180016b10     libucrt:lcidtoname_downlevel.obj
 0002:00004b20       ??_C@_1M@HPKGCFGN@?$AAe?$AAn?$AA?9?$AAB?$AAZ?$AA?$AA@ 0000000180016b20     libucrt:lcidtoname_downlevel.obj
 0002:00004b30       ??_C@_1M@OLJCMLGM@?$AAe?$AAs?$AA?9?$AAP?$AAE?$AA?$AA@ 0000000180016b30     libucrt:lcidtoname_downlevel.obj
 0002:00004b40       ??_C@_1M@MKKGFKLE@?$AAa?$AAr?$AA?9?$AAJ?$AAO?$AA?$AA@ 0000000180016b40     libucrt:lcidtoname_downlevel.obj
 0002:00004b50       ??_C@_1M@EKPGLDNI@?$AAe?$AAn?$AA?9?$AAT?$AAT?$AA?$AA@ 0000000180016b50     libucrt:lcidtoname_downlevel.obj
 0002:00004b60       ??_C@_1M@OONGHFHE@?$AAe?$AAs?$AA?9?$AAA?$AAR?$AA?$AA@ 0000000180016b60     libucrt:lcidtoname_downlevel.obj
 0002:00004b70       ??_C@_1M@OOJFGBHE@?$AAa?$AAr?$AA?9?$AAL?$AAB?$AA?$AA@ 0000000180016b70     libucrt:lcidtoname_downlevel.obj
 0002:00004b80       ??_C@_1M@GCEJHNEG@?$AAe?$AAn?$AA?9?$AAZ?$AAW?$AA?$AA@ 0000000180016b80     libucrt:lcidtoname_downlevel.obj
 0002:00004b90       ??_C@_1M@JNOCAHJI@?$AAe?$AAs?$AA?9?$AAE?$AAC?$AA?$AA@ 0000000180016b90     libucrt:lcidtoname_downlevel.obj
 0002:00004ba0       ??_C@_1M@JEFHPGGB@?$AAa?$AAr?$AA?9?$AAK?$AAW?$AA?$AA@ 0000000180016ba0     libucrt:lcidtoname_downlevel.obj
 0002:00004bb0       ??_C@_1M@MLKIBJOJ@?$AAe?$AAn?$AA?9?$AAP?$AAH?$AA?$AA@ 0000000180016bb0     libucrt:lcidtoname_downlevel.obj
 0002:00004bc0       ??_C@_1M@BDNIPEND@?$AAe?$AAs?$AA?9?$AAC?$AAL?$AA?$AA@ 0000000180016bc0     libucrt:lcidtoname_downlevel.obj
 0002:00004bd0       ??_C@_1M@MPNMEKBD@?$AAa?$AAr?$AA?9?$AAA?$AAE?$AA?$AA@ 0000000180016bd0     libucrt:lcidtoname_downlevel.obj
 0002:00004be0       ??_C@_1M@KBJALCPI@?$AAe?$AAs?$AA?9?$AAU?$AAY?$AA?$AA@ 0000000180016be0     libucrt:lcidtoname_downlevel.obj
 0002:00004bf0       ??_C@_1M@LLCCOAGA@?$AAa?$AAr?$AA?9?$AAB?$AAH?$AA?$AA@ 0000000180016bf0     libucrt:lcidtoname_downlevel.obj
 0002:00004c00       ??_C@_1M@PBFNCDEL@?$AAe?$AAs?$AA?9?$AAP?$AAY?$AA?$AA@ 0000000180016c00     libucrt:lcidtoname_downlevel.obj
 0002:00004c10       ??_C@_1M@EDGINPNP@?$AAa?$AAr?$AA?9?$AAQ?$AAA?$AA?$AA@ 0000000180016c10     libucrt:lcidtoname_downlevel.obj
 0002:00004c20       ??_C@_1M@MKDBIIJI@?$AAe?$AAs?$AA?9?$AAB?$AAO?$AA?$AA@ 0000000180016c20     libucrt:lcidtoname_downlevel.obj
 0002:00004c30       ??_C@_1M@CPKKEBLD@?$AAe?$AAs?$AA?9?$AAS?$AAV?$AA?$AA@ 0000000180016c30     libucrt:lcidtoname_downlevel.obj
 0002:00004c40       ??_C@_1M@NDBGMMJL@?$AAe?$AAs?$AA?9?$AAH?$AAN?$AA?$AA@ 0000000180016c40     libucrt:lcidtoname_downlevel.obj
 0002:00004c50       ??_C@_1M@JIJIBHDP@?$AAe?$AAs?$AA?9?$AAN?$AAI?$AA?$AA@ 0000000180016c50     libucrt:lcidtoname_downlevel.obj
 0002:00004c60       ??_C@_1M@CGFMKEEK@?$AAe?$AAs?$AA?9?$AAP?$AAR?$AA?$AA@ 0000000180016c60     libucrt:lcidtoname_downlevel.obj
 0002:00004c70       ??_C@_1O@ICJHKIIK@?$AAz?$AAh?$AA?9?$AAC?$AAH?$AAT?$AA?$AA@ 0000000180016c70     libucrt:lcidtoname_downlevel.obj
 0002:00004c80       ??_C@_15CLNEJCE@?$AAs?$AAr?$AA?$AA@ 0000000180016c80     libucrt:lcidtoname_downlevel.obj
 0002:00005ad0       ??_C@_1M@KAHEKEIG@?$AAa?$AAf?$AA?9?$AAz?$AAa?$AA?$AA@ 0000000180017ad0     libucrt:lcidtoname_downlevel.obj
 0002:00005ae0       ??_C@_1M@GIECOABL@?$AAa?$AAr?$AA?9?$AAa?$AAe?$AA?$AA@ 0000000180017ae0     libucrt:lcidtoname_downlevel.obj
 0002:00005af0       ??_C@_1M@BMLMEKGI@?$AAa?$AAr?$AA?9?$AAb?$AAh?$AA?$AA@ 0000000180017af0     libucrt:lcidtoname_downlevel.obj
 0002:00005b00       ??_C@_1M@DAPFDGGB@?$AAa?$AAr?$AA?9?$AAd?$AAz?$AA?$AA@ 0000000180017b00     libucrt:lcidtoname_downlevel.obj
 0002:00005b10       ??_C@_1M@FJNKGKIG@?$AAa?$AAr?$AA?9?$AAe?$AAg?$AA?$AA@ 0000000180017b10     libucrt:lcidtoname_downlevel.obj
 0002:00005b20       ??_C@_1M@FLGKKCLO@?$AAa?$AAr?$AA?9?$AAi?$AAq?$AA?$AA@ 0000000180017b20     libucrt:lcidtoname_downlevel.obj
 0002:00005b30       ??_C@_1M@GNDIPALM@?$AAa?$AAr?$AA?9?$AAj?$AAo?$AA?$AA@ 0000000180017b30     libucrt:lcidtoname_downlevel.obj
 0002:00005b40       ??_C@_1M@DDMJFMGJ@?$AAa?$AAr?$AA?9?$AAk?$AAw?$AA?$AA@ 0000000180017b40     libucrt:lcidtoname_downlevel.obj
 0002:00005b50       ??_C@_1M@EJALMLHM@?$AAa?$AAr?$AA?9?$AAl?$AAb?$AA?$AA@ 0000000180017b50     libucrt:lcidtoname_downlevel.obj
 0002:00005b60       ??_C@_1M@MOBDBLOC@?$AAa?$AAr?$AA?9?$AAl?$AAy?$AA?$AA@ 0000000180017b60     libucrt:lcidtoname_downlevel.obj
 0002:00005b70       ??_C@_1M@JAOCLHDH@?$AAa?$AAr?$AA?9?$AAm?$AAa?$AA?$AA@ 0000000180017b70     libucrt:lcidtoname_downlevel.obj
 0002:00005b80       ??_C@_1M@JHPMKJIE@?$AAa?$AAr?$AA?9?$AAo?$AAm?$AA?$AA@ 0000000180017b80     libucrt:lcidtoname_downlevel.obj
 0002:00005b90       ??_C@_1M@OEPGHFNH@?$AAa?$AAr?$AA?9?$AAq?$AAa?$AA?$AA@ 0000000180017b90     libucrt:lcidtoname_downlevel.obj
 0002:00005ba0       ??_C@_1M@KJDONENM@?$AAa?$AAr?$AA?9?$AAs?$AAa?$AA?$AA@ 0000000180017ba0     libucrt:lcidtoname_downlevel.obj
 0002:00005bb0       ??_C@_1M@DMJDKLKM@?$AAa?$AAr?$AA?9?$AAs?$AAy?$AA?$AA@ 0000000180017bb0     libucrt:lcidtoname_downlevel.obj
 0002:00005bc0       ??_C@_1M@OMFIPEDC@?$AAa?$AAr?$AA?9?$AAt?$AAn?$AA?$AA@ 0000000180017bc0     libucrt:lcidtoname_downlevel.obj
 0002:00005bd0       ??_C@_1M@IHMHGAON@?$AAa?$AAr?$AA?9?$AAy?$AAe?$AA?$AA@ 0000000180017bd0     libucrt:lcidtoname_downlevel.obj
 0002:00005be0       ??_C@_1BG@KDCPGJGB@?$AAa?$AAz?$AA?9?$AAa?$AAz?$AA?9?$AAc?$AAy?$AAr?$AAl?$AA?$AA@ 0000000180017be0     libucrt:lcidtoname_downlevel.obj
 0002:00005bf8       ??_C@_1BG@IBCKDDOE@?$AAa?$AAz?$AA?9?$AAa?$AAz?$AA?9?$AAl?$AAa?$AAt?$AAn?$AA?$AA@ 0000000180017bf8     libucrt:lcidtoname_downlevel.obj
 0002:00005c10       ??_C@_1M@EGPFDCPD@?$AAb?$AAe?$AA?9?$AAb?$AAy?$AA?$AA@ 0000000180017c10     libucrt:lcidtoname_downlevel.obj
 0002:00005c20       ??_C@_1M@PCMGMCGC@?$AAb?$AAg?$AA?9?$AAb?$AAg?$AA?$AA@ 0000000180017c20     libucrt:lcidtoname_downlevel.obj
 0002:00005c30       ??_C@_1M@BJBMFGOB@?$AAb?$AAn?$AA?9?$AAi?$AAn?$AA?$AA@ 0000000180017c30     libucrt:lcidtoname_downlevel.obj
 0002:00005c40       ??_C@_1BG@EAKMMACD@?$AAb?$AAs?$AA?9?$AAb?$AAa?$AA?9?$AAl?$AAa?$AAt?$AAn?$AA?$AA@ 0000000180017c40     libucrt:lcidtoname_downlevel.obj
 0002:00005c58       ??_C@_1M@KGADAODK@?$AAc?$AAa?$AA?9?$AAe?$AAs?$AA?$AA@ 0000000180017c58     libucrt:lcidtoname_downlevel.obj
 0002:00005c68       ??_C@_1M@COAJPDHI@?$AAc?$AAs?$AA?9?$AAc?$AAz?$AA?$AA@ 0000000180017c68     libucrt:lcidtoname_downlevel.obj
 0002:00005c78       ??_C@_1M@DHBHFONH@?$AAc?$AAy?$AA?9?$AAg?$AAb?$AA?$AA@ 0000000180017c78     libucrt:lcidtoname_downlevel.obj
 0002:00005c88       ??_C@_1M@IMGKELGA@?$AAd?$AAa?$AA?9?$AAd?$AAk?$AA?$AA@ 0000000180017c88     libucrt:lcidtoname_downlevel.obj
 0002:00005c98       ??_C@_1M@NNDGDNGA@?$AAd?$AAe?$AA?9?$AAa?$AAt?$AA?$AA@ 0000000180017c98     libucrt:lcidtoname_downlevel.obj
 0002:00005ca8       ??_C@_1M@IKDBHEEM@?$AAd?$AAe?$AA?9?$AAc?$AAh?$AA?$AA@ 0000000180017ca8     libucrt:lcidtoname_downlevel.obj
 0002:00005cb8       ??_C@_1M@GFFOJMCJ@?$AAd?$AAe?$AA?9?$AAd?$AAe?$AA?$AA@ 0000000180017cb8     libucrt:lcidtoname_downlevel.obj
 0002:00005cc8       ??_C@_1M@MDNLKBPM@?$AAd?$AAe?$AA?9?$AAl?$AAi?$AA?$AA@ 0000000180017cc8     libucrt:lcidtoname_downlevel.obj
 0002:00005cd8       ??_C@_1M@NJBEEJNL@?$AAd?$AAe?$AA?9?$AAl?$AAu?$AA?$AA@ 0000000180017cd8     libucrt:lcidtoname_downlevel.obj
 0002:00005ce8       ??_C@_1O@GNNELBAP@?$AAd?$AAi?$AAv?$AA?9?$AAm?$AAv?$AA?$AA@ 0000000180017ce8     libucrt:lcidtoname_downlevel.obj
 0002:00005cf8       ??_C@_1M@EJLEOGAE@?$AAe?$AAl?$AA?9?$AAg?$AAr?$AA?$AA@ 0000000180017cf8     libucrt:lcidtoname_downlevel.obj
 0002:00005d08       ??_C@_1M@GMPONJN@?$AAe?$AAn?$AA?9?$AAa?$AAu?$AA?$AA@ 0000000180017d08     libucrt:lcidtoname_downlevel.obj
 0002:00005d18       ??_C@_1M@NIDIIPGF@?$AAe?$AAn?$AA?9?$AAb?$AAz?$AA?$AA@ 0000000180017d18     libucrt:lcidtoname_downlevel.obj
 0002:00005d28       ??_C@_1M@JEHMIMFO@?$AAe?$AAn?$AA?9?$AAc?$AAa?$AA?$AA@ 0000000180017d28     libucrt:lcidtoname_downlevel.obj
 0002:00005d38       ??_C@_1M@IGMJCDLA@?$AAe?$AAn?$AA?9?$AAc?$AAb?$AA?$AA@ 0000000180017d38     libucrt:lcidtoname_downlevel.obj
 0002:00005d48       ??_C@_1M@BNFIGBKG@?$AAe?$AAn?$AA?9?$AAg?$AAb?$AA?$AA@ 0000000180017d48     libucrt:lcidtoname_downlevel.obj
 0002:00005d58       ??_C@_1M@LKIFDIGP@?$AAe?$AAn?$AA?9?$AAi?$AAe?$AA?$AA@ 0000000180017d58     libucrt:lcidtoname_downlevel.obj
 0002:00005d68       ??_C@_1M@PJKFGCCO@?$AAe?$AAn?$AA?9?$AAj?$AAm?$AA?$AA@ 0000000180017d68     libucrt:lcidtoname_downlevel.obj
 0002:00005d78       ??_C@_1M@KPPKEPBO@?$AAe?$AAn?$AA?9?$AAn?$AAz?$AA?$AA@ 0000000180017d78     libucrt:lcidtoname_downlevel.obj
 0002:00005d88       ??_C@_1M@GMDGLDOB@?$AAe?$AAn?$AA?9?$AAp?$AAh?$AA?$AA@ 0000000180017d88     libucrt:lcidtoname_downlevel.obj
 0002:00005d98       ??_C@_1M@ONGIBJNA@?$AAe?$AAn?$AA?9?$AAt?$AAt?$AA?$AA@ 0000000180017d98     libucrt:lcidtoname_downlevel.obj
 0002:00005da8       ??_C@_1M@LLODPCMM@?$AAe?$AAn?$AA?9?$AAu?$AAs?$AA?$AA@ 0000000180017da8     libucrt:lcidtoname_downlevel.obj
 0002:00005db8       ??_C@_1M@LAKFNPAN@?$AAe?$AAn?$AA?9?$AAz?$AAa?$AA?$AA@ 0000000180017db8     libucrt:lcidtoname_downlevel.obj
 0002:00005dc8       ??_C@_1M@MFNHNHEO@?$AAe?$AAn?$AA?9?$AAz?$AAw?$AA?$AA@ 0000000180017dc8     libucrt:lcidtoname_downlevel.obj
 0002:00005dd8       ??_C@_1M@EJEINPHM@?$AAe?$AAs?$AA?9?$AAa?$AAr?$AA?$AA@ 0000000180017dd8     libucrt:lcidtoname_downlevel.obj
 0002:00005de8       ??_C@_1M@GNKPCCJA@?$AAe?$AAs?$AA?9?$AAb?$AAo?$AA?$AA@ 0000000180017de8     libucrt:lcidtoname_downlevel.obj
 0002:00005df8       ??_C@_1M@LEEGFONL@?$AAe?$AAs?$AA?9?$AAc?$AAl?$AA?$AA@ 0000000180017df8     libucrt:lcidtoname_downlevel.obj
 0002:00005e08       ??_C@_1M@KGPDPBDF@?$AAe?$AAs?$AA?9?$AAc?$AAo?$AA?$AA@ 0000000180017e08     libucrt:lcidtoname_downlevel.obj
 0002:00005e18       ??_C@_1M@EIAHOHH@?$AAe?$AAs?$AA?9?$AAc?$AAr?$AA?$AA@ 0000000180017e18     libucrt:lcidtoname_downlevel.obj
 0002:00005e28       ??_C@_1M@LLPGMBIN@?$AAe?$AAs?$AA?9?$AAd?$AAo?$AA?$AA@ 0000000180017e28     libucrt:lcidtoname_downlevel.obj
 0002:00005e38       ??_C@_1M@DKHMKNJA@?$AAe?$AAs?$AA?9?$AAe?$AAc?$AA?$AA@ 0000000180017e38     libucrt:lcidtoname_downlevel.obj
 0002:00005e48       ??_C@_1M@GKGFPKAP@?$AAe?$AAs?$AA?9?$AAe?$AAs?$AA?$AA@ 0000000180017e48     libucrt:lcidtoname_downlevel.obj
 0002:00005e58       ??_C@_1M@LKHKGDLN@?$AAe?$AAs?$AA?9?$AAg?$AAt?$AA?$AA@ 0000000180017e58     libucrt:lcidtoname_downlevel.obj
 0002:00005e68       ??_C@_1M@HEIIGGJD@?$AAe?$AAs?$AA?9?$AAh?$AAn?$AA?$AA@ 0000000180017e68     libucrt:lcidtoname_downlevel.obj
 0002:00005e78       ??_C@_1M@FBDHPPGD@?$AAe?$AAs?$AA?9?$AAm?$AAx?$AA?$AA@ 0000000180017e78     libucrt:lcidtoname_downlevel.obj
 0002:00005e88       ??_C@_1M@DPAGLNDH@?$AAe?$AAs?$AA?9?$AAn?$AAi?$AA?$AA@ 0000000180017e88     libucrt:lcidtoname_downlevel.obj
 0002:00005e98       ??_C@_1M@MDGOPGDD@?$AAe?$AAs?$AA?9?$AAp?$AAa?$AA?$AA@ 0000000180017e98     libucrt:lcidtoname_downlevel.obj
 0002:00005ea8       ??_C@_1M@EMAMGBGE@?$AAe?$AAs?$AA?9?$AAp?$AAe?$AA?$AA@ 0000000180017ea8     libucrt:lcidtoname_downlevel.obj
 0002:00005eb8       ??_C@_1M@IBMCAOEC@?$AAe?$AAs?$AA?9?$AAp?$AAr?$AA?$AA@ 0000000180017eb8     libucrt:lcidtoname_downlevel.obj
 0002:00005ec8       ??_C@_1M@FGMDIJED@?$AAe?$AAs?$AA?9?$AAp?$AAy?$AA?$AA@ 0000000180017ec8     libucrt:lcidtoname_downlevel.obj
 0002:00005ed8       ??_C@_1M@IIDEOLLL@?$AAe?$AAs?$AA?9?$AAs?$AAv?$AA?$AA@ 0000000180017ed8     libucrt:lcidtoname_downlevel.obj
 0002:00005ee8       ??_C@_1M@GAOBIPA@?$AAe?$AAs?$AA?9?$AAu?$AAy?$AA?$AA@ 0000000180017ee8     libucrt:lcidtoname_downlevel.obj
 0002:00005ef8       ??_C@_1M@JKFFICHJ@?$AAe?$AAs?$AA?9?$AAv?$AAe?$AA?$AA@ 0000000180017ef8     libucrt:lcidtoname_downlevel.obj
 0002:00005f08       ??_C@_1M@PNMLOJDF@?$AAe?$AAt?$AA?9?$AAe?$AAe?$AA?$AA@ 0000000180017f08     libucrt:lcidtoname_downlevel.obj
 0002:00005f18       ??_C@_1M@GHHLIKEI@?$AAe?$AAu?$AA?9?$AAe?$AAs?$AA?$AA@ 0000000180017f18     libucrt:lcidtoname_downlevel.obj
 0002:00005f28       ??_C@_1M@PBNONODE@?$AAf?$AAa?$AA?9?$AAi?$AAr?$AA?$AA@ 0000000180017f28     libucrt:lcidtoname_downlevel.obj
 0002:00005f38       ??_C@_1M@JEEHPMIL@?$AAf?$AAi?$AA?9?$AAf?$AAi?$AA?$AA@ 0000000180017f38     libucrt:lcidtoname_downlevel.obj
 0002:00005f48       ??_C@_1M@LMDCNDBA@?$AAf?$AAo?$AA?9?$AAf?$AAo?$AA?$AA@ 0000000180017f48     libucrt:lcidtoname_downlevel.obj
 0002:00005f58       ??_C@_1M@JKEOHLDK@?$AAf?$AAr?$AA?9?$AAb?$AAe?$AA?$AA@ 0000000180017f58     libucrt:lcidtoname_downlevel.obj
 0002:00005f68       ??_C@_1M@NOHADPMI@?$AAf?$AAr?$AA?9?$AAc?$AAa?$AA?$AA@ 0000000180017f68     libucrt:lcidtoname_downlevel.obj
 0002:00005f78       ??_C@_1M@KDHIHAEC@?$AAf?$AAr?$AA?9?$AAc?$AAh?$AA?$AA@ 0000000180017f78     libucrt:lcidtoname_downlevel.obj
 0002:00005f88       ??_C@_1M@MMBBFGAK@?$AAf?$AAr?$AA?9?$AAf?$AAr?$AA?$AA@ 0000000180017f88     libucrt:lcidtoname_downlevel.obj
 0002:00005f98       ??_C@_1M@PAFNENNF@?$AAf?$AAr?$AA?9?$AAl?$AAu?$AA?$AA@ 0000000180017f98     libucrt:lcidtoname_downlevel.obj
 0002:00005fa8       ??_C@_1M@EOHDJGDD@?$AAf?$AAr?$AA?9?$AAm?$AAc?$AA?$AA@ 0000000180017fa8     libucrt:lcidtoname_downlevel.obj
 0002:00005fb8       ??_C@_1M@FAPLLOPF@?$AAg?$AAl?$AA?9?$AAe?$AAs?$AA?$AA@ 0000000180017fb8     libucrt:lcidtoname_downlevel.obj
 0002:00005fc8       ??_C@_1M@FOPBFLOO@?$AAg?$AAu?$AA?9?$AAi?$AAn?$AA?$AA@ 0000000180017fc8     libucrt:lcidtoname_downlevel.obj
 0002:00005fd8       ??_C@_1M@KBMCINPM@?$AAh?$AAe?$AA?9?$AAi?$AAl?$AA?$AA@ 0000000180017fd8     libucrt:lcidtoname_downlevel.obj
 0002:00005fe8       ??_C@_1M@BBPHKFPJ@?$AAh?$AAi?$AA?9?$AAi?$AAn?$AA?$AA@ 0000000180017fe8     libucrt:lcidtoname_downlevel.obj
 0002:00005ff8       ??_C@_1M@PMBNDPHD@?$AAh?$AAr?$AA?9?$AAb?$AAa?$AA?$AA@ 0000000180017ff8     libucrt:lcidtoname_downlevel.obj
 0002:00006008       ??_C@_1M@BPCKOEGE@?$AAh?$AAr?$AA?9?$AAh?$AAr?$AA?$AA@ 0000000180018008     libucrt:lcidtoname_downlevel.obj
 0002:00006018       ??_C@_1M@GACBMHKE@?$AAh?$AAu?$AA?9?$AAh?$AAu?$AA?$AA@ 0000000180018018     libucrt:lcidtoname_downlevel.obj
 0002:00006028       ??_C@_1M@MILPAJJC@?$AAh?$AAy?$AA?9?$AAa?$AAm?$AA?$AA@ 0000000180018028     libucrt:lcidtoname_downlevel.obj
 0002:00006038       ??_C@_1M@BABBICEC@?$AAi?$AAd?$AA?9?$AAi?$AAd?$AA?$AA@ 0000000180018038     libucrt:lcidtoname_downlevel.obj
 0002:00006048       ??_C@_1M@BIKNHHPF@?$AAi?$AAs?$AA?9?$AAi?$AAs?$AA?$AA@ 0000000180018048     libucrt:lcidtoname_downlevel.obj
 0002:00006058       ??_C@_1M@NMPCJPHE@?$AAi?$AAt?$AA?9?$AAc?$AAh?$AA?$AA@ 0000000180018058     libucrt:lcidtoname_downlevel.obj
 0002:00006068       ??_C@_1M@GHKGFEDF@?$AAi?$AAt?$AA?9?$AAi?$AAt?$AA?$AA@ 0000000180018068     libucrt:lcidtoname_downlevel.obj
 0002:00006078       ??_C@_1M@NIEJCJJA@?$AAj?$AAa?$AA?9?$AAj?$AAp?$AA?$AA@ 0000000180018078     libucrt:lcidtoname_downlevel.obj
 0002:00006088       ??_C@_1M@JILFNBIM@?$AAk?$AAa?$AA?9?$AAg?$AAe?$AA?$AA@ 0000000180018088     libucrt:lcidtoname_downlevel.obj
 0002:00006098       ??_C@_1M@PACPMGPH@?$AAk?$AAk?$AA?9?$AAk?$AAz?$AA?$AA@ 0000000180018098     libucrt:lcidtoname_downlevel.obj
 0002:000060a8       ??_C@_1M@IELFGMHA@?$AAk?$AAn?$AA?9?$AAi?$AAn?$AA?$AA@ 00000001800180a8     libucrt:lcidtoname_downlevel.obj
 0002:000060b8       ??_C@_1O@IBBJHCH@?$AAk?$AAo?$AAk?$AA?9?$AAi?$AAn?$AA?$AA@ 00000001800180b8     libucrt:lcidtoname_downlevel.obj
 0002:000060c8       ??_C@_1M@DMHAEOGC@?$AAk?$AAo?$AA?9?$AAk?$AAr?$AA?$AA@ 00000001800180c8     libucrt:lcidtoname_downlevel.obj
 0002:000060d8       ??_C@_1M@HBAHBIGA@?$AAk?$AAy?$AA?9?$AAk?$AAg?$AA?$AA@ 00000001800180d8     libucrt:lcidtoname_downlevel.obj
 0002:000060e8       ??_C@_1M@KPMILCJG@?$AAl?$AAt?$AA?9?$AAl?$AAt?$AA?$AA@ 00000001800180e8     libucrt:lcidtoname_downlevel.obj
 0002:000060f8       ??_C@_1M@BDEKKCA@?$AAl?$AAv?$AA?9?$AAl?$AAv?$AA?$AA@ 00000001800180f8     libucrt:lcidtoname_downlevel.obj
 0002:00006108       ??_C@_1M@ELCKCCJJ@?$AAm?$AAi?$AA?9?$AAn?$AAz?$AA?$AA@ 0000000180018108     libucrt:lcidtoname_downlevel.obj
 0002:00006118       ??_C@_1M@CBOOLAPA@?$AAm?$AAk?$AA?9?$AAm?$AAk?$AA?$AA@ 0000000180018118     libucrt:lcidtoname_downlevel.obj
 0002:00006128       ??_C@_1M@GPHNBJKN@?$AAm?$AAl?$AA?9?$AAi?$AAn?$AA?$AA@ 0000000180018128     libucrt:lcidtoname_downlevel.obj
 0002:00006138       ??_C@_1M@PABJILIG@?$AAm?$AAn?$AA?9?$AAm?$AAn?$AA?$AA@ 0000000180018138     libucrt:lcidtoname_downlevel.obj
 0002:00006148       ??_C@_1M@FGBKKIPG@?$AAm?$AAr?$AA?9?$AAi?$AAn?$AA?$AA@ 0000000180018148     libucrt:lcidtoname_downlevel.obj
 0002:00006158       ??_C@_1M@NDBPDDAL@?$AAm?$AAs?$AA?9?$AAb?$AAn?$AA?$AA@ 0000000180018158     libucrt:lcidtoname_downlevel.obj
 0002:00006168       ??_C@_1M@OPIHOOPI@?$AAm?$AAs?$AA?9?$AAm?$AAy?$AA?$AA@ 0000000180018168     libucrt:lcidtoname_downlevel.obj
 0002:00006178       ??_C@_1M@PPDBCNFM@?$AAm?$AAt?$AA?9?$AAm?$AAt?$AA?$AA@ 0000000180018178     libucrt:lcidtoname_downlevel.obj
 0002:00006188       ??_C@_1M@KDJDKMDD@?$AAn?$AAb?$AA?9?$AAn?$AAo?$AA?$AA@ 0000000180018188     libucrt:lcidtoname_downlevel.obj
 0002:00006198       ??_C@_1M@KFCFLMJP@?$AAn?$AAl?$AA?9?$AAb?$AAe?$AA?$AA@ 0000000180018198     libucrt:lcidtoname_downlevel.obj
 0002:000061a8       ??_C@_1M@KPOPDDGO@?$AAn?$AAl?$AA?9?$AAn?$AAl?$AA?$AA@ 00000001800181a8     libucrt:lcidtoname_downlevel.obj
 0002:000061b8       ??_C@_1M@LJKPEMLN@?$AAn?$AAn?$AA?9?$AAn?$AAo?$AA?$AA@ 00000001800181b8     libucrt:lcidtoname_downlevel.obj
 0002:000061c8       ??_C@_1M@BDGHHBFL@?$AAn?$AAs?$AA?9?$AAz?$AAa?$AA?$AA@ 00000001800181c8     libucrt:lcidtoname_downlevel.obj
 0002:000061d8       ??_C@_1M@IDEHOAP@?$AAp?$AAa?$AA?9?$AAi?$AAn?$AA?$AA@ 00000001800181d8     libucrt:lcidtoname_downlevel.obj
 0002:000061e8       ??_C@_1M@HDBKGOGH@?$AAp?$AAl?$AA?9?$AAp?$AAl?$AA?$AA@ 00000001800181e8     libucrt:lcidtoname_downlevel.obj
 0002:000061f8       ??_C@_1M@LJLLCMEH@?$AAp?$AAt?$AA?9?$AAb?$AAr?$AA?$AA@ 00000001800181f8     libucrt:lcidtoname_downlevel.obj
 0002:00006208       ??_C@_1M@NCMONAAL@?$AAp?$AAt?$AA?9?$AAp?$AAt?$AA?$AA@ 0000000180018208     libucrt:lcidtoname_downlevel.obj
 0002:00006218       ??_C@_1O@EAKMAJDN@?$AAq?$AAu?$AAz?$AA?9?$AAb?$AAo?$AA?$AA@ 0000000180018218     libucrt:lcidtoname_downlevel.obj
 0002:00006228       ??_C@_1O@BHHPIGDN@?$AAq?$AAu?$AAz?$AA?9?$AAe?$AAc?$AA?$AA@ 0000000180018228     libucrt:lcidtoname_downlevel.obj
 0002:00006238       ??_C@_1O@GBAPEKMJ@?$AAq?$AAu?$AAz?$AA?9?$AAp?$AAe?$AA?$AA@ 0000000180018238     libucrt:lcidtoname_downlevel.obj
 0002:00006248       ??_C@_1M@CLGLEFBO@?$AAr?$AAo?$AA?9?$AAr?$AAo?$AA?$AA@ 0000000180018248     libucrt:lcidtoname_downlevel.obj
 0002:00006258       ??_C@_1M@CEEDODME@?$AAr?$AAu?$AA?9?$AAr?$AAu?$AA?$AA@ 0000000180018258     libucrt:lcidtoname_downlevel.obj
 0002:00006268       ??_C@_1M@HPKKKMPP@?$AAs?$AAa?$AA?9?$AAi?$AAn?$AA?$AA@ 0000000180018268     libucrt:lcidtoname_downlevel.obj
 0002:00006278       ??_C@_1M@BKMAIGOJ@?$AAs?$AAe?$AA?9?$AAf?$AAi?$AA?$AA@ 0000000180018278     libucrt:lcidtoname_downlevel.obj
 0002:00006288       ??_C@_1M@NDPIFLFI@?$AAs?$AAe?$AA?9?$AAn?$AAo?$AA?$AA@ 0000000180018288     libucrt:lcidtoname_downlevel.obj
 0002:00006298       ??_C@_1M@DANKKHJ@?$AAs?$AAe?$AA?9?$AAs?$AAe?$AA?$AA@ 0000000180018298     libucrt:lcidtoname_downlevel.obj
 0002:000062a8       ??_C@_1M@PNBLONPJ@?$AAs?$AAk?$AA?9?$AAs?$AAk?$AA?$AA@ 00000001800182a8     libucrt:lcidtoname_downlevel.obj
 0002:000062b8       ??_C@_1M@LFMODOAL@?$AAs?$AAl?$AA?9?$AAs?$AAi?$AA?$AA@ 00000001800182b8     libucrt:lcidtoname_downlevel.obj
 0002:000062c8       ??_C@_1O@DFKOMPG@?$AAs?$AAm?$AAa?$AA?9?$AAn?$AAo?$AA?$AA@ 00000001800182c8     libucrt:lcidtoname_downlevel.obj
 0002:000062d8       ??_C@_1O@NDKPBNNH@?$AAs?$AAm?$AAa?$AA?9?$AAs?$AAe?$AA?$AA@ 00000001800182d8     libucrt:lcidtoname_downlevel.obj
 0002:000062e8       ??_C@_1O@PLLKBHAB@?$AAs?$AAm?$AAj?$AA?9?$AAn?$AAo?$AA?$AA@ 00000001800182e8     libucrt:lcidtoname_downlevel.obj
 0002:000062f8       ??_C@_1O@CLEPOGCA@?$AAs?$AAm?$AAj?$AA?9?$AAs?$AAe?$AA?$AA@ 00000001800182f8     libucrt:lcidtoname_downlevel.obj
 0002:00006308       ??_C@_1O@DLGJGKMK@?$AAs?$AAm?$AAn?$AA?9?$AAf?$AAi?$AA?$AA@ 0000000180018308     libucrt:lcidtoname_downlevel.obj
 0002:00006318       ??_C@_1O@OJDJGAJC@?$AAs?$AAm?$AAs?$AA?9?$AAf?$AAi?$AA?$AA@ 0000000180018318     libucrt:lcidtoname_downlevel.obj
 0002:00006328       ??_C@_1M@BOFOGHPB@?$AAs?$AAq?$AA?9?$AAa?$AAl?$AA?$AA@ 0000000180018328     libucrt:lcidtoname_downlevel.obj
 0002:00006338       ??_C@_1BG@LJBBIPGB@?$AAs?$AAr?$AA?9?$AAb?$AAa?$AA?9?$AAc?$AAy?$AAr?$AAl?$AA?$AA@ 0000000180018338     libucrt:lcidtoname_downlevel.obj
 0002:00006350       ??_C@_1BG@JLBENFOE@?$AAs?$AAr?$AA?9?$AAb?$AAa?$AA?9?$AAl?$AAa?$AAt?$AAn?$AA?$AA@ 0000000180018350     libucrt:lcidtoname_downlevel.obj
 0002:00006368       ??_C@_1BG@KODPNHE@?$AAs?$AAr?$AA?9?$AAs?$AAp?$AA?9?$AAc?$AAy?$AAr?$AAl?$AA?$AA@ 0000000180018368     libucrt:lcidtoname_downlevel.obj
 0002:00006380       ??_C@_1BG@CIOGKHPB@?$AAs?$AAr?$AA?9?$AAs?$AAp?$AA?9?$AAl?$AAa?$AAt?$AAn?$AA?$AA@ 0000000180018380     libucrt:lcidtoname_downlevel.obj
 0002:00006398       ??_C@_1M@NGFJLMAC@?$AAs?$AAv?$AA?9?$AAf?$AAi?$AA?$AA@ 0000000180018398     libucrt:lcidtoname_downlevel.obj
 0002:000063a8       ??_C@_1M@MPJEJAJC@?$AAs?$AAv?$AA?9?$AAs?$AAe?$AA?$AA@ 00000001800183a8     libucrt:lcidtoname_downlevel.obj
 0002:000063b8       ??_C@_1M@MPNDHLFK@?$AAs?$AAw?$AA?9?$AAk?$AAe?$AA?$AA@ 00000001800183b8     libucrt:lcidtoname_downlevel.obj
 0002:000063c8       ??_C@_1O@KOHBJJI@?$AAs?$AAy?$AAr?$AA?9?$AAs?$AAy?$AA?$AA@ 00000001800183c8     libucrt:lcidtoname_downlevel.obj
 0002:000063d8       ??_C@_1M@LDCEFHA@?$AAt?$AAa?$AA?9?$AAi?$AAn?$AA?$AA@ 00000001800183d8     libucrt:lcidtoname_downlevel.obj
 0002:000063e8       ??_C@_1M@CNJOFAK@?$AAt?$AAe?$AA?9?$AAi?$AAn?$AA?$AA@ 00000001800183e8     libucrt:lcidtoname_downlevel.obj
 0002:000063f8       ??_C@_1M@GNAECACD@?$AAt?$AAh?$AA?9?$AAt?$AAh?$AA?$AA@ 00000001800183f8     libucrt:lcidtoname_downlevel.obj
 0002:00006408       ??_C@_1M@CHBIHOJO@?$AAt?$AAn?$AA?9?$AAz?$AAa?$AA?$AA@ 0000000180018408     libucrt:lcidtoname_downlevel.obj
 0002:00006418       ??_C@_1M@GCCMIGPJ@?$AAt?$AAr?$AA?9?$AAt?$AAr?$AA?$AA@ 0000000180018418     libucrt:lcidtoname_downlevel.obj
 0002:00006428       ??_C@_1M@CELMCNBK@?$AAt?$AAt?$AA?9?$AAr?$AAu?$AA?$AA@ 0000000180018428     libucrt:lcidtoname_downlevel.obj
 0002:00006438       ??_C@_1M@KLMCELGA@?$AAu?$AAk?$AA?9?$AAu?$AAa?$AA?$AA@ 0000000180018438     libucrt:lcidtoname_downlevel.obj
 0002:00006448       ??_C@_1M@EPAJJAJF@?$AAu?$AAr?$AA?9?$AAp?$AAk?$AA?$AA@ 0000000180018448     libucrt:lcidtoname_downlevel.obj
 0002:00006458       ??_C@_1BG@GEGPMCDJ@?$AAu?$AAz?$AA?9?$AAu?$AAz?$AA?9?$AAc?$AAy?$AAr?$AAl?$AA?$AA@ 0000000180018458     libucrt:lcidtoname_downlevel.obj
 0002:00006470       ??_C@_1BG@EGGKJILM@?$AAu?$AAz?$AA?9?$AAu?$AAz?$AA?9?$AAl?$AAa?$AAt?$AAn?$AA?$AA@ 0000000180018470     libucrt:lcidtoname_downlevel.obj
 0002:00006488       ??_C@_1M@GFOCLFF@?$AAv?$AAi?$AA?9?$AAv?$AAn?$AA?$AA@ 0000000180018488     libucrt:lcidtoname_downlevel.obj
 0002:00006498       ??_C@_1M@CPAMEDFI@?$AAx?$AAh?$AA?9?$AAz?$AAa?$AA?$AA@ 0000000180018498     libucrt:lcidtoname_downlevel.obj
 0002:000064a8       ??_C@_1O@EBKIFIGN@?$AAz?$AAh?$AA?9?$AAc?$AAh?$AAs?$AA?$AA@ 00000001800184a8     libucrt:lcidtoname_downlevel.obj
 0002:000064b8       ??_C@_1O@NMHPGANE@?$AAz?$AAh?$AA?9?$AAc?$AAh?$AAt?$AA?$AA@ 00000001800184b8     libucrt:lcidtoname_downlevel.obj
 0002:000064c8       ??_C@_1M@LPINJOMC@?$AAz?$AAh?$AA?9?$AAc?$AAn?$AA?$AA@ 00000001800184c8     libucrt:lcidtoname_downlevel.obj
 0002:000064d8       ??_C@_1M@OCJEJODD@?$AAz?$AAh?$AA?9?$AAh?$AAk?$AA?$AA@ 00000001800184d8     libucrt:lcidtoname_downlevel.obj
 0002:000064e8       ??_C@_1M@DNDLJINH@?$AAz?$AAh?$AA?9?$AAm?$AAo?$AA?$AA@ 00000001800184e8     libucrt:lcidtoname_downlevel.obj
 0002:000064f8       ??_C@_1M@MBFDNDND@?$AAz?$AAh?$AA?9?$AAs?$AAg?$AA?$AA@ 00000001800184f8     libucrt:lcidtoname_downlevel.obj
 0002:00006508       ??_C@_1M@IMEPLEPE@?$AAz?$AAh?$AA?9?$AAt?$AAw?$AA?$AA@ 0000000180018508     libucrt:lcidtoname_downlevel.obj
 0002:00006518       ??_C@_1M@BBGHNHJP@?$AAz?$AAu?$AA?9?$AAz?$AAa?$AA?$AA@ 0000000180018518     libucrt:lcidtoname_downlevel.obj
 0002:00006528       __real@3ff0000000000000    0000000180018528     libucrt:ceil.obj
 0002:00006780       __log10_256_lead           0000000180018780     libucrt:log10_256_lead_tail_table.obj
 0002:00006f90       __log10_256_tail           0000000180018f90     libucrt:log10_256_lead_tail_table.obj
 0002:000077a0       __log_F_inv_qword          00000001800197a0     libucrt:log_f_inv_qword_table.obj
 0002:00007fb0       ??_C@_05HGHHAHAP@log10?$AA@ 0000000180019fb0     libucrt:log_special.obj
 0002:00007fd0       ??_C@_1BA@BALFACEM@?$AAC?$AAO?$AAN?$AAO?$AAU?$AAT?$AA$?$AA?$AA@ 0000000180019fd0     libucrt:initcon.obj
 0002:00008040       _load_config_used          000000018001a040     LIBCMT:loadcfg.obj
 0002:00008440       __rtc_iaa                  000000018001a440     LIBCMT:_initsect_.obj
 0002:00008448       __rtc_izz                  000000018001a448     LIBCMT:_initsect_.obj
 0002:00008450       __rtc_taa                  000000018001a450     LIBCMT:_initsect_.obj
 0002:00008458       __rtc_tzz                  000000018001a458     LIBCMT:_initsect_.obj
 0002:00009224       __IMPORT_DESCRIPTOR_KERNEL32 000000018001b224     kernel32:KERNEL32.dll
 0002:00009238       __IMPORT_DESCRIPTOR_USER32 000000018001b238     user32:USER32.dll
 0002:0000924c       __IMPORT_DESCRIPTOR_GDI32  000000018001b24c     gdi32:GDI32.dll
 0002:00009260       __IMPORT_DESCRIPTOR_ole32  000000018001b260     ole32:ole32.dll
 0002:00009274       __NULL_IMPORT_DESCRIPTOR   000000018001b274     kernel32:KERNEL32.dll
 0003:00000000       ?g_TerminatedThreadIdx@@3JA 000000018001c000     common-kernel64:WThreads.obj
 0003:00000010       __security_cookie          000000018001c010     LIBCMT:gs_cookie.obj
 0003:00000018       __security_cookie_complement 000000018001c018     LIBCMT:gs_cookie.obj
 0003:00000020       __scrt_native_dllmain_reason 000000018001c020     LIBCMT:utility.obj
 0003:00000028       __isa_available            000000018001c028     LIBCMT:_cpu_disp_.obj
 0003:0000002c       __isa_enabled              000000018001c02c     LIBCMT:_cpu_disp_.obj
 0003:00000030       __memcpy_nt_iters          000000018001c030     LIBCMT:_cpu_disp_.obj
 0003:00000050       __abort_behavior           000000018001c050     libucrt:abort.obj
 0003:00000060       _iob                       000000018001c060     libucrt:_file.obj
 0003:00000170       __acrt_initial_locale_data 000000018001c170     libucrt:nlsdata.obj
 0003:000002c8       __acrt_initial_locale_pointers 000000018001c2c8     libucrt:nlsdata.obj
 0003:000002d8       __acrt_wide_c_locale_string 000000018001c2d8     libucrt:nlsdata.obj
 0003:000002e0       __acrt_initial_multibyte_data 000000018001c2e0     libucrt:mbctype.obj
 0003:00000508       __acrt_current_multibyte_data 000000018001c508     libucrt:mbctype.obj
 0003:00000610       _mbctype                   000000018001c610     libucrt:mbctype.obj
 0003:00000720       _mbcasemap                 000000018001c720     libucrt:mbctype.obj
 0003:00000820       __globallocalestatus       000000018001c820     libucrt:glstatus.obj
 0003:00000830       __acrt_lconv_c             000000018001c830     libucrt:localeconv.obj
 0003:000008c8       __acrt_lconv_static_decimal 000000018001c8c8     libucrt:localeconv.obj
 0003:000008cc       __acrt_lconv_static_W_decimal 000000018001c8cc     libucrt:localeconv.obj
 0003:000008e8       __dcrt_lowio_console_output_handle 000000018001c8e8     libucrt:initcon.obj
 0003:000008f0       _fltused                   000000018001c8f0     LIBCMT:fltused.obj
 0003:00000900       ?ghModule@@3PEAUHINSTANCE__@@EA 000000018001c900     gdip.obj
 0003:00000908       ?gnLastWin32Error@@3KA     000000018001c908     gdip.obj
 0003:00000910       ?ghHeap@@3PEAXEA           000000018001c910     common-kernel64:Memory.obj
 0003:00000918       ?g_LastDeletePtr@@3PEAXEA  000000018001c918     common-kernel64:Memory.obj
 0003:00000920       ?g_ThreadsIdx@@3JA         000000018001c920     common-kernel64:WThreads.obj
 0003:00009138       ?_OptionsStorage@?1??__local_stdio_printf_options@@9@4_KA 0000000180025138     common-kernel64:WThreads.obj
 0003:000096c0       ?__type_info_root_node@@3U__type_info_node@@A 00000001800256c0     LIBCMT:tncleanup.obj
 0003:000096d0       ?_OptionsStorage@?1??__local_stdio_scanf_options@@9@4_KA 00000001800256d0     LIBCMT:default_local_stdio_options.obj
 0003:000096d8       __scrt_current_native_startup_state 00000001800256d8     LIBCMT:utility.obj
 0003:000096e0       __scrt_native_startup_lock 00000001800256e0     LIBCMT:utility.obj
 0003:0000971c       __scrt_debugger_hook_flag  000000018002571c     LIBCMT:utility_desktop.obj
 0003:00009720       __favor                    0000000180025720     LIBCMT:_cpu_disp_.obj
 0003:00009728       ?m_pGetParameter@UnDecorator@@0P6APEADJ@ZEA 0000000180025728     libvcruntime:undname.obj
 0003:00009730       ?m_CHPENameOffset@UnDecorator@@0KA 0000000180025730     libvcruntime:undname.obj
 0003:00009734       ?m_recursionLevel@UnDecorator@@0KA 0000000180025734     libvcruntime:undname.obj
 0003:00009738       ?pArgList@UnDecorator@@0PEAVReplicator@@EA 0000000180025738     libvcruntime:undname.obj
 0003:00009740       ?pZNameList@UnDecorator@@0PEAVReplicator@@EA 0000000180025740     libvcruntime:undname.obj
 0003:00009748       ?pTemplateArgList@UnDecorator@@0PEAVReplicator@@EA 0000000180025748     libvcruntime:undname.obj
 0003:00009750       ?gName@UnDecorator@@0PEBDEB 0000000180025750     libvcruntime:undname.obj
 0003:00009758       ?name@UnDecorator@@0PEBDEB 0000000180025758     libvcruntime:undname.obj
 0003:00009760       ?disableFlags@UnDecorator@@0KA 0000000180025760     libvcruntime:undname.obj
 0003:00009764       ?fExplicitTemplateParams@UnDecorator@@0_NA 0000000180025764     libvcruntime:undname.obj
 0003:00009765       ?fGetTemplateArgumentList@UnDecorator@@0_NA 0000000180025765     libvcruntime:undname.obj
 0003:00009878       __pPurecall                0000000180025878     libvcruntime:purevirt_data.obj
 0003:00009880       ?__WinRTOutOfMemoryExceptionCallback@@3P6APEAXXZEA 0000000180025880     libvcruntime:ehhelpers.obj
 0003:000099a8       _environ_table             00000001800259a8     libucrt:environment_initialization.obj
 0003:000099b0       _wenviron_table            00000001800259b0     libucrt:environment_initialization.obj
 0003:000099b8       __dcrt_initial_wide_environment 00000001800259b8     libucrt:environment_initialization.obj
 0003:000099c0       __dcrt_initial_narrow_environment 00000001800259c0     libucrt:environment_initialization.obj
 0003:000099c8       __acrt_atexit_table        00000001800259c8     libucrt:onexit.obj
 0003:000099e0       __acrt_at_quick_exit_table 00000001800259e0     libucrt:onexit.obj
 0003:00009a00       _nstream                   0000000180025a00     libucrt:_file.obj
 0003:00009a08       __piob                     0000000180025a08     libucrt:_file.obj
 0003:00009a18       __acrt_stdout_buffer       0000000180025a18     libucrt:_sftbuf.obj
 0003:00009a20       __acrt_stderr_buffer       0000000180025a20     libucrt:_sftbuf.obj
 0003:00009a28       __acrt_locale_changed_data 0000000180025a28     libucrt:wsetlocale.obj
 0003:00009a30       __acrt_current_locale_data 0000000180025a30     libucrt:nlsdata.obj
 0003:00009a40       __pioinfo                  0000000180025a40     libucrt:ioinit.obj
 0003:00009e40       _nhandle                   0000000180025e40     libucrt:ioinit.obj
 0003:0000a204       __mbcodepage               0000000180026204     libucrt:mbctype.obj
 0003:0000a208       __ismbcodepage             0000000180026208     libucrt:mbctype.obj
 0003:0000a210       __mbulinfo                 0000000180026210     libucrt:mbctype.obj
 0003:0000a220       __mblocalename             0000000180026220     libucrt:mbctype.obj
 0003:0000a22c       __argc                     000000018002622c     libucrt:argv_data.obj
 0003:0000a230       __argv                     0000000180026230     libucrt:argv_data.obj
 0003:0000a238       __wargv                    0000000180026238     libucrt:argv_data.obj
 0003:0000a240       _acmdln                    0000000180026240     libucrt:argv_data.obj
 0003:0000a248       _wcmdln                    0000000180026248     libucrt:argv_data.obj
 0003:0000a250       _pgmptr                    0000000180026250     libucrt:argv_data.obj
 0003:0000a258       __acrt_heap                0000000180026258     libucrt:heap_handle.obj
 0003:0000a294       __acrt_lconv_static_null   0000000180026294     libucrt:localeconv.obj
 0003:0000a298       __acrt_lconv_static_W_null 0000000180026298     libucrt:localeconv.obj
 0003:0000a2a0       __fma3_is_available        00000001800262a0     libucrt:fma3_available.obj
 0003:0000a2a4       __use_fma3_lib             00000001800262a4     libucrt:fma3_available.obj
 0003:0000a2a8       __scrt_ucrt_dll_is_in_use  00000001800262a8     <common>
 0003:0000a2b0       __dyn_tls_init_callback    00000001800262b0     <common>

 entry point at        0001:000021b4

 Static symbols

 0000:fffd6000       .debug$S                   0000000180000000     kernel32:KERNEL32.dll
 0000:fffd6000       .debug$S                   0000000180000000     kernel32:KERNEL32.dll
 0000:fffd6000       .debug$S                   0000000180000000     kernel32:KERNEL32.dll
 0000:fffd6000       .debug$S                   0000000180000000     gdi32:GDI32.dll
 0000:fffd6000       .debug$S                   0000000180000000     kernel32:KERNEL32.dll
 0000:fffd6000       .debug$S                   0000000180000000     kernel32:KERNEL32.dll
 0000:fffd6000       .debug$S                   0000000180000000     gdi32:GDI32.dll
 0000:fffd6000       .debug$S                   0000000180000000     kernel32:KERNEL32.dll
 0000:fffd6000       .debug$S                   0000000180000000     user32:USER32.dll
 0000:fffd6000       .debug$S                   0000000180000000     kernel32:KERNEL32.dll
 0000:fffd6000       .debug$S                   0000000180000000     kernel32:KERNEL32.dll
 0000:fffd6000       .debug$S                   0000000180000000     gdi+.exp
 0000:fffd6000       .debug$S                   0000000180000000     kernel32:KERNEL32.dll
 0000:fffd6000       .debug$S                   0000000180000000     gdi32:GDI32.dll
 0000:fffd6000       .debug$S                   0000000180000000     kernel32:KERNEL32.dll
 0000:fffd6000       .debug$S                   0000000180000000     kernel32:KERNEL32.dll
 0000:fffd6000       .debug$S                   0000000180000000     gdi32:GDI32.dll
 0000:fffd6000       .debug$S                   0000000180000000     ole32:ole32.dll
 0000:fffd6000       .debug$S                   0000000180000000     kernel32:KERNEL32.dll
 0000:fffd6000       .debug$S                   0000000180000000     kernel32:KERNEL32.dll
 0000:fffd6000       .debug$S                   0000000180000000     kernel32:KERNEL32.dll
 0000:fffd6000       .debug$S                   0000000180000000     ole32:ole32.dll
 0000:fffd6000       .debug$S                   0000000180000000     kernel32:KERNEL32.dll
 0000:fffd6000       .debug$S                   0000000180000000     kernel32:KERNEL32.dll
 0000:fffd6000       .debug$S                   0000000180000000     kernel32:KERNEL32.dll
 0000:fffd6000       .debug$S                   0000000180000000     kernel32:KERNEL32.dll
 0000:fffd6000       .debug$S                   0000000180000000     kernel32:KERNEL32.dll
 0000:fffd6000       .debug$S                   0000000180000000     kernel32:KERNEL32.dll
 0000:fffd6000       .debug$S                   0000000180000000     kernel32:KERNEL32.dll
 0000:fffd6000       .debug$S                   0000000180000000     kernel32:KERNEL32.dll
 0000:fffd6000       .debug$S                   0000000180000000     kernel32:KERNEL32.dll
 0000:fffd6000       .debug$S                   0000000180000000     kernel32:KERNEL32.dll
 0000:fffd6000       .debug$S                   0000000180000000     kernel32:KERNEL32.dll
 0000:fffd6000       .debug$S                   0000000180000000     kernel32:KERNEL32.dll
 0000:fffd6000       .debug$S                   0000000180000000     kernel32:KERNEL32.dll
 0000:fffd6000       .debug$S                   0000000180000000     kernel32:KERNEL32.dll
 0000:fffd6000       .debug$S                   0000000180000000     kernel32:KERNEL32.dll
 0000:fffd6000       .debug$S                   0000000180000000     kernel32:KERNEL32.dll
 0000:fffd6000       .debug$S                   0000000180000000     kernel32:KERNEL32.dll
 0000:fffd6000       .debug$S                   0000000180000000     kernel32:KERNEL32.dll
 0000:fffd6000       .debug$S                   0000000180000000     kernel32:KERNEL32.dll
 0000:fffd6000       .debug$S                   0000000180000000     kernel32:KERNEL32.dll
 0000:fffd6000       .debug$S                   0000000180000000     kernel32:KERNEL32.dll
 0000:fffd6000       .debug$S                   0000000180000000     kernel32:KERNEL32.dll
 0000:fffd6000       .debug$S                   0000000180000000     kernel32:KERNEL32.dll
 0000:fffd6000       .debug$S                   0000000180000000     kernel32:KERNEL32.dll
 0000:fffd6000       .debug$S                   0000000180000000     kernel32:KERNEL32.dll
 0000:fffd6000       .debug$S                   0000000180000000     kernel32:KERNEL32.dll
 0000:fffd6000       .debug$S                   0000000180000000     kernel32:KERNEL32.dll
 0000:fffd6000       .debug$S                   0000000180000000     kernel32:KERNEL32.dll
 0000:fffd6000       .debug$S                   0000000180000000     kernel32:KERNEL32.dll
 0000:fffd6000       .debug$S                   0000000180000000     kernel32:KERNEL32.dll
 0000:fffd6000       .debug$S                   0000000180000000     kernel32:KERNEL32.dll
 0000:fffd6000       .debug$S                   0000000180000000     kernel32:KERNEL32.dll
 0000:fffd6000       .debug$S                   0000000180000000     kernel32:KERNEL32.dll
 0000:fffd6000       .debug$S                   0000000180000000     kernel32:KERNEL32.dll
 0000:fffd6000       .debug$S                   0000000180000000     kernel32:KERNEL32.dll
 0000:fffd6000       .debug$S                   0000000180000000     kernel32:KERNEL32.dll
 0000:fffd6000       .debug$S                   0000000180000000     kernel32:KERNEL32.dll
 0000:fffd6000       .debug$S                   0000000180000000     kernel32:KERNEL32.dll
 0000:fffd6000       .debug$S                   0000000180000000     kernel32:KERNEL32.dll
 0000:fffd6000       .debug$S                   0000000180000000     kernel32:KERNEL32.dll
 0000:fffd6000       .debug$S                   0000000180000000     kernel32:KERNEL32.dll
 0000:fffd6000       .debug$S                   0000000180000000     kernel32:KERNEL32.dll
 0000:fffd6000       .debug$S                   0000000180000000     kernel32:KERNEL32.dll
 0000:fffd6000       .debug$S                   0000000180000000     kernel32:KERNEL32.dll
 0000:fffd6000       .debug$S                   0000000180000000     kernel32:KERNEL32.dll
 0000:fffd6000       .debug$S                   0000000180000000     kernel32:KERNEL32.dll
 0000:fffd6000       .debug$S                   0000000180000000     kernel32:KERNEL32.dll
 0000:fffd6000       .debug$S                   0000000180000000     kernel32:KERNEL32.dll
 0000:fffd6000       .debug$S                   0000000180000000     kernel32:KERNEL32.dll
 0000:fffd6000       .debug$S                   0000000180000000     kernel32:KERNEL32.dll
 0000:fffd6000       .debug$S                   0000000180000000     kernel32:KERNEL32.dll
 0000:fffd6000       .debug$S                   0000000180000000     kernel32:KERNEL32.dll
 0000:fffd6000       .debug$S                   0000000180000000     kernel32:KERNEL32.dll
 0000:fffd6000       .debug$S                   0000000180000000     kernel32:KERNEL32.dll
 0000:fffd6000       .debug$S                   0000000180000000     kernel32:KERNEL32.dll
 0000:fffd6000       .debug$S                   0000000180000000     kernel32:KERNEL32.dll
 0000:fffd6000       .debug$S                   0000000180000000     kernel32:KERNEL32.dll
 0000:fffd6000       .debug$S                   0000000180000000     kernel32:KERNEL32.dll
 0000:fffd6000       .debug$S                   0000000180000000     kernel32:KERNEL32.dll
 0000:fffd6000       .debug$S                   0000000180000000     kernel32:KERNEL32.dll
 0000:fffd6000       .debug$S                   0000000180000000     kernel32:KERNEL32.dll
 0000:fffd6000       .debug$S                   0000000180000000     kernel32:KERNEL32.dll
 0000:fffd6000       .debug$S                   0000000180000000     kernel32:KERNEL32.dll
 0000:fffd6000       .debug$S                   0000000180000000     kernel32:KERNEL32.dll
 0000:fffd6000       .debug$S                   0000000180000000     kernel32:KERNEL32.dll
 0000:fffd6000       .debug$S                   0000000180000000     kernel32:KERNEL32.dll
 0000:fffd6000       .debug$S                   0000000180000000     kernel32:KERNEL32.dll
 0000:fffd6000       .debug$S                   0000000180000000     kernel32:KERNEL32.dll
 0000:fffd6000       .debug$S                   0000000180000000     kernel32:KERNEL32.dll
 0000:fffd6000       .debug$S                   0000000180000000     kernel32:KERNEL32.dll
 0000:fffd6000       .debug$S                   0000000180000000     kernel32:KERNEL32.dll
 0000:fffd6000       .debug$S                   0000000180000000     kernel32:KERNEL32.dll
 0000:fffd6000       .debug$S                   0000000180000000     kernel32:KERNEL32.dll
 0000:fffd6000       .debug$S                   0000000180000000     kernel32:KERNEL32.dll
 0000:fffd6000       .debug$S                   0000000180000000     kernel32:KERNEL32.dll
 0000:fffd6000       .debug$S                   0000000180000000     kernel32:KERNEL32.dll
 0000:fffd6000       .debug$S                   0000000180000000     kernel32:KERNEL32.dll
 0000:fffd6000       .debug$S                   0000000180000000     kernel32:KERNEL32.dll
 0000:fffd6000       .debug$S                   0000000180000000     kernel32:KERNEL32.dll
 0000:fffd6000       .debug$S                   0000000180000000     kernel32:KERNEL32.dll
 0000:fffd6000       .debug$S                   0000000180000000     kernel32:KERNEL32.dll
 0000:fffd6000       .debug$S                   0000000180000000     kernel32:KERNEL32.dll
 0000:fffd6000       .debug$S                   0000000180000000     kernel32:KERNEL32.dll
 0000:fffd6000       .debug$S                   0000000180000000     kernel32:KERNEL32.dll
 0000:fffd6000       .debug$S                   0000000180000000     user32:USER32.dll
 0000:fffd6000       .debug$S                   0000000180000000     kernel32:KERNEL32.dll
 0000:fffd6000       .debug$S                   0000000180000000     kernel32:KERNEL32.dll
 0000:fffd6000       .debug$S                   0000000180000000     kernel32:KERNEL32.dll
 0000:fffd6000       .debug$S                   0000000180000000     kernel32:KERNEL32.dll
 0000:fffd6000       .debug$S                   0000000180000000     gdi32:GDI32.dll
 0000:fffd6000       .debug$S                   0000000180000000     gdi32:GDI32.dll
 0000:fffd6000       .debug$S                   0000000180000000     user32:USER32.dll
 0000:fffd6000       .debug$S                   0000000180000000     kernel32:KERNEL32.dll
 0000:fffd6000       .debug$S                   0000000180000000     kernel32:KERNEL32.dll
 0000:fffd6000       .debug$S                   0000000180000000     kernel32:KERNEL32.dll
 0001:00001cf4       capture_current_context    0000000180002cf4 f   LIBCMT:gs_report.obj
 0001:00001d64       capture_previous_context   0000000180002d64 f   LIBCMT:gs_report.obj
 0001:00001e60       $$000000                   0000000180002e60     LIBCMT:_amdsecgs_.obj
 0001:00001e94       ?dllmain_crt_dispatch@@YAHQEAUHINSTANCE__@@KQEAX@Z 0000000180002e94 f   LIBCMT:dll_dllmain.obj
 0001:00001ee4       ?dllmain_crt_process_attach@@YAHQEAUHINSTANCE__@@QEAX@Z 0000000180002ee4 f   LIBCMT:dll_dllmain.obj
 0001:00001ffc       ?dllmain_crt_process_detach@@YAH_N@Z 0000000180002ffc f   LIBCMT:dll_dllmain.obj
 0001:00002080       ?dllmain_dispatch@@YAHQEAUHINSTANCE__@@KQEAX@Z 0000000180003080 f   LIBCMT:dll_dllmain.obj
 0001:00002ae0       $$000000                   0000000180003ae0     libvcruntime:memset.obj
 0001:00002bdc       MsetTab                    0000000180003bdc     libvcruntime:memset.obj
 0001:00003140       $$000000                   0000000180004140     libvcruntime:_jmpuwind_.obj
 0001:00003408       ?try_get_function@@YAPEAXW4function_id@?A0x89697e75@@QEBDQEBW4module_id@2@2@Z 0000000180004408 f   libvcruntime:winapi_downlevel.obj
 0001:000037f0       $$000000                   00000001800047f0     libvcruntime:memcpy.obj
 0001:00003897       MoveSmall                  0000000180004897     libvcruntime:memcpy.obj
 0001:00003c50       $$000000                   0000000180004c50     libvcruntime:handlers.obj
 0001:00005548       ?atexit_exception_filter@@YAHK@Z 0000000180006548 f   libucrt:exit.obj
 0001:00005554       ?common_exit@@YAXHW4_crt_exit_cleanup_mode@@W4_crt_exit_return_mode@@@Z 0000000180006554 f   libucrt:exit.obj
 0001:000056c0       ?exit_or_terminate_process@@YAXI@Z 00000001800066c0 f   libucrt:exit.obj
 0001:0000570c       ?try_cor_exit_process@@YAXI@Z 000000018000670c f   libucrt:exit.obj
 0001:000057a4       ??$parse_command_line@D@@YAXPEADPEAPEAD0PEA_K2@Z 00000001800067a4 f   libucrt:argv_parsing.obj
 0001:00005b3c       ??$common_initialize_environment_nolock@D@@YAHXZ 0000000180006b3c f   libucrt:environment_initialization.obj
 0001:00005ba8       ??$create_environment@D@@YAQEAPEADQEAD@Z 0000000180006ba8 f   libucrt:environment_initialization.obj
 0001:00005ca4       ??$free_environment@D@@YAXQEAPEAD@Z 0000000180006ca4 f   libucrt:environment_initialization.obj
 0001:00005ca4       ??$free_environment@_W@@YAXQEAPEA_W@Z 0000000180006ca4 f   libucrt:environment_initialization.obj
 0001:00005ce8       ??$uninitialize_environment_internal@D@@YAXAEAPEAPEAD@Z 0000000180006ce8 f   libucrt:environment_initialization.obj
 0001:00005d04       ??$uninitialize_environment_internal@_W@@YAXAEAPEAPEA_W@Z 0000000180006d04 f   libucrt:environment_initialization.obj
 0001:00005f7c       initialize_global_variables 0000000180006f7c f   libucrt:initialization.obj
 0001:00005f90       initialize_c               0000000180006f90 f   libucrt:initialization.obj
 0001:00005fb4       uninitialize_c             0000000180006fb4 f   libucrt:initialization.obj
 0001:00005fb4       report_memory_leaks        0000000180006fb4 f   libucrt:initialization.obj
 0001:00005fb4       uninitialize_global_state_isolation 0000000180006fb4 f   libucrt:initialization.obj
 0001:00005fb4       initialize_global_state_isolation 0000000180006fb4 f   libucrt:initialization.obj
 0001:00005fb4       initialize_environment     0000000180006fb4 f   libucrt:initialization.obj
 0001:00005fb8       uninitialize_environment   0000000180006fb8 f   libucrt:initialization.obj
 0001:00005fc8       initialize_pointers        0000000180006fc8 f   libucrt:initialization.obj
 0001:0000601c       uninitialize_vcruntime     000000018000701c f   libucrt:initialization.obj
 0001:00006024       uninitialize_allocated_memory 0000000180007024 f   libucrt:initialization.obj
 0001:000064e0       $$000000                   00000001800074e0     libucrt:strncmp.obj
 0001:000068b8       ?internal_isupper_l@@YA_NHQEAU__crt_locale_pointers@@@Z 00000001800078b8 f   libucrt:tolower_toupper.obj
 0001:0000738c       ?construct_ptd_array@@YAXQEAU__acrt_ptd@@@Z 000000018000838c f   libucrt:per_thread_data.obj
 0001:0000745c       ?destroy_fls@@YAXPEAX@Z    000000018000845c f   libucrt:per_thread_data.obj
 0001:0000747c       ?destroy_ptd_array@@YAXQEAU__acrt_ptd@@@Z 000000018000847c f   libucrt:per_thread_data.obj
 0001:00007574       ?replace_current_thread_locale_nolock@@YAXQEAU__acrt_ptd@@QEAU__crt_locale_data@@@Z 0000000180008574 f   libucrt:per_thread_data.obj
 0001:00007884       ?fp_format_a@@YAHQEBNPEAD_KQEAD2H_NIQEAU__crt_locale_pointers@@@Z 0000000180008884 f   libucrt:cvt.obj
 0001:00007be4       ?fp_format_e@@YAHQEBNQEAD_K12H_NIQEAU__crt_locale_pointers@@@Z 0000000180008be4 f   libucrt:cvt.obj
 0001:00007cb4       ?fp_format_e_internal@@YAHQEAD_KH_NIQEAU_strflt@@2QEAU__crt_locale_pointers@@@Z 0000000180008cb4 f   libucrt:cvt.obj
 0001:00007e90       ?fp_format_f_internal@@YAHQEAD_KHQEAU_strflt@@_NQEAU__crt_locale_pointers@@@Z 0000000180008e90 f   libucrt:cvt.obj
 0001:00007fd8       ?fp_format_g@@YAHQEBNQEAD_K12H_NIQEAU__crt_locale_pointers@@@Z 0000000180008fd8 f   libucrt:cvt.obj
 0001:00008110       ?fp_format_nan_or_infinity@@YAHW4__acrt_fp_class@@_NPEAD_K1@Z 0000000180009110 f   libucrt:cvt.obj
 0001:000086c0       ?initialize_inherited_file_handles_nolock@@YAXXZ 00000001800096c0 f   libucrt:ioinit.obj
 0001:000087ac       ?initialize_stdio_handles_nolock@@YAXXZ 00000001800097ac f   libucrt:ioinit.obj
 0001:000089dc       ?try_get_function@@YAPEAXW4function_id@?A0x63058377@@QEBDQEBW4module_id@2@2@Z 00000001800099dc f   libucrt:winapi_thunks.obj
 0001:00009038       ?<helper_func_cdecl>@<lambda_2feae5270eb4d0d5532525f423405775>@@CAHPEBX0@Z 000000018000a038 f   libucrt:argv_wildcards.obj
 0001:0000904c       ??$common_expand_argv_wildcards@D@@YAHQEAPEADQEAPEAPEAD@Z 000000018000a04c f   libucrt:argv_wildcards.obj
 0001:00009258       ??$copy_and_add_argument_to_buffer@D@@YAHQEBD0_KAEAV?$argument_list@D@?A0xca0879c4@@@Z 000000018000a258 f   libucrt:argv_wildcards.obj
 0001:00009368       ??$expand_argument_wildcards@D@@YAHQEAD0AEAV?$argument_list@D@?A0xca0879c4@@@Z 000000018000a368 f   libucrt:argv_wildcards.obj
 0001:0000961c       ??R<lambda_ad1ced32f4ac17aa236e5ef05d6b3b7c>@@QEBAXXZ 000000018000a61c f   libucrt:mbctype.obj
 0001:00009834       ?getSystemCP@@YAHH@Z       000000018000a834 f   libucrt:mbctype.obj
 0001:000098b4       ?setSBCS@@YAXPEAU__crt_multibyte_data@@@Z 000000018000a8b4 f   libucrt:mbctype.obj
 0001:00009944       ?setSBUpLow@@YAXPEAU__crt_multibyte_data@@@Z 000000018000a944 f   libucrt:mbctype.obj
 0001:00009b28       ?setmbcp_internal@@YAHH_N@Z 000000018000ab28 f   libucrt:mbctype.obj
 0001:0000a070       ?x_ismbbtype_l@@YAHPEAU__crt_locale_pointers@@IHH@Z 000000018000b070 f   libucrt:ismbbyte.obj
 0001:0000a974       ?__acrt_LCMapStringA_stat@@YAHPEAU__crt_locale_pointers@@PEB_WKPEBDHPEADHHH@Z 000000018000b974 f   libucrt:lcmapstringa.obj
 0001:0000ca7c       memcpy_s                   000000018000da7c f   libucrt:cfout.obj
 0001:0000cc88       common_flush_all           000000018000dc88 f   libucrt:fflush.obj
 0001:0000cf84       ?free_crt_array_internal@@YAXQEAPEBX_K@Z 000000018000df84 f   libucrt:inittime.obj
 0001:0000d5b4       ?GetTableIndexFromLocaleName@@YAHPEB_W@Z 000000018000e5b4 f   libucrt:lcidtoname_downlevel.obj
 0001:0000d6b0       ?shortsort@@YAXPEAD0_KP6AHPEBX2@Z@Z 000000018000e6b0 f   libucrt:qsort.obj
 0001:0000dcc8       ?initialize_multibyte@@YAHXZ 000000018000ecc8 f   libucrt:multibyte_initializer.obj
 0001:0000df40       $$000000                   000000018000ef40     libucrt:log10.obj
 0001:0000e4ec       ?write_double_translated_ansi_nolock@@YA?AUwrite_result@?A0x9c548279@@HQEBDI@Z 000000018000f4ec f   libucrt:write.obj
 0001:0000e6f4       ?write_text_ansi_nolock@@YA?AUwrite_result@?A0x9c548279@@HQEBDI@Z 000000018000f6f4 f   libucrt:write.obj
 0001:0000e7fc       ?write_text_utf16le_nolock@@YA?AUwrite_result@?A0x9c548279@@HQEBDI@Z 000000018000f7fc f   libucrt:write.obj
 0001:0000e918       ?write_text_utf8_nolock@@YA?AUwrite_result@?A0x9c548279@@HQEBDI@Z 000000018000f918 f   libucrt:write.obj
 0001:0000ee5c       ??$common_lseek_nolock@_J@@YA_JH_JH@Z 000000018000fe5c f   libucrt:lseek.obj
 0001:0000f248       common_control87           0000000180010248 f   libucrt:ieee.obj
 0001:0000f4e0       _call_matherr              00000001800104e0 f   libucrt:libm_error.obj
 0001:0000f548       _exception_enabled         0000000180010548 f   libucrt:libm_error.obj
 0001:0000f7e0       _log_special_common        00000001800107e0 f   libucrt:log_special.obj
 0001:0000faf0       $$000000                   0000000180010af0     libucrt:fpsr.obj
 0001:000100c0       $$000000                   00000001800110c0     LIBCMT:_chkstk_.obj
 0001:00010130       $$000000                   0000000180011130     libvcruntime:memcmp.obj
 0001:00010210       $$000000                   0000000180011210     LIBCMT:_guard_dispatch_.obj
 0001:00010230       ?fin$0@?0??dllmain_crt_process_attach@@YAHQEAUHINSTANCE__@@QEAX@Z@4HA 0000000180011230 f   LIBCMT:dll_dllmain.obj
 0001:00010247       ?fin$0@?0??dllmain_crt_process_detach@@YAH_N@Z@4HA 0000000180011247 f   LIBCMT:dll_dllmain.obj
 0001:00010263       ?filt$0@?0??dllmain_dispatch@@YAHQEAUHINSTANCE__@@KQEAX@Z@4HA 0000000180011263 f   LIBCMT:dll_dllmain.obj
 0001:00010299       __scrt_is_nonwritable_in_current_image$filt$0 0000000180011299 f   LIBCMT:utility.obj
 0001:000102b1       __DestructExceptionObject$filt$0 00000001800112b1 f   libvcruntime:ehhelpers.obj
 0001:000102c9       ?filt$0@?0??common_exit@@YAXHW4_crt_exit_cleanup_mode@@W4_crt_exit_return_mode@@@Z@4HA 00000001800112c9 f   libucrt:exit.obj
 0001:000102e4       ?fin$1@?0??common_exit@@YAXHW4_crt_exit_cleanup_mode@@W4_crt_exit_return_mode@@@Z@4HA 00000001800112e4 f   libucrt:exit.obj
 0001:000102fd       ?fin$0@?0???$?RV<lambda_e24bbb7b643b32fcea6fa61b31d4c984>@@AEAV<lambda_275893d493268fdec8709772e3fcec0e>@@V<lambda_9d71df4d7cf3f480f8d633942495c3b0>@@@?$__crt_seh_guarded_call@H@@QEAAH$$QEAV<lambda_e24bbb7b643b32fcea6fa61b31d4c984>@@AEAV<lambda_275893d493268fdec8709772e3fcec0e>@@$$QEAV<lambda_9d71df4d7cf3f480f8d633942495c3b0>@@@Z@4HA 00000001800112fd f   libucrt:onexit.obj
 0001:0001031a       ?fin$0@?0???$?RV<lambda_c36588078e9f5dfd39652860aa6b3aaf>@@AEAV<lambda_ec61778202f4f5fc7e7711acc23c3bca>@@V<lambda_dc9d2797ccde5d239b4a0efae8ebd7db>@@@?$__crt_seh_guarded_call@P6AXH@Z@@QEAAP6AXH@Z$$QEAV<lambda_c36588078e9f5dfd39652860aa6b3aaf>@@AEAV<lambda_ec61778202f4f5fc7e7711acc23c3bca>@@$$QEAV<lambda_dc9d2797ccde5d239b4a0efae8ebd7db>@@@Z@4HA 000000018001131a f   libucrt:signal.obj
 0001:0001031a       ?fin$0@?0???$?RV<lambda_fb3a7dec4e47f37f22dae91bb15c9095>@@AEAV<lambda_698284760c8add0bfb0756c19673e34b>@@V<lambda_dfb8eca1e75fef3034a8fb18dd509707>@@@?$__crt_seh_guarded_call@X@@QEAAX$$QEAV<lambda_fb3a7dec4e47f37f22dae91bb15c9095>@@AEAV<lambda_698284760c8add0bfb0756c19673e34b>@@$$QEAV<lambda_dfb8eca1e75fef3034a8fb18dd509707>@@@Z@4HA 000000018001131a f   libucrt:per_thread_data.obj
 0001:0001031a       ?fin$0@?0???$?RV<lambda_99476a1ad63dd22509b5d3e65b0ffc95>@@AEAV<lambda_ad1ced32f4ac17aa236e5ef05d6b3b7c>@@V<lambda_f7424dd8d45958661754dc4f2697e9c3>@@@?$__crt_seh_guarded_call@X@@QEAAX$$QEAV<lambda_99476a1ad63dd22509b5d3e65b0ffc95>@@AEAV<lambda_ad1ced32f4ac17aa236e5ef05d6b3b7c>@@$$QEAV<lambda_f7424dd8d45958661754dc4f2697e9c3>@@@Z@4HA 000000018001131a f   libucrt:mbctype.obj
 0001:0001031a       ?fin$0@?0???$?RV<lambda_46352004c1216016012b18bd6f87e700>@@AEAV<lambda_3bd07e1a1191394380780325891bf33f>@@V<lambda_334532d3f185bcaa59b5be82d7d22bff>@@@?$__crt_seh_guarded_call@X@@QEAAX$$QEAV<lambda_46352004c1216016012b18bd6f87e700>@@AEAV<lambda_3bd07e1a1191394380780325891bf33f>@@$$QEAV<lambda_334532d3f185bcaa59b5be82d7d22bff>@@@Z@4HA 000000018001131a f   libucrt:per_thread_data.obj
 0001:0001031a       ?fin$0@?0???$?RV<lambda_72d1df2b273a38828b1ce30cbf4cdab5>@@AEAV<lambda_876a65b173b8412d3a47c70a915b0cf4>@@V<lambda_41932305e351933ebe8f8be3ed8bb5dc>@@@?$__crt_seh_guarded_call@X@@QEAAX$$QEAV<lambda_72d1df2b273a38828b1ce30cbf4cdab5>@@AEAV<lambda_876a65b173b8412d3a47c70a915b0cf4>@@$$QEAV<lambda_41932305e351933ebe8f8be3ed8bb5dc>@@@Z@4HA 000000018001131a f   libucrt:per_thread_data.obj
 0001:0001031a       ?fin$0@?0???$?RV<lambda_5e887d1dcbef67a5eb4283622ba103bf>@@AEAV<lambda_4466841279450cc726390878d4a41900>@@V<lambda_341c25c0346d94847f1f3c463c57e077>@@@?$__crt_seh_guarded_call@X@@QEAAX$$QEAV<lambda_5e887d1dcbef67a5eb4283622ba103bf>@@AEAV<lambda_4466841279450cc726390878d4a41900>@@$$QEAV<lambda_341c25c0346d94847f1f3c463c57e077>@@@Z@4HA 000000018001131a f   libucrt:per_thread_data.obj
 0001:00010334       __acrt_update_thread_locale_data$fin$0 0000000180011334 f   libucrt:locale_refcounting.obj
 0001:00010334       __acrt_uninitialize_locale$fin$0 0000000180011334 f   libucrt:wsetlocale.obj
 0001:0001034d       __acrt_initialize_lowio$fin$0 000000018001134d f   libucrt:ioinit.obj
 0001:0001034d       __acrt_lowio_ensure_fh_exists$fin$0 000000018001134d f   libucrt:osfinfo.obj
 0001:00010366       __acrt_update_thread_multibyte_data$fin$0 0000000180011366 f   libucrt:mbctype.obj
 0001:0001037f       _query_new_handler$fin$0   000000018001137f f   libucrt:new_handler.obj
 0001:00010395       raise$fin$0                0000000180011395 f   libucrt:signal.obj
 0001:000103b9       _fcloseall$fin$0           00000001800113b9 f   libucrt:closeall.obj
 0001:000103d2       common_flush_all$fin$0     00000001800113d2 f   libucrt:fflush.obj
 0001:000103ec       common_flush_all$fin$1     00000001800113ec f   libucrt:fflush.obj
 0001:00010405       _write$fin$0               0000000180011405 f   libucrt:write.obj
 0001:0001041c       fclose$fin$0               000000018001141c f   libucrt:fclose.obj
 0001:00010434       ?fin$0@?0???$?RV<lambda_b521505b218e5242e90febf6bfebc422>@@AEAV<lambda_6978c1fb23f02e42e1d9e99668cc68aa>@@V<lambda_314360699dd331753a4119843814e9a7>@@@?$__crt_seh_guarded_call@H@@QEAAH$$QEAV<lambda_b521505b218e5242e90febf6bfebc422>@@AEAV<lambda_6978c1fb23f02e42e1d9e99668cc68aa>@@$$QEAV<lambda_314360699dd331753a4119843814e9a7>@@@Z@4HA 0000000180011434 f   libucrt:commit.obj
 0001:00010434       ?fin$0@?0???$?RV<lambda_bfedae4ebbf01fab1bb6dcc6a9e276e0>@@AEAV<lambda_2fe9b910cf3cbf4a0ab98a02ba45b3ec>@@V<lambda_237c231691f317818eb88cc1d5d642d6>@@@?$__crt_seh_guarded_call@H@@QEAAH$$QEAV<lambda_bfedae4ebbf01fab1bb6dcc6a9e276e0>@@AEAV<lambda_2fe9b910cf3cbf4a0ab98a02ba45b3ec>@@$$QEAV<lambda_237c231691f317818eb88cc1d5d642d6>@@@Z@4HA 0000000180011434 f   libucrt:close.obj
 0001:0001044e       common_control87$filt$0    000000018001144e f   libucrt:ieee.obj
 0001:0001044e       _ctrlfp$filt$0             000000018001144e f   libucrt:fpctrl.obj
 0001:00010480       _IsNonwritableInCurrentImage$filt$0 0000000180011480 f   LIBCMT:pesect.obj
 0002:00000630       GS_ExceptionPointers       0000000180012630     LIBCMT:gs_report.obj
 0002:00000650       ?tokenTable@@3QBQEBDB      0000000180012650     libvcruntime:undname.obj
 0002:000006c8       ?rttiTable@@3QBQEBDB       00000001800126c8     libvcruntime:undname.obj
 0002:000006f0       ?nameTable@@3QBQEBDB       00000001800126f0     libvcruntime:undname.obj
 0002:00000ff8       ?module_names@?A0x89697e75@@3QBQEB_WB 0000000180012ff8     libvcruntime:winapi_downlevel.obj
 0002:000010c8       ?candidate_modules@?1??try_get_FlsAlloc@@YAP6AKP6AXPEAX@Z@ZXZ@4QBW4module_id@?A0x89697e75@@B 00000001800130c8     libvcruntime:winapi_downlevel.obj
 0002:000010e0       ?candidate_modules@?1??try_get_FlsFree@@YAP6AHK@ZXZ@4QBW4module_id@?A0x89697e75@@B 00000001800130e0     libvcruntime:winapi_downlevel.obj
 0002:000010f0       ?candidate_modules@?1??try_get_FlsGetValue@@YAP6APEAXK@ZXZ@4QBW4module_id@?A0x89697e75@@B 00000001800130f0     libvcruntime:winapi_downlevel.obj
 0002:00001108       ?candidate_modules@?1??try_get_FlsSetValue@@YAP6AHKPEAX@ZXZ@4QBW4module_id@?A0x89697e75@@B 0000000180013108     libvcruntime:winapi_downlevel.obj
 0002:00001120       ?candidate_modules@?1??try_get_InitializeCriticalSectionEx@@YAP6AHPEAU_RTL_CRITICAL_SECTION@@KK@ZXZ@4QBW4module_id@?A0x89697e75@@B 0000000180013120     libvcruntime:winapi_downlevel.obj
 0002:000012d0       __acrt_initializers        00000001800132d0     libucrt:initialization.obj
 0002:000013c0       errtable                   00000001800133c0     libucrt:errno.obj
 0002:00001c00       module_names               0000000180013c00     libucrt:winapi_thunks.obj
 0002:00002148       ?candidate_modules@?1??try_get_FlsAlloc@@YAP6AKP6AXPEAX@Z@ZXZ@4QBW4module_id@?A0x63058377@@B 0000000180014148     libucrt:winapi_thunks.obj
 0002:00002150       ?candidate_modules@?1??try_get_FlsFree@@YAP6AHK@ZXZ@4QBW4module_id@?A0x63058377@@B 0000000180014150     libucrt:winapi_thunks.obj
 0002:00002158       ?candidate_modules@?1??try_get_FlsGetValue@@YAP6APEAXK@ZXZ@4QBW4module_id@?A0x63058377@@B 0000000180014158     libucrt:winapi_thunks.obj
 0002:00002160       ?candidate_modules@?1??try_get_FlsSetValue@@YAP6AHKPEAX@ZXZ@4QBW4module_id@?A0x63058377@@B 0000000180014160     libucrt:winapi_thunks.obj
 0002:00002168       ?candidate_modules@?1??try_get_GetCurrentPackageId@@YAP6AJPEAIPEAE@ZXZ@4QBW4module_id@?A0x63058377@@B 0000000180014168     libucrt:winapi_thunks.obj
 0002:00002188       ?candidate_modules@?1??try_get_InitializeCriticalSectionEx@@YAP6AHPEAU_RTL_CRITICAL_SECTION@@KK@ZXZ@4QBW4module_id@?A0x63058377@@B 0000000180014188     libucrt:winapi_thunks.obj
 0002:00002190       ?candidate_modules@?1??try_get_LCMapStringEx@@YAP6AHPEB_WK0HPEA_WHPEAU_nlsversioninfo@@PEAX_J@ZXZ@4QBW4module_id@?A0x63058377@@B 0000000180014190     libucrt:winapi_thunks.obj
 0002:000021a8       ?candidate_modules@?1??try_get_LocaleNameToLCID@@YAP6AKPEB_WK@ZXZ@4QBW4module_id@?A0x63058377@@B 00000001800141a8     libucrt:winapi_thunks.obj
 0002:000021c8       _mb_locale_names           00000001800141c8     libucrt:mbctype.obj
 0002:00003230       LcidToLocaleNameTable      0000000180015230     libucrt:lcidtoname_downlevel.obj
 0002:00004c90       LocaleNameToIndexTable     0000000180016c90     libucrt:lcidtoname_downlevel.obj
 0002:00006530       __real_ninf                0000000180018530     libucrt:log10.obj
 0002:00006540       __real_inf                 0000000180018540     libucrt:log10.obj
 0002:00006550       __real_neg_qnan            0000000180018550     libucrt:log10.obj
 0002:00006560       __real_qnanbit             0000000180018560     libucrt:log10.obj
 0002:00006570       __int_1023                 0000000180018570     libucrt:log10.obj
 0002:00006580       __mask_001                 0000000180018580     libucrt:log10.obj
 0002:00006590       __mask_mant                0000000180018590     libucrt:log10.obj
 0002:000065a0       __mask_mant_top8           00000001800185a0     libucrt:log10.obj
 0002:000065b0       __mask_mant9               00000001800185b0     libucrt:log10.obj
 0002:000065c0       __real_log10_e             00000001800185c0     libucrt:log10.obj
 0002:000065d0       __real_log10_e_lead        00000001800185d0     libucrt:log10.obj
 0002:000065e0       __real_log10_e_tail        00000001800185e0     libucrt:log10.obj
 0002:000065f0       __real_log10_2_lead        00000001800185f0     libucrt:log10.obj
 0002:00006600       __real_log10_2_tail        0000000180018600     libucrt:log10.obj
 0002:00006610       __real_two                 0000000180018610     libucrt:log10.obj
 0002:00006620       __real_one                 0000000180018620     libucrt:log10.obj
 0002:00006630       __real_half                0000000180018630     libucrt:log10.obj
 0002:00006640       __mask_100                 0000000180018640     libucrt:log10.obj
 0002:00006650       __real_1_over_512          0000000180018650     libucrt:log10.obj
 0002:00006660       __real_1_over_2            0000000180018660     libucrt:log10.obj
 0002:00006670       __real_1_over_3            0000000180018670     libucrt:log10.obj
 0002:00006680       __real_1_over_4            0000000180018680     libucrt:log10.obj
 0002:00006690       __real_1_over_5            0000000180018690     libucrt:log10.obj
 0002:000066a0       __real_1_over_6            00000001800186a0     libucrt:log10.obj
 0002:000066b0       __real_neg_1023            00000001800186b0     libucrt:log10.obj
 0002:000066c0       __mask_2045                00000001800186c0     libucrt:log10.obj
 0002:000066d0       __real_threshold           00000001800186d0     libucrt:log10.obj
 0002:000066e0       __real_near_one_lt         00000001800186e0     libucrt:log10.obj
 0002:000066f0       __real_near_one_gt         00000001800186f0     libucrt:log10.obj
 0002:00006700       __real_min_norm            0000000180018700     libucrt:log10.obj
 0002:00006710       __real_notsign             0000000180018710     libucrt:log10.obj
 0002:00006720       __real_ca1                 0000000180018720     libucrt:log10.obj
 0002:00006730       __real_ca2                 0000000180018730     libucrt:log10.obj
 0002:00006740       __real_ca3                 0000000180018740     libucrt:log10.obj
 0002:00006750       __real_ca4                 0000000180018750     libucrt:log10.obj
 0002:00006760       __mask_lower               0000000180018760     libucrt:log10.obj
 0002:00006770       __flag_x_zero              0000000180018770     libucrt:log10.obj
 0002:00006774       __flag_x_neg               0000000180018774     libucrt:log10.obj
 0002:00006778       __flag_x_nan               0000000180018778     libucrt:log10.obj
 0002:00007fc0       __real@433fffffffffffff    0000000180019fc0     libucrt:fpsr.obj
 0002:00007fc8       __real@c33fffffffffffff    0000000180019fc8     libucrt:fpsr.obj
 0002:00008460       $unwind$?Init@GDIPlusDecoder@@QEAA_NPEAUCET_Init@@@Z 000000018001a460     gdip.obj
 0002:00008478       $unwind$__vcrt_initialize_ptd 000000018001a478     libvcruntime:per_thread_data.obj
 0002:00008478       $unwind$__acrt_uninitialize_critical 000000018001a478     libucrt:initialization.obj
 0002:00008478       $unwind$?dllmain_crt_dispatch@@YAHQEAUHINSTANCE__@@KQEAX@Z 000000018001a478     LIBCMT:dll_dllmain.obj
 0002:00008478       $unwind$?HeapInitialize@@YA_NXZ 000000018001a478     common-kernel64:Memory.obj
 0002:00008478       $unwind$__dcrt_uninitialize_environments_nolock 000000018001a478     libucrt:environment_initialization.obj
 0002:00008478       $unwind$__scrt_initialize_default_local_stdio_options 000000018001a478     LIBCMT:default_local_stdio_options.obj
 0002:00008478       $unwind$_getfpcontrolword  000000018001a478     libucrt:_fenvutils.obj
 0002:00008478       $unwind$?HeapDeinitialize@@YAXXZ 000000018001a478     common-kernel64:Memory.obj
 0002:00008478       $unwind$_get_osfhandle     000000018001a478     libucrt:osfinfo.obj
 0002:00008478       $unwind$??_V@YAXPEAX@Z     000000018001a478     common-kernel64:Memory.obj
 0002:00008478       $unwind$?state_case_size@?$output_processor@DV?$string_output_adapter@D@__crt_stdio_output@@V?$standard_base@DV?$string_output_adapter@D@__crt_stdio_output@@@2@@__crt_stdio_output@@AEAA_NXZ 000000018001a478     libucrt:output.obj
 0002:00008478       $unwind$__doserrno         000000018001a478     libucrt:errno.obj
 0002:00008478       $unwind$?FreeThreadProc@GDIPlusDecoder@@SAKPEAX@Z 000000018001a478     gdip.obj
 0002:00008478       $unwind$__vcrt_freefls     000000018001a478     libvcruntime:per_thread_data.obj
 0002:00008478       $unwind$__acrt_initialize_heap 000000018001a478     libucrt:heap_handle.obj
 0002:00008478       $unwind$_errno             000000018001a478     libucrt:errno.obj
 0002:00008478       $unwind$__vcrt_uninitialize_ptd 000000018001a478     libvcruntime:per_thread_data.obj
 0002:00008478       $unwind$?state_case_normal_tchar@?$output_processor@DV?$string_output_adapter@D@__crt_stdio_output@@V?$standard_base@DV?$string_output_adapter@D@__crt_stdio_output@@@2@@__crt_stdio_output@@AEAA_ND@Z 000000018001a478     libucrt:output.obj
 0002:00008478       $unwind$__pctype_func      000000018001a478     libucrt:ctype.obj
 0002:00008478       $unwind$__scrt_dllmain_before_initialize_c 000000018001a478     LIBCMT:utility.obj
 0002:00008478       $unwind$_getfpstatusword   000000018001a478     libucrt:_fenvutils.obj
 0002:00008478       $unwind$__acrt_thread_attach 000000018001a478     libucrt:initialization.obj
 0002:00008478       $unwind$_isatty            000000018001a478     libucrt:isatty.obj
 0002:00008478       $unwind$__scrt_dllmain_after_initialize_c 000000018001a478     LIBCMT:utility.obj
 0002:00008478       $unwind$abort              000000018001a478     libucrt:abort.obj
 0002:00008478       $unwind$__dcrt_terminate_console_output 000000018001a478     libucrt:initcon.obj
 0002:00008478       $unwind$__acrt_initialize_command_line 000000018001a478     libucrt:argv_data.obj
 0002:00008478       $unwind$__scrt_dllmain_uninitialize_c 000000018001a478     LIBCMT:utility.obj
 0002:00008478       $unwind$__acrt_initialize_multibyte 000000018001a478     libucrt:mbctype.obj
 0002:00008478       $unwind$__acrt_thread_detach 000000018001a478     libucrt:initialization.obj
 0002:00008478       $unwind$__vcrt_thread_detach 000000018001a478     libvcruntime:initialization.obj
 0002:00008478       $unwind$__scrt_dllmain_uninitialize_critical 000000018001a478     LIBCMT:utility.obj
 0002:00008478       $unwind$__vcrt_thread_attach 000000018001a478     libvcruntime:initialization.obj
 0002:00008478       $unwind$?initialize_multibyte@@YAHXZ 000000018001a478     libucrt:multibyte_initializer.obj
 0002:00008478       $unwind$_invoke_watson     000000018001a478     libucrt:invalid_parameter.obj
 0002:00008478       $unwind$__scrt_dllmain_crt_thread_attach 000000018001a478     LIBCMT:utility.obj
 0002:00008478       $unwind$__acrt_DownlevelLocaleNameToLCID 000000018001a478     libucrt:lcidtoname_downlevel.obj
 0002:00008478       $unwind$??3@YAXPEAX@Z      000000018001a478     common-kernel64:Memory.obj
 0002:00008478       $unwind$__scrt_dllmain_crt_thread_detach 000000018001a478     LIBCMT:utility.obj
 0002:00008478       $unwind$??$uninitialize_environment_internal@D@@YAXAEAPEAPEAD@Z 000000018001a478     libucrt:environment_initialization.obj
 0002:00008478       $unwind$initialize_c       000000018001a478     libucrt:initialization.obj
 0002:00008478       $unwind$_set_errno_from_matherr 000000018001a478     libucrt:fpexcept.obj
 0002:00008478       $unwind$uninitialize_environment 000000018001a478     libucrt:initialization.obj
 0002:00008478       $unwind$__vcrt_uninitialize_critical 000000018001a478     libvcruntime:initialization.obj
 0002:00008478       $unwind$?CET_Done@@YAXPEAUCET_Init@@@Z 000000018001a478     gdip.obj
 0002:00008478       $unwind$__vcrt_uninitialize 000000018001a478     libvcruntime:initialization.obj
 0002:00008478       $unwind$tolower            000000018001a478     libucrt:tolower_toupper.obj
 0002:00008478       $unwind$__vcrt_initialize  000000018001a478     libvcruntime:initialization.obj
 0002:00008478       $unwind$__acrt_initialize_ptd 000000018001a478     libucrt:per_thread_data.obj
 0002:00008478       $unwind$__scrt_acquire_startup_lock 000000018001a478     LIBCMT:utility.obj
 0002:00008478       $unwind$__acrt_release_locale_ref 000000018001a478     libucrt:locale_refcounting.obj
 0002:00008478       $unwind$__report_rangecheckfailure 000000018001a478     LIBCMT:gs_report.obj
 0002:00008478       $unwind$__GSHandlerCheck   000000018001a478     LIBCMT:_gshandler_.obj
 0002:00008478       $unwind$_fileno            000000018001a478     libucrt:fileno.obj
 0002:00008478       $unwind$??$uninitialize_environment_internal@_W@@YAXAEAPEAPEA_W@Z 000000018001a478     libucrt:environment_initialization.obj
 0002:00008478       $unwind$_msize             000000018001a478     libucrt:msize.obj
 0002:00008478       $unwind$??2@YAPEAX_K@Z     000000018001a478     common-kernel64:Memory.obj
 0002:00008478       $unwind$__acrt_uninitialize_ptd 000000018001a478     libucrt:per_thread_data.obj
 0002:00008478       $unwind$_statfp            000000018001a478     libucrt:fpctrl.obj
 0002:00008480       $unwind$?Close@GDIPlusDecoder@@QEAAXXZ 000000018001a480     gdip.obj
 0002:0000848c       $unwind$?Open@GDIPlusImage@@QEAA_N_NPEB_WPEBE_JU_COORD@@@Z 000000018001a48c     gdip.obj
 0002:000084b0       $unwind$__acrt_LocaleNameToLCID 000000018001a4b0     libucrt:winapi_thunks.obj
 0002:000084b0       $unwind$__acrt_execute_uninitializers 000000018001a4b0     libucrt:shared_initialization.obj
 0002:000084b0       $unwind$__acrt_FlsSetValue 000000018001a4b0     libucrt:winapi_thunks.obj
 0002:000084b0       $unwind$_exception_enabled 000000018001a4b0     libucrt:libm_error.obj
 0002:000084b0       $unwind$_DllMainCRTStartup 000000018001a4b0     LIBCMT:dll_dllmain.obj
 0002:000084b0       $unwind$memcpy_s           000000018001a4b0     libucrt:cfout.obj
 0002:000084b0       $unwind$_initterm_e        000000018001a4b0     libucrt:initterm.obj
 0002:000084b0       $unwind$?type_case_Z@?$output_processor@DV?$string_output_adapter@D@__crt_stdio_output@@V?$standard_base@DV?$string_output_adapter@D@__crt_stdio_output@@@2@@__crt_stdio_output@@AEAA_NXZ 000000018001a4b0     libucrt:output.obj
 0002:000084b0       $unwind$??R<lambda_ad1ced32f4ac17aa236e5ef05d6b3b7c>@@QEBAXXZ 000000018001a4b0     libucrt:mbctype.obj
 0002:000084b0       $unwind$?type_case_s@?$output_processor@DV?$string_output_adapter@D@__crt_stdio_output@@V?$standard_base@DV?$string_output_adapter@D@__crt_stdio_output@@@2@@__crt_stdio_output@@AEAA_NXZ 000000018001a4b0     libucrt:output.obj
 0002:000084b0       $unwind$?free_crt_array_internal@@YAXQEAPEBX_K@Z 000000018001a4b0     libucrt:inittime.obj
 0002:000084b0       $unwind$__vcrt_getptd_noexit 000000018001a4b0     libvcruntime:per_thread_data.obj
 0002:000084b0       $unwind$__acrt_getptd_noexit 000000018001a4b0     libucrt:per_thread_data.obj
 0002:000084b0       $unwind$__acrt_stdio_flush_nolock 000000018001a4b0     libucrt:fflush.obj
 0002:000084b0       $unwind$__vcrt_InitializeCriticalSectionEx 000000018001a4b0     libvcruntime:winapi_downlevel.obj
 0002:000084b0       $unwind$?SelectPage@GDIPlusImage@@QEAA_NI@Z 000000018001a4b0     gdip.obj
 0002:000084b0       $unwind$??$common_lseek_nolock@_J@@YA_JH_JH@Z 000000018001a4b0     libucrt:lseek.obj
 0002:000084b0       $unwind$?type_case_n@?$output_processor@DV?$string_output_adapter@D@__crt_stdio_output@@V?$standard_base@DV?$string_output_adapter@D@__crt_stdio_output@@@2@@__crt_stdio_output@@AEAA_NXZ 000000018001a4b0     libucrt:output.obj
 0002:000084c0       $unwind$?force_decimal_point@__crt_stdio_output@@YAXPEADQEAU__crt_locale_pointers@@@Z 000000018001a4c0     libucrt:output.obj
 0002:000084c0       $unwind$?CET_Init@@YAHPEAU0@@Z 000000018001a4c0     gdip.obj
 0002:000084c0       $unwind$?type_case_c_tchar@?$output_processor@DV?$string_output_adapter@D@__crt_stdio_output@@V?$standard_base@DV?$string_output_adapter@D@__crt_stdio_output@@@2@@__crt_stdio_output@@AEAA_ND@Z 000000018001a4c0     libucrt:output.obj
 0002:000084c0       $unwind$strncpy_s          000000018001a4c0     libucrt:strncpy_s.obj
 0002:000084c0       $unwind$__acrt_invoke_user_matherr 000000018001a4c0     libucrt:matherr.obj
 0002:000084c0       $unwind$??$common_initialize_environment_nolock@D@@YAHXZ 000000018001a4c0     libucrt:environment_initialization.obj
 0002:000084c0       $unwind$_fclose_nolock     000000018001a4c0     libucrt:fclose.obj
 0002:000084c0       $unwind$?Close@GDIPlusImage@@QEAAXXZ 000000018001a4c0     gdip.obj
 0002:000084c0       $unwind$??0_LocaleUpdate@@QEAA@QEAU__crt_locale_pointers@@@Z 000000018001a4c0     libucrt:output.obj
 0002:000084c0       $unwind$_RTC_Initialize    000000018001a4c0     LIBCMT:_initsect_.obj
 0002:000084c0       $unwind$__acrt_errno_map_os_error 000000018001a4c0     libucrt:errno.obj
 0002:000084c0       $unwind$_RTC_Terminate     000000018001a4c0     LIBCMT:_initsect_.obj
 0002:000084c0       $unwind$_close_nolock      000000018001a4c0     libucrt:close.obj
 0002:000084c0       $unwind$__acrt_uninitialize_lowio 000000018001a4c0     libucrt:ioinit.obj
 0002:000084c0       $unwind$__acrt_FlsAlloc    000000018001a4c0     libucrt:winapi_thunks.obj
 0002:000084c0       $unwind$__acrt_getptd      000000018001a4c0     libucrt:per_thread_data.obj
 0002:000084c0       $unwind$?replace_current_thread_locale_nolock@@YAXQEAU__acrt_ptd@@QEAU__crt_locale_data@@@Z 000000018001a4c0     libucrt:per_thread_data.obj
 0002:000084c0       $unwind$_updatetlocinfoEx_nolock 000000018001a4c0     libucrt:locale_refcounting.obj
 0002:000084c0       $unwind$_callnewh          000000018001a4c0     libucrt:new_handler.obj
 0002:000084c0       $unwind$__acrt_FlsGetValue 000000018001a4c0     libucrt:winapi_thunks.obj
 0002:000084c0       $unwind$?try_cor_exit_process@@YAXI@Z 000000018001a4c0     libucrt:exit.obj
 0002:000084c0       $unwind$__vcrt_FlsSetValue 000000018001a4c0     libvcruntime:winapi_downlevel.obj
 0002:000084c0       $unwind$?internal_isupper_l@@YA_NHQEAU__crt_locale_pointers@@@Z 000000018001a4c0     libucrt:tolower_toupper.obj
 0002:000084c0       $unwind$__acrt_FlsFree     000000018001a4c0     libucrt:winapi_thunks.obj
 0002:000084c0       $unwind$_realloc_base      000000018001a4c0     libucrt:realloc_base.obj
 0002:000084cc       $unwind$?GetExifTagValueAsInt@GDIPlusImage@@QEAA_NKAEAH@Z 000000018001a4cc     gdip.obj
 0002:000084e0       $unwind$?GetTableIndexFromLocaleName@@YAHPEB_W@Z 000000018001a4e0     libucrt:lcidtoname_downlevel.obj
 0002:000084e0       $unwind$?CalculateShowSize@GDIPlusImage@@QEAAXAEAH0000@Z 000000018001a4e0     gdip.obj
 0002:000084f8       $unwind$?GetPageBits@GDIPlusImage@@QEAA_NPEAUCET_LoadInfo@@@Z 000000018001a4f8     gdip.obj
 0002:0000851c       $unwind$?CET_Load@@YAHPEAUCET_LoadInfo@@@Z 000000018001a51c     gdip.obj
 0002:00008538       $unwind$?CET_Free@@YAXPEAUCET_LoadInfo@@@Z 000000018001a538     gdip.obj
 0002:00008538       $unwind$__acrt_locale_free_monetary 000000018001a538     libucrt:initmon.obj
 0002:00008540       $unwind$?StringCchVPrintfA@@YAJPEAD_KPEBD0@Z 000000018001a540     common-kernel64:WThreads.obj
 0002:00008540       $unwind$_invalid_parameter 000000018001a540     libucrt:invalid_parameter.obj
 0002:00008540       $unwind$?apiCreateThread@@YAPEAXP6AKPEAX@Z0PEAKPEBDH@Z 000000018001a540     common-kernel64:WThreads.obj
 0002:00008558       $unwind$?apiTerminateThreadEx@@YAHPEAXKPEBDH@Z 000000018001a558     common-kernel64:WThreads.obj
 0002:00008574       $unwind$?SetThreadName@@YAXKPEAD@Z 000000018001a574     common-kernel64:WThreads.obj
 0002:00008594       $unwind$?apiThreadHelper@@YAKPEAX@Z 000000018001a594     common-kernel64:WThreads.obj
 0002:000085a8       $unwind$??$sprintf_c@$0CI@@@YAHAEAY0CI@DPEBDZZ 000000018001a5a8     common-kernel64:WThreads.obj
 0002:000085b0       $unwind$?sprintf_c@@YAHPEAD_JPEBDZZ 000000018001a5b0     common-kernel64:MStrSafe.obj
 0002:000085bc       $unwind$__report_securityfailure 000000018001a5bc     LIBCMT:gs_report.obj
 0002:000085c4       $unwind$__report_gsfailure 000000018001a5c4     LIBCMT:gs_report.obj
 0002:000085c4       $unwind$_putwch_nolock     000000018001a5c4     libucrt:putwch.obj
 0002:000085cc       $unwind$capture_current_context 000000018001a5cc     LIBCMT:gs_report.obj
 0002:000085d8       $unwind$capture_previous_context 000000018001a5d8     LIBCMT:gs_report.obj
 0002:000085e4       $unwind$__std_type_info_destroy_list 000000018001a5e4     libvcruntime:std_type_info.obj
 0002:000085e4       $unwind$uninitialize_allocated_memory 000000018001a5e4     libucrt:initialization.obj
 0002:000085e4       $unwind$initialize_pointers 000000018001a5e4     libucrt:initialization.obj
 0002:000085e4       $unwind$__acrt_initialize_locks 000000018001a5e4     libucrt:locks.obj
 0002:000085e4       $unwind$__acrt_fp_strflt_to_string 000000018001a5e4     libucrt:_fptostr.obj
 0002:000085e4       $unwind$__acrt_uninitialize_stdio 000000018001a5e4     libucrt:_file.obj
 0002:000085e4       $unwind$__acrt_uninitialize_winapi_thunks 000000018001a5e4     libucrt:winapi_thunks.obj
 0002:000085e4       $unwind$fegetenv           000000018001a5e4     libucrt:fegetenv.obj
 0002:000085e4       $unwind$__acrt_uninitialize_locks 000000018001a5e4     libucrt:locks.obj
 0002:000085e4       $unwind$__vcrt_FlsGetValue 000000018001a5e4     libvcruntime:winapi_downlevel.obj
 0002:000085e4       $unwind$__acrt_allocate_buffer_for_argv 000000018001a5e4     libucrt:argv_parsing.obj
 0002:000085e4       $unwind$_fflush_nolock     000000018001a5e4     libucrt:fflush.obj
 0002:000085e4       $unwind$__vcrt_freeptd     000000018001a5e4     libvcruntime:per_thread_data.obj
 0002:000085e4       $unwind$_setfpstatusword   000000018001a5e4     libucrt:_fenvutils.obj
 0002:000085e4       $unwind$__vcrt_initialize_locks 000000018001a5e4     libvcruntime:locks.obj
 0002:000085e4       $unwind$__vcrt_uninitialize_locks 000000018001a5e4     libvcruntime:locks.obj
 0002:000085e4       $unwind$__raise_securityfailure 000000018001a5e4     LIBCMT:gs_report.obj
 0002:000085e4       $unwind$__acrt_update_multibyte_info 000000018001a5e4     libucrt:locale_update.obj
 0002:000085e4       $unwind$_clearfp           000000018001a5e4     libucrt:ieee.obj
 0002:000085e4       $unwind$__vcrt_FlsAlloc    000000018001a5e4     libvcruntime:winapi_downlevel.obj
 0002:000085e4       $unwind$__acrt_stdio_free_buffer_nolock 000000018001a5e4     libucrt:_freebuf.obj
 0002:000085e4       $unwind$_calloc_base       000000018001a5e4     libucrt:calloc_base.obj
 0002:000085e4       $unwind$?exit_or_terminate_process@@YAXI@Z 000000018001a5e4     libucrt:exit.obj
 0002:000085e4       $unwind$fesetenv           000000018001a5e4     libucrt:fesetenv.obj
 0002:000085e4       $unwind$feholdexcept       000000018001a5e4     libucrt:feholdexcept.obj
 0002:000085e4       $unwind$?type_case_integer@?$output_processor@DV?$string_output_adapter@D@__crt_stdio_output@@V?$standard_base@DV?$string_output_adapter@D@__crt_stdio_output@@@2@@__crt_stdio_output@@AEAA_NI_N@Z 000000018001a5e4     libucrt:output.obj
 0002:000085e4       $unwind$??0?$output_processor@DV?$string_output_adapter@D@__crt_stdio_output@@V?$standard_base@DV?$string_output_adapter@D@__crt_stdio_output@@@2@@__crt_stdio_output@@QEAA@AEBV?$string_output_adapter@D@1@_KQEBDQEAU__crt_locale_pointers@@QEAD@Z 000000018001a5e4     libucrt:output.obj
 0002:000085e4       $unwind$_set_statfp        000000018001a5e4     libucrt:fpctrl.obj
 0002:000085e4       $unwind$strcpy_s           000000018001a5e4     libucrt:strcpy_s.obj
 0002:000085e4       $unwind$?state_case_normal@?$output_processor@DV?$string_output_adapter@D@__crt_stdio_output@@V?$standard_base@DV?$string_output_adapter@D@__crt_stdio_output@@@2@@__crt_stdio_output@@AEAA_NXZ 000000018001a5e4     libucrt:output.obj
 0002:000085e4       $unwind$__vcrt_FlsFree     000000018001a5e4     libvcruntime:winapi_downlevel.obj
 0002:000085e4       $unwind$__acrt_freeptd     000000018001a5e4     libucrt:per_thread_data.obj
 0002:000085e4       $unwind$_clrfp             000000018001a5e4     libucrt:fpctrl.obj
 0002:000085e4       $unwind$__scrt_uninitialize_crt 000000018001a5e4     LIBCMT:utility.obj
 0002:000085e4       $unwind$__acrt_update_locale_info 000000018001a5e4     libucrt:locale_update.obj
 0002:000085e4       $unwind$_malloc_base       000000018001a5e4     libucrt:malloc_base.obj
 0002:000085e4       $unwind$__scrt_initialize_crt 000000018001a5e4     LIBCMT:utility.obj
 0002:000085e4       $unwind$__scrt_release_startup_lock 000000018001a5e4     LIBCMT:utility.obj
 0002:000085ec       $unwind$__GSHandlerCheckCommon 000000018001a5ec     LIBCMT:_gshandler_.obj
 0002:000085f8       $xdatasym                  000000018001a5f8     LIBCMT:_amdsecgs_.obj
 0002:000085fc       $unwind$?dllmain_crt_process_attach@@YAHQEAUHINSTANCE__@@QEAX@Z 000000018001a5fc     LIBCMT:dll_dllmain.obj
 0002:00008638       $unwind$_ctrlfp$filt$0     000000018001a638     libucrt:fpctrl.obj
 0002:00008638       $unwind$__acrt_uninitialize_locale$fin$0 000000018001a638     libucrt:wsetlocale.obj
 0002:00008638       $unwind$_write$fin$0       000000018001a638     libucrt:write.obj
 0002:00008638       $unwind$common_flush_all$fin$1 000000018001a638     libucrt:fflush.obj
 0002:00008638       $unwind$common_control87$filt$0 000000018001a638     libucrt:ieee.obj
 0002:00008638       $unwind$?fin$0@?0??dllmain_crt_process_detach@@YAH_N@Z@4HA 000000018001a638     LIBCMT:dll_dllmain.obj
 0002:00008638       $unwind$__acrt_update_thread_multibyte_data$fin$0 000000018001a638     libucrt:mbctype.obj
 0002:00008638       $unwind$common_flush_all$fin$0 000000018001a638     libucrt:fflush.obj
 0002:00008638       $unwind$fclose$fin$0       000000018001a638     libucrt:fclose.obj
 0002:00008638       $unwind$_fcloseall$fin$0   000000018001a638     libucrt:closeall.obj
 0002:00008638       $unwind$?fin$0@?0???$?RV<lambda_bfedae4ebbf01fab1bb6dcc6a9e276e0>@@AEAV<lambda_2fe9b910cf3cbf4a0ab98a02ba45b3ec>@@V<lambda_237c231691f317818eb88cc1d5d642d6>@@@?$__crt_seh_guarded_call@H@@QEAAH$$QEAV<lambda_bfedae4ebbf01fab1bb6dcc6a9e276e0>@@AEAV<lambda_2fe9b910cf3cbf4a0ab98a02ba45b3ec>@@$$QEAV<lambda_237c231691f317818eb88cc1d5d642d6>@@@Z@4HA 000000018001a638     libucrt:close.obj
 0002:00008638       $unwind$__acrt_lowio_ensure_fh_exists$fin$0 000000018001a638     libucrt:osfinfo.obj
 0002:00008638       $unwind$?fin$0@?0???$?RV<lambda_b521505b218e5242e90febf6bfebc422>@@AEAV<lambda_6978c1fb23f02e42e1d9e99668cc68aa>@@V<lambda_314360699dd331753a4119843814e9a7>@@@?$__crt_seh_guarded_call@H@@QEAAH$$QEAV<lambda_b521505b218e5242e90febf6bfebc422>@@AEAV<lambda_6978c1fb23f02e42e1d9e99668cc68aa>@@$$QEAV<lambda_314360699dd331753a4119843814e9a7>@@@Z@4HA 000000018001a638     libucrt:commit.obj
 0002:00008638       $unwind$?fin$0@?0???$?RV<lambda_46352004c1216016012b18bd6f87e700>@@AEAV<lambda_3bd07e1a1191394380780325891bf33f>@@V<lambda_334532d3f185bcaa59b5be82d7d22bff>@@@?$__crt_seh_guarded_call@X@@QEAAX$$QEAV<lambda_46352004c1216016012b18bd6f87e700>@@AEAV<lambda_3bd07e1a1191394380780325891bf33f>@@$$QEAV<lambda_334532d3f185bcaa59b5be82d7d22bff>@@@Z@4HA 000000018001a638     libucrt:per_thread_data.obj
 0002:00008638       $unwind$?fin$0@?0??dllmain_crt_process_attach@@YAHQEAUHINSTANCE__@@QEAX@Z@4HA 000000018001a638     LIBCMT:dll_dllmain.obj
 0002:00008638       $unwind$?fin$0@?0???$?RV<lambda_e24bbb7b643b32fcea6fa61b31d4c984>@@AEAV<lambda_275893d493268fdec8709772e3fcec0e>@@V<lambda_9d71df4d7cf3f480f8d633942495c3b0>@@@?$__crt_seh_guarded_call@H@@QEAAH$$QEAV<lambda_e24bbb7b643b32fcea6fa61b31d4c984>@@AEAV<lambda_275893d493268fdec8709772e3fcec0e>@@$$QEAV<lambda_9d71df4d7cf3f480f8d633942495c3b0>@@@Z@4HA 000000018001a638     libucrt:onexit.obj
 0002:00008638       $unwind$?fin$0@?0???$?RV<lambda_fb3a7dec4e47f37f22dae91bb15c9095>@@AEAV<lambda_698284760c8add0bfb0756c19673e34b>@@V<lambda_dfb8eca1e75fef3034a8fb18dd509707>@@@?$__crt_seh_guarded_call@X@@QEAAX$$QEAV<lambda_fb3a7dec4e47f37f22dae91bb15c9095>@@AEAV<lambda_698284760c8add0bfb0756c19673e34b>@@$$QEAV<lambda_dfb8eca1e75fef3034a8fb18dd509707>@@@Z@4HA 000000018001a638     libucrt:per_thread_data.obj
 0002:00008638       $unwind$__acrt_update_thread_locale_data$fin$0 000000018001a638     libucrt:locale_refcounting.obj
 0002:00008638       $unwind$?fin$1@?0??common_exit@@YAXHW4_crt_exit_cleanup_mode@@W4_crt_exit_return_mode@@@Z@4HA 000000018001a638     libucrt:exit.obj
 0002:00008638       $unwind$__DestructExceptionObject$filt$0 000000018001a638     libvcruntime:ehhelpers.obj
 0002:00008638       $unwind$?fin$0@?0???$?RV<lambda_5e887d1dcbef67a5eb4283622ba103bf>@@AEAV<lambda_4466841279450cc726390878d4a41900>@@V<lambda_341c25c0346d94847f1f3c463c57e077>@@@?$__crt_seh_guarded_call@X@@QEAAX$$QEAV<lambda_5e887d1dcbef67a5eb4283622ba103bf>@@AEAV<lambda_4466841279450cc726390878d4a41900>@@$$QEAV<lambda_341c25c0346d94847f1f3c463c57e077>@@@Z@4HA 000000018001a638     libucrt:per_thread_data.obj
 0002:00008638       $unwind$?fin$0@?0???$?RV<lambda_99476a1ad63dd22509b5d3e65b0ffc95>@@AEAV<lambda_ad1ced32f4ac17aa236e5ef05d6b3b7c>@@V<lambda_f7424dd8d45958661754dc4f2697e9c3>@@@?$__crt_seh_guarded_call@X@@QEAAX$$QEAV<lambda_99476a1ad63dd22509b5d3e65b0ffc95>@@AEAV<lambda_ad1ced32f4ac17aa236e5ef05d6b3b7c>@@$$QEAV<lambda_f7424dd8d45958661754dc4f2697e9c3>@@@Z@4HA 000000018001a638     libucrt:mbctype.obj
 0002:00008638       $unwind$?filt$0@?0??common_exit@@YAXHW4_crt_exit_cleanup_mode@@W4_crt_exit_return_mode@@@Z@4HA 000000018001a638     libucrt:exit.obj
 0002:00008638       $unwind$?fin$0@?0???$?RV<lambda_c36588078e9f5dfd39652860aa6b3aaf>@@AEAV<lambda_ec61778202f4f5fc7e7711acc23c3bca>@@V<lambda_dc9d2797ccde5d239b4a0efae8ebd7db>@@@?$__crt_seh_guarded_call@P6AXH@Z@@QEAAP6AXH@Z$$QEAV<lambda_c36588078e9f5dfd39652860aa6b3aaf>@@AEAV<lambda_ec61778202f4f5fc7e7711acc23c3bca>@@$$QEAV<lambda_dc9d2797ccde5d239b4a0efae8ebd7db>@@@Z@4HA 000000018001a638     libucrt:signal.obj
 0002:00008638       $unwind$raise$fin$0        000000018001a638     libucrt:signal.obj
 0002:00008638       $unwind$__acrt_initialize_lowio$fin$0 000000018001a638     libucrt:ioinit.obj
 0002:00008638       $unwind$_query_new_handler$fin$0 000000018001a638     libucrt:new_handler.obj
 0002:00008638       $unwind$?fin$0@?0???$?RV<lambda_72d1df2b273a38828b1ce30cbf4cdab5>@@AEAV<lambda_876a65b173b8412d3a47c70a915b0cf4>@@V<lambda_41932305e351933ebe8f8be3ed8bb5dc>@@@?$__crt_seh_guarded_call@X@@QEAAX$$QEAV<lambda_72d1df2b273a38828b1ce30cbf4cdab5>@@AEAV<lambda_876a65b173b8412d3a47c70a915b0cf4>@@$$QEAV<lambda_41932305e351933ebe8f8be3ed8bb5dc>@@@Z@4HA 000000018001a638     libucrt:per_thread_data.obj
 0002:00008638       $unwind$_IsNonwritableInCurrentImage$filt$0 000000018001a638     LIBCMT:pesect.obj
 0002:00008640       $unwind$?dllmain_crt_process_detach@@YAH_N@Z 000000018001a640     LIBCMT:dll_dllmain.obj
 0002:00008674       $unwind$?dllmain_dispatch@@YAHQEAUHINSTANCE__@@KQEAX@Z 000000018001a674     LIBCMT:dll_dllmain.obj
 0002:0000869c       $unwind$?filt$0@?0??dllmain_dispatch@@YAHQEAUHINSTANCE__@@KQEAX@Z@4HA 000000018001a69c     LIBCMT:dll_dllmain.obj
 0002:000086a4       $unwind$__security_init_cookie 000000018001a6a4     LIBCMT:gs_support.obj
 0002:000086b0       $unwind$__scrt_is_nonwritable_in_current_image 000000018001a6b0     LIBCMT:utility.obj
 0002:000086d0       $unwind$__scrt_is_nonwritable_in_current_image$filt$0 000000018001a6d0     LIBCMT:utility.obj
 0002:000086d8       $unwind$__scrt_initialize_onexit_tables 000000018001a6d8     LIBCMT:utility.obj
 0002:000086e4       $unwind$__acrt_InitializeCriticalSectionEx 000000018001a6e4     libucrt:winapi_thunks.obj
 0002:000086e4       $unwind$??$ensure_buffer_is_big_enough@D@formatting_buffer@__crt_stdio_output@@QEAA_N_K@Z 000000018001a6e4     libucrt:output.obj
 0002:000086e4       $unwind$_seh_filter_exe    000000018001a6e4     libucrt:exception_filter.obj
 0002:000086e4       $unwind$_recalloc_base     000000018001a6e4     libucrt:recalloc.obj
 0002:000086e4       $unwind$__scrt_dllmain_exception_filter 000000018001a6e4     LIBCMT:utility.obj
 0002:000086e4       $unwind$__acrt_free_locale 000000018001a6e4     libucrt:locale_refcounting.obj
 0002:000086e4       $unwind$?setSBCS@@YAXPEAU__crt_multibyte_data@@@Z 000000018001a6e4     libucrt:mbctype.obj
 0002:000086e4       $unwind$__acrt_lowio_create_handle_array 000000018001a6e4     libucrt:osfinfo.obj
 0002:000086e4       $unwind$__acrt_execute_initializers 000000018001a6e4     libucrt:shared_initialization.obj
 0002:000086e4       $unwind$?expand_if_necessary@?$argument_list@D@?A0xca0879c4@@AEAAHXZ 000000018001a6e4     libucrt:argv_wildcards.obj
 0002:000086f8       $unwind$__scrt_fastfail    000000018001a6f8     LIBCMT:utility_desktop.obj
 0002:00008708       $unwind$__isa_available_init 000000018001a708     LIBCMT:_cpu_disp_.obj
 0002:00008720       $xdatasym                  000000018001a720     LIBCMT:_guard_dispatch_.obj
 0002:00008728       $xdatasym                  000000018001a728     libvcruntime:memset.obj
 0002:0000872c       $unwind$strchr             000000018001a72c     libvcruntime:strchr.obj
 0002:0000872c       $unwind$strrchr            000000018001a72c     libvcruntime:strrchr.obj
 0002:00008734       $unwind$__C_specific_handler 000000018001a734     libvcruntime:_riscchandler_.obj
 0002:00008750       $xdatasym                  000000018001a750     libvcruntime:_jmpuwind_.obj
 0002:00008764       $unwind$__acrt_initialize_winapi_thunks 000000018001a764     libucrt:winapi_thunks.obj
 0002:00008764       $unwind$__vcrt_initialize_winapi_thunks 000000018001a764     libvcruntime:winapi_downlevel.obj
 0002:0000876c       $unwind$__vcrt_uninitialize_winapi_thunks 000000018001a76c     libvcruntime:winapi_downlevel.obj
 0002:00008774       $unwind$?try_get_function@@YAPEAXW4function_id@?A0x89697e75@@QEBDQEBW4module_id@2@2@Z 000000018001a774     libvcruntime:winapi_downlevel.obj
 0002:00008774       $unwind$?try_get_function@@YAPEAXW4function_id@?A0x63058377@@QEBDQEBW4module_id@2@2@Z 000000018001a774     libucrt:winapi_thunks.obj
 0002:00008790       $xdatasym                  000000018001a790     libvcruntime:memcpy.obj
 0002:00008798       $xdatasym                  000000018001a798     libvcruntime:handlers.obj
 0002:000087a0       $unwind$__DestructExceptionObject 000000018001a7a0     libvcruntime:ehhelpers.obj
 0002:000087c0       $unwind$__stdio_common_vsprintf 000000018001a7c0     libucrt:output.obj
 0002:000087e4       $unwind$??$parse_command_line@D@@YAXPEADPEAPEAD0PEA_K2@Z 000000018001a7e4     libucrt:argv_parsing.obj
 0002:000087e4       $unwind$?write_string@?$string_output_adapter@D@__crt_stdio_output@@QEBAXQEBDHQEAH1@Z 000000018001a7e4     libucrt:output.obj
 0002:00008800       $unwind$?process@?$output_processor@DV?$string_output_adapter@D@__crt_stdio_output@@V?$standard_base@DV?$string_output_adapter@D@__crt_stdio_output@@@2@@__crt_stdio_output@@QEAAHXZ 000000018001a800     libucrt:output.obj
 0002:00008810       $unwind$?parse_int_from_format_string@?$output_processor@DV?$string_output_adapter@D@__crt_stdio_output@@V?$standard_base@DV?$string_output_adapter@D@__crt_stdio_output@@@2@@__crt_stdio_output@@AEAA_NQEAH@Z 000000018001a810     libucrt:output.obj
 0002:00008824       $unwind$?state_case_type@?$output_processor@DV?$string_output_adapter@D@__crt_stdio_output@@V?$standard_base@DV?$string_output_adapter@D@__crt_stdio_output@@@2@@__crt_stdio_output@@AEAA_NXZ 000000018001a824     libucrt:output.obj
 0002:0000883c       $unwind$?type_case_a@?$output_processor@DV?$string_output_adapter@D@__crt_stdio_output@@V?$standard_base@DV?$string_output_adapter@D@__crt_stdio_output@@@2@@__crt_stdio_output@@AEAA_NXZ 000000018001a83c     libucrt:output.obj
 0002:00008848       $unwind$?write_stored_string_tchar@?$output_processor@DV?$string_output_adapter@D@__crt_stdio_output@@V?$standard_base@DV?$string_output_adapter@D@__crt_stdio_output@@@2@@__crt_stdio_output@@AEAA_ND@Z 000000018001a848     libucrt:output.obj
 0002:00008860       $unwind$??$type_case_integer_parse_into_buffer@I@?$output_processor@DV?$string_output_adapter@D@__crt_stdio_output@@V?$standard_base@DV?$string_output_adapter@D@__crt_stdio_output@@@2@@__crt_stdio_output@@AEAAXII_N@Z 000000018001a860     libucrt:output.obj
 0002:00008860       $unwind$??$type_case_integer_parse_into_buffer@_K@?$output_processor@DV?$string_output_adapter@D@__crt_stdio_output@@V?$standard_base@DV?$string_output_adapter@D@__crt_stdio_output@@@2@@__crt_stdio_output@@AEAAX_KI_N@Z 000000018001a860     libucrt:output.obj
 0002:00008860       $unwind$??$write_multiple_characters@V?$string_output_adapter@D@__crt_stdio_output@@D@__crt_stdio_output@@YAXAEBV?$string_output_adapter@D@0@DHQEAH@Z 000000018001a860     libucrt:output.obj
 0002:00008868       $unwind$__acrt_initialize_stdio 000000018001a868     libucrt:_file.obj
 0002:00008868       $unwind$_initterm          000000018001a868     libucrt:initterm.obj
 0002:00008880       $unwind$?common_exit@@YAXHW4_crt_exit_cleanup_mode@@W4_crt_exit_return_mode@@@Z 000000018001a880     libucrt:exit.obj
 0002:000088c0       $unwind$_configure_narrow_argv 000000018001a8c0     libucrt:argv_parsing.obj
 0002:000088d4       $unwind$??$free_environment@_W@@YAXQEAPEA_W@Z 000000018001a8d4     libucrt:environment_initialization.obj
 0002:000088d4       $unwind$??$free_environment@D@@YAXQEAPEAD@Z 000000018001a8d4     libucrt:environment_initialization.obj
 0002:000088e0       $unwind$??$create_environment@D@@YAQEAPEADQEAD@Z 000000018001a8e0     libucrt:environment_initialization.obj
 0002:000088f8       $unwind$_execute_onexit_table 000000018001a8f8     libucrt:onexit.obj
 0002:00008900       $unwind$??$?RV<lambda_e24bbb7b643b32fcea6fa61b31d4c984>@@AEAV<lambda_275893d493268fdec8709772e3fcec0e>@@V<lambda_9d71df4d7cf3f480f8d633942495c3b0>@@@?$__crt_seh_guarded_call@H@@QEAAH$$QEAV<lambda_e24bbb7b643b32fcea6fa61b31d4c984>@@AEAV<lambda_275893d493268fdec8709772e3fcec0e>@@$$QEAV<lambda_9d71df4d7cf3f480f8d633942495c3b0>@@@Z 000000018001a900     libucrt:onexit.obj
 0002:00008930       $unwind$terminate          000000018001a930     libucrt:terminate.obj
 0002:00008950       $unwind$??$parse_integer@KV?$c_string_character_source@D@__crt_strtox@@@__crt_strtox@@YAKQEAU__crt_locale_pointers@@V?$c_string_character_source@D@0@H_N@Z 000000018001a950     libucrt:atox.obj
 0002:00008970       $xdatasym                  000000018001a970     libucrt:strncmp.obj
 0002:00008974       $unwind$wctomb_s           000000018001a974     libucrt:wctomb.obj
 0002:00008974       $unwind$_invalid_parameter_noinfo 000000018001a974     libucrt:invalid_parameter.obj
 0002:00008974       $unwind$_log10_special     000000018001a974     libucrt:log_special.obj
 0002:0000897c       $unwind$__acrt_call_reportfault 000000018001a97c     libucrt:invalid_parameter.obj
 0002:0000899c       $unwind$_isleadbyte_l      000000018001a99c     libucrt:_wctype.obj
 0002:0000899c       $unwind$isdigit            000000018001a99c     libucrt:_ctype.obj
 0002:0000899c       $unwind$?getSystemCP@@YAHH@Z 000000018001a99c     libucrt:mbctype.obj
 0002:000089a4       $unwind$_tolower_l         000000018001a9a4     libucrt:tolower_toupper.obj
 0002:000089b4       $unwind$?destroy_fls@@YAXPEAX@Z 000000018001a9b4     libucrt:per_thread_data.obj
 0002:000089b4       $unwind$__acrt_locale_free_lc_time_if_unreferenced 000000018001a9b4     libucrt:locale_refcounting.obj
 0002:000089b4       $unwind$_free_base         000000018001a9b4     libucrt:free_base.obj
 0002:000089b4       $unwind$__acrt_locale_free_numeric 000000018001a9b4     libucrt:initnum.obj
 0002:000089bc       $unwind$strtol             000000018001a9bc     libucrt:strtox.obj
 0002:000089c4       $unwind$_mbtowc_l          000000018001a9c4     libucrt:mbtowc.obj
 0002:000089c4       $unwind$__acrt_LCMapStringEx 000000018001a9c4     libucrt:winapi_thunks.obj
 0002:000089dc       $unwind$_wctomb_s_l        000000018001a9dc     libucrt:wctomb.obj
 0002:000089ec       $unwind$wcsnlen            000000018001a9ec     libucrt:strnlen.obj
 0002:000089ec       $unwind$strnlen            000000018001a9ec     libucrt:strnlen.obj
 0002:000089f4       $unwind$?construct_ptd_array@@YAXQEAU__acrt_ptd@@@Z 000000018001a9f4     libucrt:per_thread_data.obj
 0002:000089fc       $unwind$?destroy_ptd_array@@YAXQEAU__acrt_ptd@@@Z 000000018001a9fc     libucrt:per_thread_data.obj
 0002:00008a04       $unwind$??$?RV<lambda_72d1df2b273a38828b1ce30cbf4cdab5>@@AEAV<lambda_876a65b173b8412d3a47c70a915b0cf4>@@V<lambda_41932305e351933ebe8f8be3ed8bb5dc>@@@?$__crt_seh_guarded_call@X@@QEAAX$$QEAV<lambda_72d1df2b273a38828b1ce30cbf4cdab5>@@AEAV<lambda_876a65b173b8412d3a47c70a915b0cf4>@@$$QEAV<lambda_41932305e351933ebe8f8be3ed8bb5dc>@@@Z 000000018001aa04     libucrt:per_thread_data.obj
 0002:00008a28       $unwind$??$?RV<lambda_5e887d1dcbef67a5eb4283622ba103bf>@@AEAV<lambda_4466841279450cc726390878d4a41900>@@V<lambda_341c25c0346d94847f1f3c463c57e077>@@@?$__crt_seh_guarded_call@X@@QEAAX$$QEAV<lambda_5e887d1dcbef67a5eb4283622ba103bf>@@AEAV<lambda_4466841279450cc726390878d4a41900>@@$$QEAV<lambda_341c25c0346d94847f1f3c463c57e077>@@@Z 000000018001aa28     libucrt:per_thread_data.obj
 0002:00008a4c       $unwind$??$?RV<lambda_46352004c1216016012b18bd6f87e700>@@AEAV<lambda_3bd07e1a1191394380780325891bf33f>@@V<lambda_334532d3f185bcaa59b5be82d7d22bff>@@@?$__crt_seh_guarded_call@X@@QEAAX$$QEAV<lambda_46352004c1216016012b18bd6f87e700>@@AEAV<lambda_3bd07e1a1191394380780325891bf33f>@@$$QEAV<lambda_334532d3f185bcaa59b5be82d7d22bff>@@@Z 000000018001aa4c     libucrt:per_thread_data.obj
 0002:00008a70       $unwind$??$?RV<lambda_fb3a7dec4e47f37f22dae91bb15c9095>@@AEAV<lambda_698284760c8add0bfb0756c19673e34b>@@V<lambda_dfb8eca1e75fef3034a8fb18dd509707>@@@?$__crt_seh_guarded_call@X@@QEAAX$$QEAV<lambda_fb3a7dec4e47f37f22dae91bb15c9095>@@AEAV<lambda_698284760c8add0bfb0756c19673e34b>@@$$QEAV<lambda_dfb8eca1e75fef3034a8fb18dd509707>@@@Z 000000018001aa70     libucrt:per_thread_data.obj
 0002:00008a94       $unwind$__acrt_fp_format   000000018001aa94     libucrt:cvt.obj
 0002:00008ab0       $unwind$?fp_format_nan_or_infinity@@YAHW4__acrt_fp_class@@_NPEAD_K1@Z 000000018001aab0     libucrt:cvt.obj
 0002:00008ac4       $unwind$?fp_format_e_internal@@YAHQEAD_KH_NIQEAU_strflt@@2QEAU__crt_locale_pointers@@@Z 000000018001aac4     libucrt:cvt.obj
 0002:00008adc       $unwind$?fp_format_e@@YAHQEBNQEAD_K12H_NIQEAU__crt_locale_pointers@@@Z 000000018001aadc     libucrt:cvt.obj
 0002:00008af0       $unwind$?fp_format_a@@YAHQEBNPEAD_KQEAD2H_NIQEAU__crt_locale_pointers@@@Z 000000018001aaf0     libucrt:cvt.obj
 0002:00008b0c       $unwind$?fp_format_f_internal@@YAHQEAD_KHQEAU_strflt@@_NQEAU__crt_locale_pointers@@@Z 000000018001ab0c     libucrt:cvt.obj
 0002:00008b0c       $unwind$__dcrt_get_narrow_environment_from_os 000000018001ab0c     libucrt:get_environment_from_os.obj
 0002:00008b24       $unwind$?fp_format_g@@YAHQEBNQEAD_K12H_NIQEAU__crt_locale_pointers@@@Z 000000018001ab24     libucrt:cvt.obj
 0002:00008b38       $unwind$__acrt_uninitialize_locale 000000018001ab38     libucrt:wsetlocale.obj
 0002:00008b58       $unwind$__acrt_initialize_lowio 000000018001ab58     libucrt:ioinit.obj
 0002:00008b78       $unwind$?initialize_inherited_file_handles_nolock@@YAXXZ 000000018001ab78     libucrt:ioinit.obj
 0002:00008b94       $unwind$?initialize_stdio_handles_nolock@@YAXXZ 000000018001ab94     libucrt:ioinit.obj
 0002:00008b94       $unwind$_free_osfhnd       000000018001ab94     libucrt:osfinfo.obj
 0002:00008ba8       $unwind$__acrt_is_packaged_app 000000018001aba8     libucrt:winapi_thunks.obj
 0002:00008bb4       $unwind$??$common_expand_argv_wildcards@D@@YAHQEAPEADQEAPEAPEAD@Z 000000018001abb4     libucrt:argv_wildcards.obj
 0002:00008bcc       $unwind$??$copy_and_add_argument_to_buffer@D@@YAHQEBD0_KAEAV?$argument_list@D@?A0xca0879c4@@@Z 000000018001abcc     libucrt:argv_wildcards.obj
 0002:00008be8       $unwind$??$expand_argument_wildcards@D@@YAHQEAD0AEAV?$argument_list@D@?A0xca0879c4@@@Z 000000018001abe8     libucrt:argv_wildcards.obj
 0002:00008c08       $unwind$__acrt_update_thread_multibyte_data 000000018001ac08     libucrt:mbctype.obj
 0002:00008c2c       $unwind$_setmbcp_nolock    000000018001ac2c     libucrt:mbctype.obj
 0002:00008c4c       $unwind$?setSBUpLow@@YAXPEAU__crt_multibyte_data@@@Z 000000018001ac4c     libucrt:mbctype.obj
 0002:00008c68       $unwind$?setmbcp_internal@@YAHH_N@Z 000000018001ac68     libucrt:mbctype.obj
 0002:00008c78       $unwind$??$?RV<lambda_99476a1ad63dd22509b5d3e65b0ffc95>@@AEAV<lambda_ad1ced32f4ac17aa236e5ef05d6b3b7c>@@V<lambda_f7424dd8d45958661754dc4f2697e9c3>@@@?$__crt_seh_guarded_call@X@@QEAAX$$QEAV<lambda_99476a1ad63dd22509b5d3e65b0ffc95>@@AEAV<lambda_ad1ced32f4ac17aa236e5ef05d6b3b7c>@@$$QEAV<lambda_f7424dd8d45958661754dc4f2697e9c3>@@@Z 000000018001ac78     libucrt:mbctype.obj
 0002:00008c9c       $unwind$?x_ismbbtype_l@@YAHPEAU__crt_locale_pointers@@IHH@Z 000000018001ac9c     libucrt:ismbbyte.obj
 0002:00008cac       $unwind$_query_new_handler 000000018001acac     libucrt:new_handler.obj
 0002:00008ccc       $unwind$__acrt_get_sigabrt_handler 000000018001accc     libucrt:signal.obj
 0002:00008cd4       $unwind$raise              000000018001acd4     libucrt:signal.obj
 0002:00008d00       $unwind$??$?RV<lambda_c36588078e9f5dfd39652860aa6b3aaf>@@AEAV<lambda_ec61778202f4f5fc7e7711acc23c3bca>@@V<lambda_dc9d2797ccde5d239b4a0efae8ebd7db>@@@?$__crt_seh_guarded_call@P6AXH@Z@@QEAAP6AXH@Z$$QEAV<lambda_c36588078e9f5dfd39652860aa6b3aaf>@@AEAV<lambda_ec61778202f4f5fc7e7711acc23c3bca>@@$$QEAV<lambda_dc9d2797ccde5d239b4a0efae8ebd7db>@@@Z 000000018001ad00     libucrt:signal.obj
 0002:00008d24       $unwind$_isctype_l         000000018001ad24     libucrt:isctype.obj
 0002:00008d40       $unwind$__acrt_LCMapStringA 000000018001ad40     libucrt:lcmapstringa.obj
 0002:00008d50       $unwind$?__acrt_LCMapStringA_stat@@YAHPEAU__crt_locale_pointers@@PEB_WKPEBDHPEADHHH@Z 000000018001ad50     libucrt:lcmapstringa.obj
 0002:00008d78       $unwind$__acrt_update_thread_locale_data 000000018001ad78     libucrt:locale_refcounting.obj
 0002:00008d9c       $unwind$__acrt_fltout      000000018001ad9c     libucrt:cfout.obj
 0002:00008dbc       $unwind$?divide@__crt_strtox@@YA_KAEAUbig_integer@1@AEBU21@@Z 000000018001adbc     libucrt:cfout.obj
 0002:00008ddc       $chain$5$?divide@__crt_strtox@@YA_KAEAUbig_integer@1@AEBU21@@Z 000000018001addc     libucrt:cfout.obj
 0002:00008df0       $chain$6$?divide@__crt_strtox@@YA_KAEAUbig_integer@1@AEBU21@@Z 000000018001adf0     libucrt:cfout.obj
 0002:00008e00       $unwind$_fcloseall         000000018001ae00     libucrt:closeall.obj
 0002:00008e24       $unwind$common_flush_all   000000018001ae24     libucrt:fflush.obj
 0002:00008e60       $unwind$__acrt_locale_free_time 000000018001ae60     libucrt:inittime.obj
 0002:00008e70       $unwind$__acrt_GetStringTypeA 000000018001ae70     libucrt:getstringtypea.obj
 0002:00008e98       $unwind$__acrt_lowio_destroy_handle_array 000000018001ae98     libucrt:osfinfo.obj
 0002:00008ea8       $unwind$__acrt_lowio_ensure_fh_exists 000000018001aea8     libucrt:osfinfo.obj
 0002:00008ed4       $unwind$qsort              000000018001aed4     libucrt:qsort.obj
 0002:00008eec       $chain$4$qsort             000000018001aeec     libucrt:qsort.obj
 0002:00008f10       $chain$5$qsort             000000018001af10     libucrt:qsort.obj
 0002:00008f20       $unwind$?shortsort@@YAXPEAD0_KP6AHPEBX2@Z@Z 000000018001af20     libucrt:qsort.obj
 0002:00008f30       $chain$2$?shortsort@@YAXPEAD0_KP6AHPEBX2@Z@Z 000000018001af30     libucrt:qsort.obj
 0002:00008f4c       $chain$3$?shortsort@@YAXPEAD0_KP6AHPEBX2@Z@Z 000000018001af4c     libucrt:qsort.obj
 0002:00008f5c       $unwind$strpbrk            000000018001af5c     libucrt:strpbrk.obj
 0002:00008f6c       $unwind$_mbsdec_l          000000018001af6c     libucrt:mbsdec.obj
 0002:00008f78       $xdatasym                  000000018001af78     libucrt:log10.obj
 0002:00008f84       $unwind$_write             000000018001af84     libucrt:write.obj
 0002:00008fb4       $unwind$_write_nolock      000000018001afb4     libucrt:write.obj
 0002:00008fcc       $unwind$?write_double_translated_ansi_nolock@@YA?AUwrite_result@?A0x9c548279@@HQEBDI@Z 000000018001afcc     libucrt:write.obj
 0002:00008fec       $unwind$?write_text_utf16le_nolock@@YA?AUwrite_result@?A0x9c548279@@HQEBDI@Z 000000018001afec     libucrt:write.obj
 0002:00008fec       $unwind$?write_text_ansi_nolock@@YA?AUwrite_result@?A0x9c548279@@HQEBDI@Z 000000018001afec     libucrt:write.obj
 0002:0000900c       $unwind$?write_text_utf8_nolock@@YA?AUwrite_result@?A0x9c548279@@HQEBDI@Z 000000018001b00c     libucrt:write.obj
 0002:00009030       $unwind$fclose             000000018001b030     libucrt:fclose.obj
 0002:00009054       $unwind$_close             000000018001b054     libucrt:close.obj
 0002:00009054       $unwind$_commit            000000018001b054     libucrt:commit.obj
 0002:0000905c       $unwind$??$?RV<lambda_b521505b218e5242e90febf6bfebc422>@@AEAV<lambda_6978c1fb23f02e42e1d9e99668cc68aa>@@V<lambda_314360699dd331753a4119843814e9a7>@@@?$__crt_seh_guarded_call@H@@QEAAH$$QEAV<lambda_b521505b218e5242e90febf6bfebc422>@@AEAV<lambda_6978c1fb23f02e42e1d9e99668cc68aa>@@$$QEAV<lambda_314360699dd331753a4119843814e9a7>@@@Z 000000018001b05c     libucrt:commit.obj
 0002:00009080       $unwind$common_control87   000000018001b080     libucrt:ieee.obj
 0002:000090b0       $unwind$_call_matherr      000000018001b0b0     libucrt:libm_error.obj
 0002:000090b8       $unwind$_handle_error      000000018001b0b8     libucrt:libm_error.obj
 0002:000090d8       $unwind$__acrt_initialize_fma3 000000018001b0d8     libucrt:fma3_available.obj
 0002:000090e0       $unwind$_log_special_common 000000018001b0e0     libucrt:log_special.obj
 0002:000090ec       $unwind$??$?RV<lambda_bfedae4ebbf01fab1bb6dcc6a9e276e0>@@AEAV<lambda_2fe9b910cf3cbf4a0ab98a02ba45b3ec>@@V<lambda_237c231691f317818eb88cc1d5d642d6>@@@?$__crt_seh_guarded_call@H@@QEAAH$$QEAV<lambda_bfedae4ebbf01fab1bb6dcc6a9e276e0>@@AEAV<lambda_2fe9b910cf3cbf4a0ab98a02ba45b3ec>@@$$QEAV<lambda_237c231691f317818eb88cc1d5d642d6>@@@Z 000000018001b0ec     libucrt:close.obj
 0002:00009110       $xdatasym                  000000018001b110     libucrt:fpsr.obj
 0002:00009118       $unwind$__dcrt_lowio_initialize_console_output 000000018001b118     libucrt:initcon.obj
 0002:00009118       $unwind$_raise_exc         000000018001b118     libucrt:fpexcept.obj
 0002:00009120       $unwind$_raise_exc_ex      000000018001b120     libucrt:fpexcept.obj
 0002:00009134       $unwind$_ctrlfp            000000018001b134     libucrt:fpctrl.obj
 0002:0000915c       $unwind$_IsNonwritableInCurrentImage 000000018001b15c     LIBCMT:pesect.obj
 0002:00009180       $xdatasym                  000000018001b180     LIBCMT:_chkstk_.obj
 0002:00009188       $xdatasym                  000000018001b188     libvcruntime:memcmp.obj
 0002:00009190       .edata                     000000018001b190     gdi+.exp
 0002:000091b8       rgpv                       000000018001b1b8     gdi+.exp
 0002:000091cc       rgszName                   000000018001b1cc     gdi+.exp
 0002:000091e0       rgwOrd                     000000018001b1e0     gdi+.exp
 0002:000091ea       szName                     000000018001b1ea     gdi+.exp
 0002:000091f3       $N00001                    000000018001b1f3     gdi+.exp
 0002:000091fe       $N00002                    000000018001b1fe     gdi+.exp
 0002:00009207       $N00003                    000000018001b207     gdi+.exp
 0002:00009210       $N00004                    000000018001b210     gdi+.exp
 0002:00009219       $N00005                    000000018001b219     gdi+.exp
 0002:000096a2       .idata$6                   000000018001b6a2     kernel32:KERNEL32.dll
 0002:000096da       .idata$6                   000000018001b6da     user32:USER32.dll
 0002:00009750       .idata$6                   000000018001b750     gdi32:GDI32.dll
 0002:0000977c       .idata$6                   000000018001b77c     ole32:ole32.dll
 0003:00000040       ?__vcrt_flsindex@@3KA      000000018001c040     libvcruntime:per_thread_data.obj
 0003:00000054       errno_no_memory            000000018001c054     libucrt:errno.obj
 0003:00000058       doserrno_no_memory         000000018001c058     libucrt:errno.obj
 0003:0000005c       __acrt_flsindex            000000018001c05c     libucrt:per_thread_data.obj
 0003:00000510       __rgctypeflag              000000018001c510     libucrt:mbctype.obj
 0003:00000520       __rgcode_page_info         000000018001c520     libucrt:mbctype.obj
 0003:000008d0       ?dazSupported@?1??common_control87@@9@9 000000018001c8d0     libucrt:ieee.obj
 0003:000008e0       ?dazSupported@?1??_ctrlfp@@9@9 000000018001c8e0     libucrt:fpctrl.obj
 0003:00000930       ?g_Threads@@3PAUConEmuThreadInfo@@A 000000018001c930     common-kernel64:WThreads.obj
 0003:00009130       ?gh_UnknownTerminatedThread@@3PEAXEA 0000000180025130     common-kernel64:WThreads.obj
 0003:00009140       GS_ExceptionRecord         0000000180025140     LIBCMT:gs_report.obj
 0003:000091e0       GS_ContextRecord           00000001800251e0     LIBCMT:gs_report.obj
 0003:000096b0       ?__proc_attached@@3HA      00000001800256b0     LIBCMT:dll_dllmain.obj
 0003:000096dc       ?module_local_atexit_table_initialized@@3_NA 00000001800256dc     LIBCMT:utility.obj
 0003:000096e8       ?module_local_atexit_table@@3U_onexit_table_t@@A 00000001800256e8     LIBCMT:utility.obj
 0003:00009700       ?module_local_at_quick_exit_table@@3U_onexit_table_t@@A 0000000180025700     LIBCMT:utility.obj
 0003:00009718       ?is_initialized_as_dll@@3_NA 0000000180025718     LIBCMT:utility.obj
 0003:00009768       ?heap@@3V_HeapManager@@A   0000000180025768     libvcruntime:undname.obj
 0003:00009790       ?__vcrt_startup_thread_ptd@@3U__vcrt_ptd@@A 0000000180025790     libvcruntime:per_thread_data.obj
 0003:00009808       __vcrt_lock_table          0000000180025808     libvcruntime:locks.obj
 0003:00009830       __vcrt_locks_initialized   0000000180025830     libvcruntime:locks.obj
 0003:00009838       ?module_handles@@3PAPEAUHINSTANCE__@@A 0000000180025838     libvcruntime:winapi_downlevel.obj
 0003:00009850       ?encoded_function_pointers@@3PAPEAXA 0000000180025850     libvcruntime:winapi_downlevel.obj
 0003:00009888       c_termination_complete     0000000180025888     libucrt:exit.obj
 0003:00009890       thread_local_exit_callback_func 0000000180025890     libucrt:exit.obj
 0003:00009898       ?c_exit_complete@?5??common_exit@@YAXHW4_crt_exit_cleanup_mode@@W4_crt_exit_return_mode@@@Z@4_NA 0000000180025898     libucrt:exit.obj
 0003:000098a0       ?program_name@?5???$common_configure_argv@D@@YAHW4_crt_argv_mode@@@Z@4PADA 00000001800258a0     libucrt:argv_parsing.obj
 0003:000099f8       __acrt_invalid_parameter_handler 00000001800259f8     libucrt:invalid_parameter.obj
 0003:00009a10       enable_percent_n           0000000180025a10     libucrt:printf_count_output.obj
 0003:00009e50       __acrt_lock_table          0000000180025e50     libucrt:locks.obj
 0003:0000a058       __acrt_locks_initialized   0000000180026058     libucrt:locks.obj
 0003:0000a060       module_handles             0000000180026060     libucrt:winapi_thunks.obj
 0003:0000a100       encoded_function_pointers  0000000180026100     libucrt:winapi_thunks.obj
 0003:0000a200       ?state_cache@?1??__acrt_is_packaged_app@@9@4JA 0000000180026200     libucrt:winapi_thunks.obj
 0003:0000a21c       fSystemSet                 000000018002621c     libucrt:mbctype.obj
 0003:0000a228       ?initialized@?1??__acrt_initialize_multibyte@@9@4_NA 0000000180026228     libucrt:mbctype.obj
 0003:0000a260       __acrt_new_handler         0000000180026260     libucrt:new_handler.obj
 0003:0000a268       ctrlc_action               0000000180026268     libucrt:signal.obj
 0003:0000a270       ctrlbreak_action           0000000180026270     libucrt:signal.obj
 0003:0000a278       abort_action               0000000180026278     libucrt:signal.obj
 0003:0000a280       term_action                0000000180026280     libucrt:signal.obj
 0003:0000a288       user_matherr               0000000180026288     libucrt:matherr.obj
 0003:0000a290       __acrt_global_new_mode     0000000180026290     libucrt:new_mode.obj
 0003:0000a29c       __acrt_app_type            000000018002629c     libucrt:report_runtime_error.obj
 0004:00000000       $pdata$?Init@GDIPlusDecoder@@QEAA_NPEAUCET_Init@@@Z 0000000180027000     gdip.obj
 0004:0000000c       $pdata$?FreeThreadProc@GDIPlusDecoder@@SAKPEAX@Z 000000018002700c     gdip.obj
 0004:00000018       $pdata$?Close@GDIPlusDecoder@@QEAAXXZ 0000000180027018     gdip.obj
 0004:00000024       $pdata$?Open@GDIPlusImage@@QEAA_N_NPEB_WPEBE_JU_COORD@@@Z 0000000180027024     gdip.obj
 0004:00000030       $pdata$?SelectPage@GDIPlusImage@@QEAA_NI@Z 0000000180027030     gdip.obj
 0004:0000003c       $pdata$?Close@GDIPlusImage@@QEAAXXZ 000000018002703c     gdip.obj
 0004:00000048       $pdata$?GetExifTagValueAsInt@GDIPlusImage@@QEAA_NKAEAH@Z 0000000180027048     gdip.obj
 0004:00000054       $pdata$?CalculateShowSize@GDIPlusImage@@QEAAXAEAH0000@Z 0000000180027054     gdip.obj
 0004:00000060       $pdata$?GetPageBits@GDIPlusImage@@QEAA_NPEAUCET_LoadInfo@@@Z 0000000180027060     gdip.obj
 0004:0000006c       $pdata$?CET_Init@@YAHPEAU0@@Z 000000018002706c     gdip.obj
 0004:00000078       $pdata$?CET_Done@@YAXPEAUCET_Init@@@Z 0000000180027078     gdip.obj
 0004:00000084       $pdata$?CET_Load@@YAHPEAUCET_LoadInfo@@@Z 0000000180027084     gdip.obj
 0004:00000090       $pdata$?CET_Free@@YAXPEAUCET_LoadInfo@@@Z 0000000180027090     gdip.obj
 0004:0000009c       $pdata$??2@YAPEAX_K@Z      000000018002709c     common-kernel64:Memory.obj
 0004:000000a8       $pdata$??3@YAXPEAX@Z       00000001800270a8     common-kernel64:Memory.obj
 0004:000000a8       $pdata$??_V@YAXPEAX@Z      00000001800270a8     common-kernel64:Memory.obj
 0004:000000b4       $pdata$?HeapInitialize@@YA_NXZ 00000001800270b4     common-kernel64:Memory.obj
 0004:000000c0       $pdata$?HeapDeinitialize@@YAXXZ 00000001800270c0     common-kernel64:Memory.obj
 0004:000000cc       $pdata$?StringCchVPrintfA@@YAJPEAD_KPEBD0@Z 00000001800270cc     common-kernel64:WThreads.obj
 0004:000000d8       $pdata$?apiCreateThread@@YAPEAXP6AKPEAX@Z0PEAKPEBDH@Z 00000001800270d8     common-kernel64:WThreads.obj
 0004:000000e4       $pdata$?apiTerminateThreadEx@@YAHPEAXKPEBDH@Z 00000001800270e4     common-kernel64:WThreads.obj
 0004:000000f0       $pdata$?SetThreadName@@YAXKPEAD@Z 00000001800270f0     common-kernel64:WThreads.obj
 0004:000000fc       $pdata$?apiThreadHelper@@YAKPEAX@Z 00000001800270fc     common-kernel64:WThreads.obj
 0004:00000108       $pdata$??$sprintf_c@$0CI@@@YAHAEAY0CI@DPEBDZZ 0000000180027108     common-kernel64:WThreads.obj
 0004:00000114       $pdata$?sprintf_c@@YAHPEAD_JPEBDZZ 0000000180027114     common-kernel64:MStrSafe.obj
 0004:00000120       $pdata$__report_securityfailure 0000000180027120     LIBCMT:gs_report.obj
 0004:0000012c       $pdata$__report_rangecheckfailure 000000018002712c     LIBCMT:gs_report.obj
 0004:00000138       $pdata$__report_gsfailure  0000000180027138     LIBCMT:gs_report.obj
 0004:00000144       $pdata$capture_current_context 0000000180027144     LIBCMT:gs_report.obj
 0004:00000150       $pdata$capture_previous_context 0000000180027150     LIBCMT:gs_report.obj
 0004:0000015c       $pdata$__raise_securityfailure 000000018002715c     LIBCMT:gs_report.obj
 0004:00000168       $pdata$__GSHandlerCheckCommon 0000000180027168     LIBCMT:_gshandler_.obj
 0004:00000174       $pdata$__GSHandlerCheck    0000000180027174     LIBCMT:_gshandler_.obj
 0004:0000018c       $pdata$?dllmain_crt_process_attach@@YAHQEAUHINSTANCE__@@QEAX@Z 000000018002718c     LIBCMT:dll_dllmain.obj
 0004:00000198       $pdata$?fin$0@?0??dllmain_crt_process_attach@@YAHQEAUHINSTANCE__@@QEAX@Z@4HA 0000000180027198     LIBCMT:dll_dllmain.obj
 0004:000001a4       $pdata$?dllmain_crt_process_detach@@YAH_N@Z 00000001800271a4     LIBCMT:dll_dllmain.obj
 0004:000001b0       $pdata$?fin$0@?0??dllmain_crt_process_detach@@YAH_N@Z@4HA 00000001800271b0     LIBCMT:dll_dllmain.obj
 0004:000001bc       $pdata$?dllmain_crt_dispatch@@YAHQEAUHINSTANCE__@@KQEAX@Z 00000001800271bc     LIBCMT:dll_dllmain.obj
 0004:000001c8       $pdata$?dllmain_dispatch@@YAHQEAUHINSTANCE__@@KQEAX@Z 00000001800271c8     LIBCMT:dll_dllmain.obj
 0004:000001d4       $pdata$?filt$0@?0??dllmain_dispatch@@YAHQEAUHINSTANCE__@@KQEAX@Z@4HA 00000001800271d4     LIBCMT:dll_dllmain.obj
 0004:000001e0       $pdata$_DllMainCRTStartup  00000001800271e0     LIBCMT:dll_dllmain.obj
 0004:000001ec       $pdata$__security_init_cookie 00000001800271ec     LIBCMT:gs_support.obj
 0004:000001f8       $pdata$__scrt_initialize_default_local_stdio_options 00000001800271f8     LIBCMT:default_local_stdio_options.obj
 0004:00000204       $pdata$__scrt_is_nonwritable_in_current_image 0000000180027204     LIBCMT:utility.obj
 0004:00000210       $pdata$__scrt_is_nonwritable_in_current_image$filt$0 0000000180027210     LIBCMT:utility.obj
 0004:0000021c       $pdata$__scrt_acquire_startup_lock 000000018002721c     LIBCMT:utility.obj
 0004:00000228       $pdata$__scrt_release_startup_lock 0000000180027228     LIBCMT:utility.obj
 0004:00000234       $pdata$__scrt_initialize_crt 0000000180027234     LIBCMT:utility.obj
 0004:00000240       $pdata$__scrt_uninitialize_crt 0000000180027240     LIBCMT:utility.obj
 0004:0000024c       $pdata$__scrt_initialize_onexit_tables 000000018002724c     LIBCMT:utility.obj
 0004:00000258       $pdata$__scrt_dllmain_exception_filter 0000000180027258     LIBCMT:utility.obj
 0004:00000264       $pdata$__scrt_dllmain_before_initialize_c 0000000180027264     LIBCMT:utility.obj
 0004:00000270       $pdata$__scrt_dllmain_after_initialize_c 0000000180027270     LIBCMT:utility.obj
 0004:0000027c       $pdata$__scrt_dllmain_uninitialize_c 000000018002727c     LIBCMT:utility.obj
 0004:00000288       $pdata$__scrt_dllmain_uninitialize_critical 0000000180027288     LIBCMT:utility.obj
 0004:00000294       $pdata$__scrt_dllmain_crt_thread_attach 0000000180027294     LIBCMT:utility.obj
 0004:000002a0       $pdata$__scrt_dllmain_crt_thread_detach 00000001800272a0     LIBCMT:utility.obj
 0004:000002ac       $pdata$__scrt_fastfail     00000001800272ac     LIBCMT:utility_desktop.obj
 0004:000002b8       $pdata$_RTC_Initialize     00000001800272b8     LIBCMT:_initsect_.obj
 0004:000002c4       $pdata$_RTC_Terminate      00000001800272c4     LIBCMT:_initsect_.obj
 0004:000002d0       $pdata$__isa_available_init 00000001800272d0     LIBCMT:_cpu_disp_.obj
 0004:000002f4       $pdata$strchr              00000001800272f4     libvcruntime:strchr.obj
 0004:00000300       $pdata$strrchr             0000000180027300     libvcruntime:strrchr.obj
 0004:0000030c       $pdata$__C_specific_handler 000000018002730c     libvcruntime:_riscchandler_.obj
 0004:00000318       $pdata$__std_type_info_destroy_list 0000000180027318     libvcruntime:std_type_info.obj
 0004:00000324       $pdata$__vcrt_initialize   0000000180027324     libvcruntime:initialization.obj
 0004:00000330       $pdata$__vcrt_uninitialize 0000000180027330     libvcruntime:initialization.obj
 0004:0000033c       $pdata$__vcrt_uninitialize_critical 000000018002733c     libvcruntime:initialization.obj
 0004:00000348       $pdata$__vcrt_thread_attach 0000000180027348     libvcruntime:initialization.obj
 0004:00000354       $pdata$__vcrt_thread_detach 0000000180027354     libvcruntime:initialization.obj
 0004:00000390       $pdata$__vcrt_initialize_ptd 0000000180027390     libvcruntime:per_thread_data.obj
 0004:0000039c       $pdata$__vcrt_uninitialize_ptd 000000018002739c     libvcruntime:per_thread_data.obj
 0004:000003a8       $pdata$__vcrt_getptd_noexit 00000001800273a8     libvcruntime:per_thread_data.obj
 0004:000003b4       $pdata$__vcrt_freeptd      00000001800273b4     libvcruntime:per_thread_data.obj
 0004:000003c0       $pdata$__vcrt_freefls      00000001800273c0     libvcruntime:per_thread_data.obj
 0004:000003cc       $pdata$__vcrt_initialize_locks 00000001800273cc     libvcruntime:locks.obj
 0004:000003d8       $pdata$__vcrt_uninitialize_locks 00000001800273d8     libvcruntime:locks.obj
 0004:000003e4       $pdata$__vcrt_FlsAlloc     00000001800273e4     libvcruntime:winapi_downlevel.obj
 0004:000003f0       $pdata$__vcrt_FlsFree      00000001800273f0     libvcruntime:winapi_downlevel.obj
 0004:000003fc       $pdata$__vcrt_FlsGetValue  00000001800273fc     libvcruntime:winapi_downlevel.obj
 0004:00000408       $pdata$__vcrt_FlsSetValue  0000000180027408     libvcruntime:winapi_downlevel.obj
 0004:00000414       $pdata$__vcrt_InitializeCriticalSectionEx 0000000180027414     libvcruntime:winapi_downlevel.obj
 0004:00000420       $pdata$__vcrt_initialize_winapi_thunks 0000000180027420     libvcruntime:winapi_downlevel.obj
 0004:0000042c       $pdata$__vcrt_uninitialize_winapi_thunks 000000018002742c     libvcruntime:winapi_downlevel.obj
 0004:00000438       $pdata$?try_get_function@@YAPEAXW4function_id@?A0x89697e75@@QEBDQEBW4module_id@2@2@Z 0000000180027438     libvcruntime:winapi_downlevel.obj
 0004:0000045c       $pdata$__DestructExceptionObject 000000018002745c     libvcruntime:ehhelpers.obj
 0004:00000468       $pdata$__DestructExceptionObject$filt$0 0000000180027468     libvcruntime:ehhelpers.obj
 0004:00000474       $pdata$??0_LocaleUpdate@@QEAA@QEAU__crt_locale_pointers@@@Z 0000000180027474     libucrt:output.obj
 0004:00000480       $pdata$__stdio_common_vsprintf 0000000180027480     libucrt:output.obj
 0004:0000048c       $pdata$?force_decimal_point@__crt_stdio_output@@YAXPEADQEAU__crt_locale_pointers@@@Z 000000018002748c     libucrt:output.obj
 0004:00000498       $pdata$?write_string@?$string_output_adapter@D@__crt_stdio_output@@QEBAXQEBDHQEAH1@Z 0000000180027498     libucrt:output.obj
 0004:000004a4       $pdata$??0?$output_processor@DV?$string_output_adapter@D@__crt_stdio_output@@V?$standard_base@DV?$string_output_adapter@D@__crt_stdio_output@@@2@@__crt_stdio_output@@QEAA@AEBV?$string_output_adapter@D@1@_KQEBDQEAU__crt_locale_pointers@@QEAD@Z 00000001800274a4     libucrt:output.obj
 0004:000004b0       $pdata$?process@?$output_processor@DV?$string_output_adapter@D@__crt_stdio_output@@V?$standard_base@DV?$string_output_adapter@D@__crt_stdio_output@@@2@@__crt_stdio_output@@QEAAHXZ 00000001800274b0     libucrt:output.obj
 0004:000004bc       $pdata$?state_case_normal@?$output_processor@DV?$string_output_adapter@D@__crt_stdio_output@@V?$standard_base@DV?$string_output_adapter@D@__crt_stdio_output@@@2@@__crt_stdio_output@@AEAA_NXZ 00000001800274bc     libucrt:output.obj
 0004:000004c8       $pdata$?state_case_normal_tchar@?$output_processor@DV?$string_output_adapter@D@__crt_stdio_output@@V?$standard_base@DV?$string_output_adapter@D@__crt_stdio_output@@@2@@__crt_stdio_output@@AEAA_ND@Z 00000001800274c8     libucrt:output.obj
 0004:000004d4       $pdata$?parse_int_from_format_string@?$output_processor@DV?$string_output_adapter@D@__crt_stdio_output@@V?$standard_base@DV?$string_output_adapter@D@__crt_stdio_output@@@2@@__crt_stdio_output@@AEAA_NQEAH@Z 00000001800274d4     libucrt:output.obj
 0004:000004e0       $pdata$?state_case_size@?$output_processor@DV?$string_output_adapter@D@__crt_stdio_output@@V?$standard_base@DV?$string_output_adapter@D@__crt_stdio_output@@@2@@__crt_stdio_output@@AEAA_NXZ 00000001800274e0     libucrt:output.obj
 0004:000004ec       $pdata$?state_case_type@?$output_processor@DV?$string_output_adapter@D@__crt_stdio_output@@V?$standard_base@DV?$string_output_adapter@D@__crt_stdio_output@@@2@@__crt_stdio_output@@AEAA_NXZ 00000001800274ec     libucrt:output.obj
 0004:000004f8       $pdata$?type_case_c_tchar@?$output_processor@DV?$string_output_adapter@D@__crt_stdio_output@@V?$standard_base@DV?$string_output_adapter@D@__crt_stdio_output@@@2@@__crt_stdio_output@@AEAA_ND@Z 00000001800274f8     libucrt:output.obj
 0004:00000504       $pdata$?type_case_Z@?$output_processor@DV?$string_output_adapter@D@__crt_stdio_output@@V?$standard_base@DV?$string_output_adapter@D@__crt_stdio_output@@@2@@__crt_stdio_output@@AEAA_NXZ 0000000180027504     libucrt:output.obj
 0004:00000510       $pdata$?type_case_s@?$output_processor@DV?$string_output_adapter@D@__crt_stdio_output@@V?$standard_base@DV?$string_output_adapter@D@__crt_stdio_output@@@2@@__crt_stdio_output@@AEAA_NXZ 0000000180027510     libucrt:output.obj
 0004:0000051c       $pdata$?type_case_a@?$output_processor@DV?$string_output_adapter@D@__crt_stdio_output@@V?$standard_base@DV?$string_output_adapter@D@__crt_stdio_output@@@2@@__crt_stdio_output@@AEAA_NXZ 000000018002751c     libucrt:output.obj
 0004:00000528       $pdata$?type_case_integer@?$output_processor@DV?$string_output_adapter@D@__crt_stdio_output@@V?$standard_base@DV?$string_output_adapter@D@__crt_stdio_output@@@2@@__crt_stdio_output@@AEAA_NI_N@Z 0000000180027528     libucrt:output.obj
 0004:00000534       $pdata$?type_case_n@?$output_processor@DV?$string_output_adapter@D@__crt_stdio_output@@V?$standard_base@DV?$string_output_adapter@D@__crt_stdio_output@@@2@@__crt_stdio_output@@AEAA_NXZ 0000000180027534     libucrt:output.obj
 0004:00000540       $pdata$?write_stored_string_tchar@?$output_processor@DV?$string_output_adapter@D@__crt_stdio_output@@V?$standard_base@DV?$string_output_adapter@D@__crt_stdio_output@@@2@@__crt_stdio_output@@AEAA_ND@Z 0000000180027540     libucrt:output.obj
 0004:0000054c       $pdata$??$write_multiple_characters@V?$string_output_adapter@D@__crt_stdio_output@@D@__crt_stdio_output@@YAXAEBV?$string_output_adapter@D@0@DHQEAH@Z 000000018002754c     libucrt:output.obj
 0004:00000558       $pdata$??$ensure_buffer_is_big_enough@D@formatting_buffer@__crt_stdio_output@@QEAA_N_K@Z 0000000180027558     libucrt:output.obj
 0004:00000564       $pdata$??$type_case_integer_parse_into_buffer@_K@?$output_processor@DV?$string_output_adapter@D@__crt_stdio_output@@V?$standard_base@DV?$string_output_adapter@D@__crt_stdio_output@@@2@@__crt_stdio_output@@AEAAX_KI_N@Z 0000000180027564     libucrt:output.obj
 0004:00000570       $pdata$??$type_case_integer_parse_into_buffer@I@?$output_processor@DV?$string_output_adapter@D@__crt_stdio_output@@V?$standard_base@DV?$string_output_adapter@D@__crt_stdio_output@@@2@@__crt_stdio_output@@AEAAXII_N@Z 0000000180027570     libucrt:output.obj
 0004:0000057c       $pdata$_initterm           000000018002757c     libucrt:initterm.obj
 0004:00000588       $pdata$_initterm_e         0000000180027588     libucrt:initterm.obj
 0004:00000594       $pdata$_seh_filter_exe     0000000180027594     libucrt:exception_filter.obj
 0004:000005a0       $pdata$?try_cor_exit_process@@YAXI@Z 00000001800275a0     libucrt:exit.obj
 0004:000005ac       $pdata$?exit_or_terminate_process@@YAXI@Z 00000001800275ac     libucrt:exit.obj
 0004:000005b8       $pdata$?common_exit@@YAXHW4_crt_exit_cleanup_mode@@W4_crt_exit_return_mode@@@Z 00000001800275b8     libucrt:exit.obj
 0004:000005c4       $pdata$?filt$0@?0??common_exit@@YAXHW4_crt_exit_cleanup_mode@@W4_crt_exit_return_mode@@@Z@4HA 00000001800275c4     libucrt:exit.obj
 0004:000005d0       $pdata$?fin$1@?0??common_exit@@YAXHW4_crt_exit_cleanup_mode@@W4_crt_exit_return_mode@@@Z@4HA 00000001800275d0     libucrt:exit.obj
 0004:000005dc       $pdata$_configure_narrow_argv 00000001800275dc     libucrt:argv_parsing.obj
 0004:000005e8       $pdata$__acrt_allocate_buffer_for_argv 00000001800275e8     libucrt:argv_parsing.obj
 0004:000005f4       $pdata$??$parse_command_line@D@@YAXPEADPEAPEAD0PEA_K2@Z 00000001800275f4     libucrt:argv_parsing.obj
 0004:00000600       $pdata$__dcrt_uninitialize_environments_nolock 0000000180027600     libucrt:environment_initialization.obj
 0004:0000060c       $pdata$??$common_initialize_environment_nolock@D@@YAHXZ 000000018002760c     libucrt:environment_initialization.obj
 0004:00000618       $pdata$??$uninitialize_environment_internal@D@@YAXAEAPEAPEAD@Z 0000000180027618     libucrt:environment_initialization.obj
 0004:00000624       $pdata$??$uninitialize_environment_internal@_W@@YAXAEAPEAPEA_W@Z 0000000180027624     libucrt:environment_initialization.obj
 0004:00000630       $pdata$??$free_environment@D@@YAXQEAPEAD@Z 0000000180027630     libucrt:environment_initialization.obj
 0004:00000630       $pdata$??$free_environment@_W@@YAXQEAPEA_W@Z 0000000180027630     libucrt:environment_initialization.obj
 0004:0000063c       $pdata$??$create_environment@D@@YAQEAPEADQEAD@Z 000000018002763c     libucrt:environment_initialization.obj
 0004:00000648       $pdata$_execute_onexit_table 0000000180027648     libucrt:onexit.obj
 0004:00000654       $pdata$??$?RV<lambda_e24bbb7b643b32fcea6fa61b31d4c984>@@AEAV<lambda_275893d493268fdec8709772e3fcec0e>@@V<lambda_9d71df4d7cf3f480f8d633942495c3b0>@@@?$__crt_seh_guarded_call@H@@QEAAH$$QEAV<lambda_e24bbb7b643b32fcea6fa61b31d4c984>@@AEAV<lambda_275893d493268fdec8709772e3fcec0e>@@$$QEAV<lambda_9d71df4d7cf3f480f8d633942495c3b0>@@@Z 0000000180027654     libucrt:onexit.obj
 0004:00000660       $pdata$?fin$0@?0???$?RV<lambda_e24bbb7b643b32fcea6fa61b31d4c984>@@AEAV<lambda_275893d493268fdec8709772e3fcec0e>@@V<lambda_9d71df4d7cf3f480f8d633942495c3b0>@@@?$__crt_seh_guarded_call@H@@QEAAH$$QEAV<lambda_e24bbb7b643b32fcea6fa61b31d4c984>@@AEAV<lambda_275893d493268fdec8709772e3fcec0e>@@$$QEAV<lambda_9d71df4d7cf3f480f8d633942495c3b0>@@@Z@4HA 0000000180027660     libucrt:onexit.obj
 0004:0000066c       $pdata$__acrt_uninitialize_critical 000000018002766c     libucrt:initialization.obj
 0004:00000678       $pdata$__acrt_thread_attach 0000000180027678     libucrt:initialization.obj
 0004:00000684       $pdata$__acrt_thread_detach 0000000180027684     libucrt:initialization.obj
 0004:00000690       $pdata$initialize_c        0000000180027690     libucrt:initialization.obj
 0004:0000069c       $pdata$uninitialize_environment 000000018002769c     libucrt:initialization.obj
 0004:000006a8       $pdata$initialize_pointers 00000001800276a8     libucrt:initialization.obj
 0004:000006b4       $pdata$uninitialize_allocated_memory 00000001800276b4     libucrt:initialization.obj
 0004:000006c0       $pdata$terminate           00000001800276c0     libucrt:terminate.obj
 0004:000006cc       $pdata$strcpy_s            00000001800276cc     libucrt:strcpy_s.obj
 0004:000006d8       $pdata$??$parse_integer@KV?$c_string_character_source@D@__crt_strtox@@@__crt_strtox@@YAKQEAU__crt_locale_pointers@@V?$c_string_character_source@D@0@H_N@Z 00000001800276d8     libucrt:atox.obj
 0004:000006f0       $pdata$abort               00000001800276f0     libucrt:abort.obj
 0004:000006fc       $pdata$_invalid_parameter_noinfo 00000001800276fc     libucrt:invalid_parameter.obj
 0004:00000708       $pdata$_invoke_watson      0000000180027708     libucrt:invalid_parameter.obj
 0004:00000714       $pdata$__acrt_call_reportfault 0000000180027714     libucrt:invalid_parameter.obj
 0004:00000720       $pdata$_invalid_parameter  0000000180027720     libucrt:invalid_parameter.obj
 0004:0000072c       $pdata$isdigit             000000018002772c     libucrt:_ctype.obj
 0004:00000738       $pdata$tolower             0000000180027738     libucrt:tolower_toupper.obj
 0004:00000744       $pdata$_tolower_l          0000000180027744     libucrt:tolower_toupper.obj
 0004:00000750       $pdata$?internal_isupper_l@@YA_NHQEAU__crt_locale_pointers@@@Z 0000000180027750     libucrt:tolower_toupper.obj
 0004:0000075c       $pdata$_errno              000000018002775c     libucrt:errno.obj
 0004:00000768       $pdata$__doserrno          0000000180027768     libucrt:errno.obj
 0004:00000774       $pdata$__acrt_errno_map_os_error 0000000180027774     libucrt:errno.obj
 0004:00000780       $pdata$_free_base          0000000180027780     libucrt:free_base.obj
 0004:0000078c       $pdata$_malloc_base        000000018002778c     libucrt:malloc_base.obj
 0004:00000798       $pdata$strtol              0000000180027798     libucrt:strtox.obj
 0004:000007a4       $pdata$_mbtowc_l           00000001800277a4     libucrt:mbtowc.obj
 0004:000007b0       $pdata$wctomb_s            00000001800277b0     libucrt:wctomb.obj
 0004:000007bc       $pdata$_wctomb_s_l         00000001800277bc     libucrt:wctomb.obj
 0004:000007c8       $pdata$wcsnlen             00000001800277c8     libucrt:strnlen.obj
 0004:000007d4       $pdata$strnlen             00000001800277d4     libucrt:strnlen.obj
 0004:000007e0       $pdata$__acrt_initialize_ptd 00000001800277e0     libucrt:per_thread_data.obj
 0004:000007ec       $pdata$__acrt_uninitialize_ptd 00000001800277ec     libucrt:per_thread_data.obj
 0004:000007f8       $pdata$__acrt_getptd       00000001800277f8     libucrt:per_thread_data.obj
 0004:00000804       $pdata$__acrt_getptd_noexit 0000000180027804     libucrt:per_thread_data.obj
 0004:00000810       $pdata$__acrt_freeptd      0000000180027810     libucrt:per_thread_data.obj
 0004:0000081c       $pdata$?destroy_fls@@YAXPEAX@Z 000000018002781c     libucrt:per_thread_data.obj
 0004:00000828       $pdata$?replace_current_thread_locale_nolock@@YAXQEAU__acrt_ptd@@QEAU__crt_locale_data@@@Z 0000000180027828     libucrt:per_thread_data.obj
 0004:00000834       $pdata$?construct_ptd_array@@YAXQEAU__acrt_ptd@@@Z 0000000180027834     libucrt:per_thread_data.obj
 0004:00000840       $pdata$?destroy_ptd_array@@YAXQEAU__acrt_ptd@@@Z 0000000180027840     libucrt:per_thread_data.obj
 0004:0000084c       $pdata$??$?RV<lambda_72d1df2b273a38828b1ce30cbf4cdab5>@@AEAV<lambda_876a65b173b8412d3a47c70a915b0cf4>@@V<lambda_41932305e351933ebe8f8be3ed8bb5dc>@@@?$__crt_seh_guarded_call@X@@QEAAX$$QEAV<lambda_72d1df2b273a38828b1ce30cbf4cdab5>@@AEAV<lambda_876a65b173b8412d3a47c70a915b0cf4>@@$$QEAV<lambda_41932305e351933ebe8f8be3ed8bb5dc>@@@Z 000000018002784c     libucrt:per_thread_data.obj
 0004:00000858       $pdata$?fin$0@?0???$?RV<lambda_fb3a7dec4e47f37f22dae91bb15c9095>@@AEAV<lambda_698284760c8add0bfb0756c19673e34b>@@V<lambda_dfb8eca1e75fef3034a8fb18dd509707>@@@?$__crt_seh_guarded_call@X@@QEAAX$$QEAV<lambda_fb3a7dec4e47f37f22dae91bb15c9095>@@AEAV<lambda_698284760c8add0bfb0756c19673e34b>@@$$QEAV<lambda_dfb8eca1e75fef3034a8fb18dd509707>@@@Z@4HA 0000000180027858     libucrt:per_thread_data.obj
 0004:00000858       $pdata$?fin$0@?0???$?RV<lambda_5e887d1dcbef67a5eb4283622ba103bf>@@AEAV<lambda_4466841279450cc726390878d4a41900>@@V<lambda_341c25c0346d94847f1f3c463c57e077>@@@?$__crt_seh_guarded_call@X@@QEAAX$$QEAV<lambda_5e887d1dcbef67a5eb4283622ba103bf>@@AEAV<lambda_4466841279450cc726390878d4a41900>@@$$QEAV<lambda_341c25c0346d94847f1f3c463c57e077>@@@Z@4HA 0000000180027858     libucrt:per_thread_data.obj
 0004:00000858       $pdata$?fin$0@?0???$?RV<lambda_46352004c1216016012b18bd6f87e700>@@AEAV<lambda_3bd07e1a1191394380780325891bf33f>@@V<lambda_334532d3f185bcaa59b5be82d7d22bff>@@@?$__crt_seh_guarded_call@X@@QEAAX$$QEAV<lambda_46352004c1216016012b18bd6f87e700>@@AEAV<lambda_3bd07e1a1191394380780325891bf33f>@@$$QEAV<lambda_334532d3f185bcaa59b5be82d7d22bff>@@@Z@4HA 0000000180027858     libucrt:per_thread_data.obj
 0004:00000858       $pdata$?fin$0@?0???$?RV<lambda_c36588078e9f5dfd39652860aa6b3aaf>@@AEAV<lambda_ec61778202f4f5fc7e7711acc23c3bca>@@V<lambda_dc9d2797ccde5d239b4a0efae8ebd7db>@@@?$__crt_seh_guarded_call@P6AXH@Z@@QEAAP6AXH@Z$$QEAV<lambda_c36588078e9f5dfd39652860aa6b3aaf>@@AEAV<lambda_ec61778202f4f5fc7e7711acc23c3bca>@@$$QEAV<lambda_dc9d2797ccde5d239b4a0efae8ebd7db>@@@Z@4HA 0000000180027858     libucrt:signal.obj
 0004:00000858       $pdata$?fin$0@?0???$?RV<lambda_72d1df2b273a38828b1ce30cbf4cdab5>@@AEAV<lambda_876a65b173b8412d3a47c70a915b0cf4>@@V<lambda_41932305e351933ebe8f8be3ed8bb5dc>@@@?$__crt_seh_guarded_call@X@@QEAAX$$QEAV<lambda_72d1df2b273a38828b1ce30cbf4cdab5>@@AEAV<lambda_876a65b173b8412d3a47c70a915b0cf4>@@$$QEAV<lambda_41932305e351933ebe8f8be3ed8bb5dc>@@@Z@4HA 0000000180027858     libucrt:per_thread_data.obj
 0004:00000858       $pdata$?fin$0@?0???$?RV<lambda_99476a1ad63dd22509b5d3e65b0ffc95>@@AEAV<lambda_ad1ced32f4ac17aa236e5ef05d6b3b7c>@@V<lambda_f7424dd8d45958661754dc4f2697e9c3>@@@?$__crt_seh_guarded_call@X@@QEAAX$$QEAV<lambda_99476a1ad63dd22509b5d3e65b0ffc95>@@AEAV<lambda_ad1ced32f4ac17aa236e5ef05d6b3b7c>@@$$QEAV<lambda_f7424dd8d45958661754dc4f2697e9c3>@@@Z@4HA 0000000180027858     libucrt:mbctype.obj
 0004:00000864       $pdata$??$?RV<lambda_5e887d1dcbef67a5eb4283622ba103bf>@@AEAV<lambda_4466841279450cc726390878d4a41900>@@V<lambda_341c25c0346d94847f1f3c463c57e077>@@@?$__crt_seh_guarded_call@X@@QEAAX$$QEAV<lambda_5e887d1dcbef67a5eb4283622ba103bf>@@AEAV<lambda_4466841279450cc726390878d4a41900>@@$$QEAV<lambda_341c25c0346d94847f1f3c463c57e077>@@@Z 0000000180027864     libucrt:per_thread_data.obj
 0004:00000870       $pdata$??$?RV<lambda_46352004c1216016012b18bd6f87e700>@@AEAV<lambda_3bd07e1a1191394380780325891bf33f>@@V<lambda_334532d3f185bcaa59b5be82d7d22bff>@@@?$__crt_seh_guarded_call@X@@QEAAX$$QEAV<lambda_46352004c1216016012b18bd6f87e700>@@AEAV<lambda_3bd07e1a1191394380780325891bf33f>@@$$QEAV<lambda_334532d3f185bcaa59b5be82d7d22bff>@@@Z 0000000180027870     libucrt:per_thread_data.obj
 0004:0000087c       $pdata$??$?RV<lambda_fb3a7dec4e47f37f22dae91bb15c9095>@@AEAV<lambda_698284760c8add0bfb0756c19673e34b>@@V<lambda_dfb8eca1e75fef3034a8fb18dd509707>@@@?$__crt_seh_guarded_call@X@@QEAAX$$QEAV<lambda_fb3a7dec4e47f37f22dae91bb15c9095>@@AEAV<lambda_698284760c8add0bfb0756c19673e34b>@@$$QEAV<lambda_dfb8eca1e75fef3034a8fb18dd509707>@@@Z 000000018002787c     libucrt:per_thread_data.obj
 0004:00000888       $pdata$__acrt_update_locale_info 0000000180027888     libucrt:locale_update.obj
 0004:00000894       $pdata$__acrt_update_multibyte_info 0000000180027894     libucrt:locale_update.obj
 0004:000008a0       $pdata$__acrt_fp_format    00000001800278a0     libucrt:cvt.obj
 0004:000008ac       $pdata$?fp_format_nan_or_infinity@@YAHW4__acrt_fp_class@@_NPEAD_K1@Z 00000001800278ac     libucrt:cvt.obj
 0004:000008b8       $pdata$?fp_format_e_internal@@YAHQEAD_KH_NIQEAU_strflt@@2QEAU__crt_locale_pointers@@@Z 00000001800278b8     libucrt:cvt.obj
 0004:000008c4       $pdata$?fp_format_e@@YAHQEBNQEAD_K12H_NIQEAU__crt_locale_pointers@@@Z 00000001800278c4     libucrt:cvt.obj
 0004:000008d0       $pdata$?fp_format_a@@YAHQEBNPEAD_KQEAD2H_NIQEAU__crt_locale_pointers@@@Z 00000001800278d0     libucrt:cvt.obj
 0004:000008dc       $pdata$?fp_format_f_internal@@YAHQEAD_KHQEAU_strflt@@_NQEAU__crt_locale_pointers@@@Z 00000001800278dc     libucrt:cvt.obj
 0004:000008e8       $pdata$?fp_format_g@@YAHQEBNQEAD_K12H_NIQEAU__crt_locale_pointers@@@Z 00000001800278e8     libucrt:cvt.obj
 0004:000008f4       $pdata$_fileno             00000001800278f4     libucrt:fileno.obj
 0004:00000900       $pdata$__acrt_initialize_stdio 0000000180027900     libucrt:_file.obj
 0004:0000090c       $pdata$__acrt_uninitialize_stdio 000000018002790c     libucrt:_file.obj
 0004:00000918       $pdata$__acrt_uninitialize_locale 0000000180027918     libucrt:wsetlocale.obj
 0004:00000924       $pdata$__acrt_uninitialize_locale$fin$0 0000000180027924     libucrt:wsetlocale.obj
 0004:00000924       $pdata$__acrt_update_thread_locale_data$fin$0 0000000180027924     libucrt:locale_refcounting.obj
 0004:00000930       $pdata$__acrt_initialize_lowio 0000000180027930     libucrt:ioinit.obj
 0004:0000093c       $pdata$__acrt_initialize_lowio$fin$0 000000018002793c     libucrt:ioinit.obj
 0004:0000093c       $pdata$__acrt_lowio_ensure_fh_exists$fin$0 000000018002793c     libucrt:osfinfo.obj
 0004:00000948       $pdata$__acrt_uninitialize_lowio 0000000180027948     libucrt:ioinit.obj
 0004:00000954       $pdata$?initialize_inherited_file_handles_nolock@@YAXXZ 0000000180027954     libucrt:ioinit.obj
 0004:00000960       $pdata$?initialize_stdio_handles_nolock@@YAXXZ 0000000180027960     libucrt:ioinit.obj
 0004:0000096c       $pdata$__acrt_initialize_locks 000000018002796c     libucrt:locks.obj
 0004:00000978       $pdata$__acrt_uninitialize_locks 0000000180027978     libucrt:locks.obj
 0004:00000984       $pdata$__acrt_FlsAlloc     0000000180027984     libucrt:winapi_thunks.obj
 0004:00000990       $pdata$__acrt_FlsFree      0000000180027990     libucrt:winapi_thunks.obj
 0004:0000099c       $pdata$__acrt_FlsGetValue  000000018002799c     libucrt:winapi_thunks.obj
 0004:000009a8       $pdata$__acrt_FlsSetValue  00000001800279a8     libucrt:winapi_thunks.obj
 0004:000009b4       $pdata$__acrt_initialize_winapi_thunks 00000001800279b4     libucrt:winapi_thunks.obj
 0004:000009c0       $pdata$__acrt_uninitialize_winapi_thunks 00000001800279c0     libucrt:winapi_thunks.obj
 0004:000009cc       $pdata$__acrt_InitializeCriticalSectionEx 00000001800279cc     libucrt:winapi_thunks.obj
 0004:000009d8       $pdata$__acrt_LCMapStringEx 00000001800279d8     libucrt:winapi_thunks.obj
 0004:000009e4       $pdata$__acrt_LocaleNameToLCID 00000001800279e4     libucrt:winapi_thunks.obj
 0004:000009f0       $pdata$__acrt_is_packaged_app 00000001800279f0     libucrt:winapi_thunks.obj
 0004:000009fc       $pdata$?try_get_function@@YAPEAXW4function_id@?A0x63058377@@QEBDQEBW4module_id@2@2@Z 00000001800279fc     libucrt:winapi_thunks.obj
 0004:00000a08       $pdata$_calloc_base        0000000180027a08     libucrt:calloc_base.obj
 0004:00000a14       $pdata$??$common_expand_argv_wildcards@D@@YAHQEAPEADQEAPEAPEAD@Z 0000000180027a14     libucrt:argv_wildcards.obj
 0004:00000a20       $pdata$?expand_if_necessary@?$argument_list@D@?A0xca0879c4@@AEAAHXZ 0000000180027a20     libucrt:argv_wildcards.obj
 0004:00000a2c       $pdata$??$copy_and_add_argument_to_buffer@D@@YAHQEBD0_KAEAV?$argument_list@D@?A0xca0879c4@@@Z 0000000180027a2c     libucrt:argv_wildcards.obj
 0004:00000a38       $pdata$??$expand_argument_wildcards@D@@YAHQEAD0AEAV?$argument_list@D@?A0xca0879c4@@@Z 0000000180027a38     libucrt:argv_wildcards.obj
 0004:00000a44       $pdata$__acrt_update_thread_multibyte_data 0000000180027a44     libucrt:mbctype.obj
 0004:00000a50       $pdata$__acrt_update_thread_multibyte_data$fin$0 0000000180027a50     libucrt:mbctype.obj
 0004:00000a5c       $pdata$__acrt_initialize_multibyte 0000000180027a5c     libucrt:mbctype.obj
 0004:00000a68       $pdata$_setmbcp_nolock     0000000180027a68     libucrt:mbctype.obj
 0004:00000a74       $pdata$?getSystemCP@@YAHH@Z 0000000180027a74     libucrt:mbctype.obj
 0004:00000a80       $pdata$?setSBCS@@YAXPEAU__crt_multibyte_data@@@Z 0000000180027a80     libucrt:mbctype.obj
 0004:00000a8c       $pdata$?setSBUpLow@@YAXPEAU__crt_multibyte_data@@@Z 0000000180027a8c     libucrt:mbctype.obj
 0004:00000a98       $pdata$?setmbcp_internal@@YAHH_N@Z 0000000180027a98     libucrt:mbctype.obj
 0004:00000aa4       $pdata$??R<lambda_ad1ced32f4ac17aa236e5ef05d6b3b7c>@@QEBAXXZ 0000000180027aa4     libucrt:mbctype.obj
 0004:00000ab0       $pdata$??$?RV<lambda_99476a1ad63dd22509b5d3e65b0ffc95>@@AEAV<lambda_ad1ced32f4ac17aa236e5ef05d6b3b7c>@@V<lambda_f7424dd8d45958661754dc4f2697e9c3>@@@?$__crt_seh_guarded_call@X@@QEAAX$$QEAV<lambda_99476a1ad63dd22509b5d3e65b0ffc95>@@AEAV<lambda_ad1ced32f4ac17aa236e5ef05d6b3b7c>@@$$QEAV<lambda_f7424dd8d45958661754dc4f2697e9c3>@@@Z 0000000180027ab0     libucrt:mbctype.obj
 0004:00000abc       $pdata$?x_ismbbtype_l@@YAHPEAU__crt_locale_pointers@@IHH@Z 0000000180027abc     libucrt:ismbbyte.obj
 0004:00000ac8       $pdata$__acrt_initialize_command_line 0000000180027ac8     libucrt:argv_data.obj
 0004:00000ad4       $pdata$__dcrt_get_narrow_environment_from_os 0000000180027ad4     libucrt:get_environment_from_os.obj
 0004:00000ae0       $pdata$_recalloc_base      0000000180027ae0     libucrt:recalloc.obj
 0004:00000aec       $pdata$__acrt_initialize_heap 0000000180027aec     libucrt:heap_handle.obj
 0004:00000af8       $pdata$__acrt_execute_initializers 0000000180027af8     libucrt:shared_initialization.obj
 0004:00000b04       $pdata$__acrt_execute_uninitializers 0000000180027b04     libucrt:shared_initialization.obj
 0004:00000b10       $pdata$_callnewh           0000000180027b10     libucrt:new_handler.obj
 0004:00000b1c       $pdata$_query_new_handler  0000000180027b1c     libucrt:new_handler.obj
 0004:00000b28       $pdata$_query_new_handler$fin$0 0000000180027b28     libucrt:new_handler.obj
 0004:00000b34       $pdata$__acrt_get_sigabrt_handler 0000000180027b34     libucrt:signal.obj
 0004:00000b40       $pdata$raise               0000000180027b40     libucrt:signal.obj
 0004:00000b4c       $pdata$raise$fin$0         0000000180027b4c     libucrt:signal.obj
 0004:00000b58       $pdata$??$?RV<lambda_c36588078e9f5dfd39652860aa6b3aaf>@@AEAV<lambda_ec61778202f4f5fc7e7711acc23c3bca>@@V<lambda_dc9d2797ccde5d239b4a0efae8ebd7db>@@@?$__crt_seh_guarded_call@P6AXH@Z@@QEAAP6AXH@Z$$QEAV<lambda_c36588078e9f5dfd39652860aa6b3aaf>@@AEAV<lambda_ec61778202f4f5fc7e7711acc23c3bca>@@$$QEAV<lambda_dc9d2797ccde5d239b4a0efae8ebd7db>@@@Z 0000000180027b58     libucrt:signal.obj
 0004:00000b64       $pdata$__acrt_invoke_user_matherr 0000000180027b64     libucrt:matherr.obj
 0004:00000b70       $pdata$__pctype_func       0000000180027b70     libucrt:ctype.obj
 0004:00000b7c       $pdata$_isctype_l          0000000180027b7c     libucrt:isctype.obj
 0004:00000b88       $pdata$_isleadbyte_l       0000000180027b88     libucrt:_wctype.obj
 0004:00000b94       $pdata$__acrt_LCMapStringA 0000000180027b94     libucrt:lcmapstringa.obj
 0004:00000ba0       $pdata$?__acrt_LCMapStringA_stat@@YAHPEAU__crt_locale_pointers@@PEB_WKPEBDHPEADHHH@Z 0000000180027ba0     libucrt:lcmapstringa.obj
 0004:00000bac       $pdata$__acrt_release_locale_ref 0000000180027bac     libucrt:locale_refcounting.obj
 0004:00000bb8       $pdata$__acrt_free_locale  0000000180027bb8     libucrt:locale_refcounting.obj
 0004:00000bc4       $pdata$__acrt_locale_free_lc_time_if_unreferenced 0000000180027bc4     libucrt:locale_refcounting.obj
 0004:00000bd0       $pdata$__acrt_update_thread_locale_data 0000000180027bd0     libucrt:locale_refcounting.obj
 0004:00000bdc       $pdata$_updatetlocinfoEx_nolock 0000000180027bdc     libucrt:locale_refcounting.obj
 0004:00000be8       $pdata$__acrt_fp_strflt_to_string 0000000180027be8     libucrt:_fptostr.obj
 0004:00000bf4       $pdata$memcpy_s            0000000180027bf4     libucrt:cfout.obj
 0004:00000c00       $pdata$__acrt_fltout       0000000180027c00     libucrt:cfout.obj
 0004:00000c0c       $pdata$?divide@__crt_strtox@@YA_KAEAUbig_integer@1@AEBU21@@Z 0000000180027c0c     libucrt:cfout.obj
 0004:00000c18       $pdata$5$?divide@__crt_strtox@@YA_KAEAUbig_integer@1@AEBU21@@Z 0000000180027c18     libucrt:cfout.obj
 0004:00000c24       $pdata$6$?divide@__crt_strtox@@YA_KAEAUbig_integer@1@AEBU21@@Z 0000000180027c24     libucrt:cfout.obj
 0004:00000c30       $pdata$_fcloseall          0000000180027c30     libucrt:closeall.obj
 0004:00000c3c       $pdata$_fcloseall$fin$0    0000000180027c3c     libucrt:closeall.obj
 0004:00000c48       $pdata$_fflush_nolock      0000000180027c48     libucrt:fflush.obj
 0004:00000c54       $pdata$__acrt_stdio_flush_nolock 0000000180027c54     libucrt:fflush.obj
 0004:00000c60       $pdata$common_flush_all    0000000180027c60     libucrt:fflush.obj
 0004:00000c6c       $pdata$common_flush_all$fin$0 0000000180027c6c     libucrt:fflush.obj
 0004:00000c78       $pdata$common_flush_all$fin$1 0000000180027c78     libucrt:fflush.obj
 0004:00000c84       $pdata$__acrt_stdio_free_buffer_nolock 0000000180027c84     libucrt:_freebuf.obj
 0004:00000c90       $pdata$_isatty             0000000180027c90     libucrt:isatty.obj
 0004:00000c9c       $pdata$__acrt_locale_free_monetary 0000000180027c9c     libucrt:initmon.obj
 0004:00000ca8       $pdata$__acrt_locale_free_numeric 0000000180027ca8     libucrt:initnum.obj
 0004:00000cb4       $pdata$__acrt_locale_free_time 0000000180027cb4     libucrt:inittime.obj
 0004:00000cc0       $pdata$?free_crt_array_internal@@YAXQEAPEBX_K@Z 0000000180027cc0     libucrt:inittime.obj
 0004:00000ccc       $pdata$__acrt_GetStringTypeA 0000000180027ccc     libucrt:getstringtypea.obj
 0004:00000cd8       $pdata$_get_osfhandle      0000000180027cd8     libucrt:osfinfo.obj
 0004:00000ce4       $pdata$_free_osfhnd        0000000180027ce4     libucrt:osfinfo.obj
 0004:00000cf0       $pdata$__acrt_lowio_create_handle_array 0000000180027cf0     libucrt:osfinfo.obj
 0004:00000cfc       $pdata$__acrt_lowio_destroy_handle_array 0000000180027cfc     libucrt:osfinfo.obj
 0004:00000d08       $pdata$__acrt_lowio_ensure_fh_exists 0000000180027d08     libucrt:osfinfo.obj
 0004:00000d14       $pdata$__acrt_DownlevelLocaleNameToLCID 0000000180027d14     libucrt:lcidtoname_downlevel.obj
 0004:00000d20       $pdata$?GetTableIndexFromLocaleName@@YAHPEB_W@Z 0000000180027d20     libucrt:lcidtoname_downlevel.obj
 0004:00000d2c       $pdata$qsort               0000000180027d2c     libucrt:qsort.obj
 0004:00000d38       $pdata$4$qsort             0000000180027d38     libucrt:qsort.obj
 0004:00000d44       $pdata$5$qsort             0000000180027d44     libucrt:qsort.obj
 0004:00000d50       $pdata$?shortsort@@YAXPEAD0_KP6AHPEBX2@Z@Z 0000000180027d50     libucrt:qsort.obj
 0004:00000d5c       $pdata$2$?shortsort@@YAXPEAD0_KP6AHPEBX2@Z@Z 0000000180027d5c     libucrt:qsort.obj
 0004:00000d68       $pdata$3$?shortsort@@YAXPEAD0_KP6AHPEBX2@Z@Z 0000000180027d68     libucrt:qsort.obj
 0004:00000d74       $pdata$strncpy_s           0000000180027d74     libucrt:strncpy_s.obj
 0004:00000d80       $pdata$strpbrk             0000000180027d80     libucrt:strpbrk.obj
 0004:00000d8c       $pdata$_mbsdec_l           0000000180027d8c     libucrt:mbsdec.obj
 0004:00000d98       $pdata$?initialize_multibyte@@YAHXZ 0000000180027d98     libucrt:multibyte_initializer.obj
 0004:00000da4       $pdata$_msize              0000000180027da4     libucrt:msize.obj
 0004:00000db0       $pdata$_realloc_base       0000000180027db0     libucrt:realloc_base.obj
 0004:00000dbc       $pdata$fegetenv            0000000180027dbc     libucrt:fegetenv.obj
 0004:00000dc8       $pdata$fesetenv            0000000180027dc8     libucrt:fesetenv.obj
 0004:00000dd4       $pdata$feholdexcept        0000000180027dd4     libucrt:feholdexcept.obj
 0004:00000dec       $pdata$_write              0000000180027dec     libucrt:write.obj
 0004:00000df8       $pdata$_write$fin$0        0000000180027df8     libucrt:write.obj
 0004:00000e04       $pdata$_write_nolock       0000000180027e04     libucrt:write.obj
 0004:00000e10       $pdata$?write_double_translated_ansi_nolock@@YA?AUwrite_result@?A0x9c548279@@HQEBDI@Z 0000000180027e10     libucrt:write.obj
 0004:00000e1c       $pdata$?write_text_ansi_nolock@@YA?AUwrite_result@?A0x9c548279@@HQEBDI@Z 0000000180027e1c     libucrt:write.obj
 0004:00000e28       $pdata$?write_text_utf16le_nolock@@YA?AUwrite_result@?A0x9c548279@@HQEBDI@Z 0000000180027e28     libucrt:write.obj
 0004:00000e34       $pdata$?write_text_utf8_nolock@@YA?AUwrite_result@?A0x9c548279@@HQEBDI@Z 0000000180027e34     libucrt:write.obj
 0004:00000e40       $pdata$??$common_lseek_nolock@_J@@YA_JH_JH@Z 0000000180027e40     libucrt:lseek.obj
 0004:00000e4c       $pdata$fclose              0000000180027e4c     libucrt:fclose.obj
 0004:00000e58       $pdata$fclose$fin$0        0000000180027e58     libucrt:fclose.obj
 0004:00000e64       $pdata$_fclose_nolock      0000000180027e64     libucrt:fclose.obj
 0004:00000e70       $pdata$_commit             0000000180027e70     libucrt:commit.obj
 0004:00000e7c       $pdata$??$?RV<lambda_b521505b218e5242e90febf6bfebc422>@@AEAV<lambda_6978c1fb23f02e42e1d9e99668cc68aa>@@V<lambda_314360699dd331753a4119843814e9a7>@@@?$__crt_seh_guarded_call@H@@QEAAH$$QEAV<lambda_b521505b218e5242e90febf6bfebc422>@@AEAV<lambda_6978c1fb23f02e42e1d9e99668cc68aa>@@$$QEAV<lambda_314360699dd331753a4119843814e9a7>@@@Z 0000000180027e7c     libucrt:commit.obj
 0004:00000e88       $pdata$?fin$0@?0???$?RV<lambda_b521505b218e5242e90febf6bfebc422>@@AEAV<lambda_6978c1fb23f02e42e1d9e99668cc68aa>@@V<lambda_314360699dd331753a4119843814e9a7>@@@?$__crt_seh_guarded_call@H@@QEAAH$$QEAV<lambda_b521505b218e5242e90febf6bfebc422>@@AEAV<lambda_6978c1fb23f02e42e1d9e99668cc68aa>@@$$QEAV<lambda_314360699dd331753a4119843814e9a7>@@@Z@4HA 0000000180027e88     libucrt:commit.obj
 0004:00000e88       $pdata$?fin$0@?0???$?RV<lambda_bfedae4ebbf01fab1bb6dcc6a9e276e0>@@AEAV<lambda_2fe9b910cf3cbf4a0ab98a02ba45b3ec>@@V<lambda_237c231691f317818eb88cc1d5d642d6>@@@?$__crt_seh_guarded_call@H@@QEAAH$$QEAV<lambda_bfedae4ebbf01fab1bb6dcc6a9e276e0>@@AEAV<lambda_2fe9b910cf3cbf4a0ab98a02ba45b3ec>@@$$QEAV<lambda_237c231691f317818eb88cc1d5d642d6>@@@Z@4HA 0000000180027e88     libucrt:close.obj
 0004:00000e94       $pdata$_setfpstatusword    0000000180027e94     libucrt:_fenvutils.obj
 0004:00000ea0       $pdata$_getfpcontrolword   0000000180027ea0     libucrt:_fenvutils.obj
 0004:00000eac       $pdata$_getfpstatusword    0000000180027eac     libucrt:_fenvutils.obj
 0004:00000eb8       $pdata$_clearfp            0000000180027eb8     libucrt:ieee.obj
 0004:00000ec4       $pdata$common_control87    0000000180027ec4     libucrt:ieee.obj
 0004:00000ed0       $pdata$_ctrlfp$filt$0      0000000180027ed0     libucrt:fpctrl.obj
 0004:00000ed0       $pdata$common_control87$filt$0 0000000180027ed0     libucrt:ieee.obj
 0004:00000edc       $pdata$_call_matherr       0000000180027edc     libucrt:libm_error.obj
 0004:00000ee8       $pdata$_exception_enabled  0000000180027ee8     libucrt:libm_error.obj
 0004:00000ef4       $pdata$_handle_error       0000000180027ef4     libucrt:libm_error.obj
 0004:00000f00       $pdata$__acrt_initialize_fma3 0000000180027f00     libucrt:fma3_available.obj
 0004:00000f0c       $pdata$_log_special_common 0000000180027f0c     libucrt:log_special.obj
 0004:00000f18       $pdata$_log10_special      0000000180027f18     libucrt:log_special.obj
 0004:00000f24       $pdata$_putwch_nolock      0000000180027f24     libucrt:putwch.obj
 0004:00000f30       $pdata$_close              0000000180027f30     libucrt:close.obj
 0004:00000f3c       $pdata$_close_nolock       0000000180027f3c     libucrt:close.obj
 0004:00000f48       $pdata$??$?RV<lambda_bfedae4ebbf01fab1bb6dcc6a9e276e0>@@AEAV<lambda_2fe9b910cf3cbf4a0ab98a02ba45b3ec>@@V<lambda_237c231691f317818eb88cc1d5d642d6>@@@?$__crt_seh_guarded_call@H@@QEAAH$$QEAV<lambda_bfedae4ebbf01fab1bb6dcc6a9e276e0>@@AEAV<lambda_2fe9b910cf3cbf4a0ab98a02ba45b3ec>@@$$QEAV<lambda_237c231691f317818eb88cc1d5d642d6>@@@Z 0000000180027f48     libucrt:close.obj
 0004:00000f60       $pdata$_set_errno_from_matherr 0000000180027f60     libucrt:fpexcept.obj
 0004:00000f6c       $pdata$_raise_exc          0000000180027f6c     libucrt:fpexcept.obj
 0004:00000f78       $pdata$_raise_exc_ex       0000000180027f78     libucrt:fpexcept.obj
 0004:00000f84       $pdata$_clrfp              0000000180027f84     libucrt:fpctrl.obj
 0004:00000f90       $pdata$_ctrlfp             0000000180027f90     libucrt:fpctrl.obj
 0004:00000f9c       $pdata$_statfp             0000000180027f9c     libucrt:fpctrl.obj
 0004:00000fa8       $pdata$_set_statfp         0000000180027fa8     libucrt:fpctrl.obj
 0004:00000fb4       $pdata$__dcrt_lowio_initialize_console_output 0000000180027fb4     libucrt:initcon.obj
 0004:00000fc0       $pdata$__dcrt_terminate_console_output 0000000180027fc0     libucrt:initcon.obj
 0004:00000fcc       $pdata$_IsNonwritableInCurrentImage 0000000180027fcc     LIBCMT:pesect.obj
 0004:00000fd8       $pdata$_IsNonwritableInCurrentImage$filt$0 0000000180027fd8     LIBCMT:pesect.obj
 0005:000000a0       $R000000                   00000001800280a0     gdip.res
 0005:000003b0       $R000310                   00000001800283b0     gdip.res
